:100000000C94592C0C945E2F0C94892F0C94B42FC3
:100010000C94DF2F0C940A300C9435300C94603023
:100020000C948B300C948A2C0C948A2C0C948A2C73
:100030000C948A2C0C948A2C0C948A2C0C948A2C68
:100040000C948A2C0C940FCA0C948A2C0C948A2C35
:100050000C948A2C0C948A2C0C9479BB0C948C2CC8
:100060000C948A2C0C94BAA60C9466A70C948A2C37
:100070000C948A2C0C948A2C0C948A2C0C948A2C28
:100080000C948A2C0C948A2C0C948A2C0C948A2C18
:100090000C948A2C0C948A2C0C948A2C0C948A2C08
:1000A0000C948A2C0C948A2C0C948A2C0C948A2CF8
:1000B0000C948A2C0C948A2C0C948A2C0C948A2CE8
:1000C0000C948A2C0C948A2C0C948A2C0C948A2CD8
:1000D0000C948A2C0C948A2C0C948A2C0C948A2CC8
:1000E0000C948A2CD42DD92DDE2DE82DF22D6B2EDB
:1000F000FC2D042E0C2E162E202E2A2E392E432EA9
:100100006B2E4D2E572E612E8F2E922E812E852EE8
:100110008B2EC92E962E9A2EA02EA42EA82EAE2E51
:10012000B22EB62EC92EBC2EC02EC42E73625362C0
:10013000596256625C625F6262626E626562806290
:1001400068626B62F5A3F3A317A414A412A449A4D4
:1001500046A444A4A2A470A46DA46BA4EDA6F3A627
:1001600004A70FA717A72CA71BA72CA71FA723A778
:100170002CA729A7084AD73B3BCE016E84BCBFFD04
:10018000C12F3D6C74319ABD56833DDA3D00C77F67
:1001900011BED9E4BB4C3E916BAAAABE0000008000
:1001A0003F05A84CCDB2D44EB93836A9020C50B98F
:1001B000918688083CA6AAAA2ABE000000803F00BB
:1001C0000D944E2C0D94A1480D9406050D944E4DA2
:1001D0004E414E494E495459494E46CDCCCC3D0A2C
:1001E000D7233C17B7D13877CC2B329595E6241F0F
:1001F000B14F0A000020410000C84200401C4620C8
:10020000BCBE4CCA1B0E5AAEC59D7400000A0B0240
:10021000090C0D0E08070304010000000000000097
:1002200000000000000000000000000000000000CE
:10023000000000000000001211100000000000008B
:1002400000000000000000000000000000000000AE
:1002500000010210202008081020401020408002D9
:1002600001020108040201010204081020408080FC
:100270004020100804020180040201804020100880
:100280000402010804020101020408102040800158
:100290000204081020408005050505070508080828
:1002A00008020202020A0A08080404040401010107
:1002B000010101010103030303030303030407070F
:1002C000070C0C0C0C0C0C0C0C02020202060606AD
:1002D00006060606060B0B0B0B0B0B0B0B00002088
:1002E000002300260029002C002F0032000001000E
:1002F0000003010601090100002200250028002B4F
:10030000002E003100340002010000050108010B3D
:100310000100002100240027002A002D00300033B6
:100320000001010000040107010A0101060D00FEA1
:1003300009016602D620FFFE0BFE0AFE0D006022B8
:100340001969808080808080800080183363A0A03D
:10035000A00357675050F850F85050025969207860
:10036000A0A0702828F02002596948A85010204009
:1003700050A89002586840A0A040A0989068281308
:1003800063808080113B6B20404080808080804073
:100390004020113B6B8040402020202020404080A6
:1003A00006556520A870A8200455652020F8202057
:1003B000113363604080065161F811336340E040BF
:1003C00002596908081010204040808002596920B5
:1003D00050888888888850200259692060A0202091
:1003E000202020F80259697088880810204080F881
:1003F000025969F8081020700808887002596910BD
:100400001030505090F81010025969F88080B0C830
:100410000808887002596970888080F08888887020
:10042000025969F8081010202040404002596970B4
:100430008888887088888870025969708888887868
:100440000808887011386840E040000040E0401122
:10045000386840E040000060408002596908102080
:10046000408040201008045464F80000F8025969E4
:100470008040201008102040800259697088880848
:10048000102020002002596970888898A8A8B080A0
:10049000780259692050888888F8888888025969C4
:1004A000F048484870484848F00259697088808090
:1004B0008080808870025969F04848484848484818
:1004C000F0025969F8808080F0808080F8025969D4
:1004D000F8808080F08080808002596970888080F8
:1004E000809888887002596988888888F888888800
:1004F00088123969E040404040404040E00259697C
:10050000381010101010109060025969888890A05F
:10051000C0A0908888025969808080808080808017
:10052000F80259698888D8A8A888888888025969F3
:1005300088C8C8A8A8989888880259697088888847
:100540008888888870025969F0888888F08080805F
:1005500080015A6A70888888888888A8700802593B
:1005600069F0888888F0A09088880259697088802E
:10057000807008088870025969F820202020202007
:10058000202002596988888888888888887002595C
:100590006988888888505050202002596988888846
:1005A00088A8A8A8A850025969888850502050509F
:1005B00088880259698888505020202020200259BC
:1005C00069F808101020404080F8113B6BE08080F3
:1005D00080808080808080E0025969808040402057
:1005E00010100808113B6BE0202020202020202044
:1005F00020E0085363205088015161F82A2262806C
:100600004002566670087888986802596980808030
:10061000F088888888F0025666708880808870022A
:10062000596908080878888888887802566670882A
:10063000F880887002596930484040F0404040409E
:1006400000586870888888780888700259698080A6
:1006500080B0C8888888881238684000C040404010
:1006600040E0004A6A1000301010101090906002B4
:10067000596980808090A0C0A09088123969C040DC
:10068000404040404040E0025666D0A8A8A8A88854
:10069000025666B0C888888888025666708888883E
:1006A0008870005868F0888888F0808080005868DA
:1006B0007888888878080808025666B0C8808080E4
:1006C000800256667088601088700258684040F05A
:1006D00040404048300256668888888898680256AC
:1006E000668888885050200256668888A8A8A85036
:1006F000025666885020205088005868888888985C
:1007000068088870025666F810204080F8015B6B1C
:100710001820202020C02020202018221969808045
:1007200080808080808080015B6BC020202020182A
:1007300020202020C008536348A890FFFFFFFFFF40
:10074000FFFFFFFFFFFFFFFFFFFFFFFFFFFFFFFFB9
:10075000FFFFFFFFFFFFFFFFFFFFFFFF0D00602216
:1007600019698000808080808080800358682070B4
:10077000A8A0A0A8702002596930484040E040403D
:1007800048B003566688705050708802596988884E
:100790005050F820F8202022196980808080008045
:1007A000808080124A6A60908060909060109060B3
:1007B0001A3262A0A00359697088A8D8C8D8A8883E
:1007C00070045767700878887800F80356662850D8
:1007D000A0A05028045363F80808163161E00359BB
:1007E000697088E8D8D8E8D888700A5161F8174449
:1007F00064609090600357672020F8202000F8077D
:10080000356540A02040E007356540A04020C02A63
:10081000226240800058688888888898E880800232
:10082000596978E8E8E8E868282828262161C02086
:100830002262408007356540C04040E00457677041
:100840008888887000F8035666A050282850A002B7
:100850005A6A40C04040E00818283808025A6A40E6
:10086000C04040E01028081038025A6A40A04020DA
:10087000A0481828380802596920002020408088A4
:100880008870025A6A40200020508888F8888802C0
:100890005A6A10200020508888F88888025A6A30E6
:1008A000480020508888F88888025A6A285000201A
:1008B000508888F88888025A6A50500020508888EA
:1008C000F88888025A6A20502020508888F8888842
:1008D00002596958A0A0A0B0E0A0A0B8005B6B705E
:1008E00088808080808088702040025A6A40200082
:1008F000F88080F08080F8025A6A102000F880802A
:10090000F08080F8025A6A304800F88080F08080D9
:10091000F8025A6A505000F88080F08080F8123A4D
:100920006A804000E04040404040E0123A6A204087
:1009300000E04040404040E0124A6A609000E040E1
:1009400040404040E0123A6AA0A000E040404040F1
:1009500040E0025969F0484848E8484848F0025ADF
:100960006A2850008888C8A8988888025A6A402057
:100970000070888888888870025A6A102000708801
:100980008888888870025A6A304800708888888809
:100990008870025A6A285000708888888888700297
:1009A0005A6A505000708888888888700355658816
:1009B00050205088015B6B08709898A8A8A8C8C8F8
:1009C0007080025A6A40200088888888888870026F
:1009D0005A6A10200088888888888870025A6A308D
:1009E000480088888888888870025A6A5050008831
:1009F000888888888870025A6A1020008888502069
:100A000020202002596980F0888888F08080800248
:100A10005969609090A0A0908888B00259694020E0
:100A2000007008788898680259691020007008786A
:100A30008898680259693048007008788898680278
:100A40005969285000700878889868025969505090
:100A500000700878889868025A6A30483000700838
:100A600078889868025666702870A0A85000586868
:100A7000708880808870204002596940200070880A
:100A8000F88088700259691020007088F88088709A
:100A90000259693048007088F8808870025969509E
:100AA00050007088F8808870123969804000C0401A
:100AB000404040E0123969204000C040404040E0E2
:100AC000124969609000C040404040E0123969A07E
:100AD000A000C040404040E0025A6A5020601070C0
:100AE0008888888870025969285000B0C88888882A
:100AF0008802596940200070888888887002596986
:100B00001020007088888888700259693048007009
:100B10008888888870025969285000708888888879
:100B20007002596950500070888888887003576730
:100B3000202000F8002020015868087098A8A8C854
:100B40007080025969402000888888889868025916
:100B500069102000888888889868025969304800A0
:100B600088888888986802596950500088888888E1
:100B70009868005B6B1020008888889868088870E7
:100B8000005A6A8080B0C88888C8B08080005B6BDB
:100B9000505000888888986808887001050700FE12
:100BA0000500FB01F220FFFE05FE05FE02004002EB
:100BB00015258080800080053242A0A00255655036
:100BC000F850F8500146562070C030E020025565BC
:100BD0009010204048025565608068906805122298
:100BE000808002253540808080400225358040404D
:100BF0004080043343A040A003334340E04001223F
:100C0000324080043141E002112180025565081014
:100C10002040800245556090909060022535C0408C
:100C2000404040024555E0106080F0024555E0101C
:100C30006010E00245552060A0F020024555F0808C
:100C4000E010E00245556080E09060024555F010EC
:100C5000204040024555609060906002455560908C
:100C600070106003132380008002142480008080B1
:100C70000235452040804020033343E000E0023548
:100C8000458040204080024555E0106000400255FC
:100C9000657088B8A870024555609090F090024544
:100CA00055E090E090E0023545608080806002452C
:100CB00055E0909090E0023545E080E080E002351C
:100CC00045E080E080800245557080B0907002451C
:100CD000559090F09090023545E0404040E002454C
:100CE00055301010906002455590A0C0A09002357C
:100CF0004580808080E002556588D8A888880245B4
:100D00005590D0B09090024555609090906002450B
:100D100055E09090E08001465660909090601002FF
:100D20004555E09090E09002455570806010E002DB
:100D30003545E0404040400245559090909060021B
:100D400045559090A0A04002556588A8A8A85002DB
:100D500045559090609090024555909070106002BB
:100D60003545E0204080E0022535C0808080C0020B
:100D700055658040201008022535C0404040C00520
:100D8000324240A0024151F00522328040024454D8
:100D90007090907002455580E09090E0023444607D
:100DA000808060024555107090907002445460B08D
:100DB000C0600235452040E04040004656709090AB
:100DC00070106002455580E09090900215258000DB
:100DD00080808000273740004040404080024555D9
:100DE0008090A0E09002152580808080800254646D
:100DF000F0A8A8A8024454E0909090024454609057
:100E00009060004656E09090E080800046567090DA
:100E100090701010023444A0C0808002445470C00E
:100E200030E002354540E04040200244549090902C
:100E3000700244549090A040025464A8A8505002FC
:100E40003444A04040A0004656909090701060023C
:100E50004454F02040F00235456040804060021567
:100E6000258080808080023545C0402040C00542FA
:100E70005250A0FFFFFFFFFFFFFFFFFFFFFFFFFF3D
:100E8000FFFFFFFFFFFFFFFFFFFFFFFFFFFFFFFF72
:100E9000FFFFFFFF020040FFFFFFFFFFFFFFFFFF1D
:100EA000FFFFFFFFFFFFFFFFFFFFFFFFFFFFFFFF52
:100EB000FFFFFFFFFFFFFFFFFFFFFFFFFFFFFFFF42
:100EC000FFFFFFFFFFFFFFFFFFFFFFFFFFFFFFFF32
:100ED000FFFFFFFFFFFFFFFFFFFFFFFFFFFFFFFF22
:100EE000FFFFFFFFFFFFFFFFFFFFFFFFFFFFFFFF12
:100EF000FFFFFFFFFFFF01050800FF06012102358C
:100F000020FFFF07FF06FF09005022165680808051
:100F1000800080153353A0A0A00257575050F850BE
:100F2000F850500257572070A07028702013355584
:100F300080A040A02002475740A0A040A0A050257C
:100F40001353808080122656408080808040122675
:100F5000568040404040800245559060F0609002CD
:100F600055552020F8202011335360408004415112
:100F7000F011335340E0400246561010204080806C
:100F800012365640A0A0A0A04012365640C04040A5
:100F900040E00246566090106080F0024656F02015
:100FA000601090600246562060A0F0202002465655
:100FB000F080E01090600246566080E09090600201
:100FC0004656F010202040400246566090609090B7
:100FD00060024656609090701060122555C0C000A7
:100FE000C0C0113656606000604080123656204006
:100FF00080804020034353F000F01236568040209A
:1010000020408012365640A0204000400158583001
:101010004898A8A8904030024656609090F0909072
:10102000024656E090E09090E00246566090808044
:101030009060024656E090909090E0024656F08014
:10104000E08080F0024656F080E0808080024656C4
:10105000609080B090600246569090F09090901210
:101060003656E040404040E002465670202020A026
:101070004002465690A0C0A0A090024656808080B4
:101080008080F002465690F0F09090900246569084
:10109000D0F0B0B0900246566090909090600246BA
:1010A00056E09090E08080014757609090D0B0600B
:1010B00010024656E09090E09090024656609040B4
:1010C000209060123656E040404040400246569024
:1010D000909090906002465690909090606002468A
:1010E00056909090F0F090024656909060609090EC
:1010F000025656888850202020024656F010204084
:1011000080F0123656E080808080E0024656808073
:1011100040201010123656E020202020E0163252D7
:1011200040A0014151F01622528040024454709078
:1011300090700246568080E09090E01234546080B7
:10114000806002465610107090907002445460B057
:10115000C060024656205040E04040014555609036
:101160007010600246568080E09090901236564093
:1011700000C04040E01137572000202020A040024E
:101180004656808090E09090123656C040404040D5
:10119000E0025454D0A8A8A8024454E090909002D1
:1011A000445460909060014555E090E08080014596
:1011B000557090701010024454A0D08080123454A6
:1011C00060C020C00246564040E0405020024454D7
:1011D00090909070123454A0A0A04002545488A85B
:1011E000A8500244549060609001455590907090D2
:1011F00060024454F02040F0024757304020C020A5
:101200004030221656808080808080024757C02060
:1012100040304020C006425250A0FFFFFFFFFFFFBA
:10122000FFFFFFFFFFFFFFFFFFFFFFFFFFFFFFFFCE
:10123000FFFFFFFFFFFFFFFFFFFFFF090050221628
:10124000568000808080800146562070A0A07020CB
:101250000246562050E04050A0025555887050700C
:10126000880256568850F820F82022175780808030
:10127000008080800247577080E0907010E0173146
:1012800051A002565670A8C8C8A87014355560A061
:101290006000E003435350A050123353E020201469
:1012A0003151E002565670E8D8E8D870173151E055
:1012B00015335340A04012355540E04000E014354E
:1012C0005540A02040E0143555C020C020C0162253
:1012D000524080014555909090E08002565678E843
:1012E000E868282824115180112252408014355575
:1012F00040C04040E014355540A04000E003435357
:10130000A050A0024757808080A060F0200247577D
:101310008080A0D010207002475780408060A0F0ED
:101320002012365640004080A040024757402060BF
:1013300090F0909002475720406090F090900247C4
:101340005760906090F0909002475750A06090F0E6
:10135000909002475790006090F09090024757603D
:10136000906090F0909002465670A0A0F0A0B0015E
:101370004757609080809060400247574020F0803F
:10138000E080F00247572040F080E080F0024757AD
:101390006090F080E080F00247579000F080E0809D
:1013A000F01237578040E0404040E012375720406D
:1013B000E0404040E012375740A0E0404040E0129B
:1013C0003757A000E0404040E00256567048E848D9
:1013D000487002475750A090D0B0909002475740B5
:1013E00020609090906002475720406090909060FD
:1013F0000247576090609090906002475750A060FD
:1014000090909060024757900060909090601233E7
:1014100053A040A002465670B0B0D0D0E00247576B
:10142000402090909090600247572040909090907C
:1014300060024757609090909090600247579000EC
:1014400090909090600257571020885020202002E2
:10145000465680E09090E0800246566090A0A090B2
:10146000A0024757402000709090700247572040DC
:10147000007090907002475720500070909070025A
:10148000475750A0007090907002465650007090E0
:10149000907002475760906070909070025454F0C2
:1014A00068B0781135556080806040024757402011
:1014B0000060B0C06002475720400060B0C06002CA
:1014C000475760900060B0C060024656500060B060
:1014D000C060123757804000C04040E012375720AC
:1014E0004000C04040E012375740A000C04040E0FC
:1014F000123656A000C04040E0024757A040A0105E
:1015000070906002475750A000E0909090024757BB
:10151000402000609090600247572040006090900B
:10152000600247576090006090906002475750A05B
:101530000060909060024656900060909060123576
:10154000554000E0004002445470B0D0E0024757DC
:10155000402000909090700247572040009090905B
:10156000700247576090009090907002465690002D
:1015700090909070014858204000909070906001C9
:1015800047578080E090E08080014757900090901E
:1015900070906025753A2530327500253032753AE5
:1015A0002530327500202020200025202000252015
:1015B000002531640025326400253364002534643D
:1015C0000025356400253664000000007E006000C0
:1015D000600060F87ECC60CC60CC60F860CC00CC61
:1015E00000CC00CC00000000000000FE7F0E702642
:1015F00064724E7A5E324C8241324C7A5E724E2672
:10160000640E70FE7F000000000000FE7F0E70C6BA
:1016100063C24382411A58BA5D1A588241C243C616
:10162000630E70FE7F00000000000088088808102C
:1016300011202220221011880888081011000000B3
:1016400000000000000000000000002022101188AF
:10165000088808101120222022101188080000009C
:10166000000000000000000000000000000000007A
:10167000000000000000000000000000000000FE6C
:101680007FFE7F06600000000000000000F00FF801
:101690001FF81FF81FF00FF00FF81FF81FF81FE0DA
:1016A00007C00380010000000030484830457272D6
:1016B0003A207574663820666F6E74206E6F7420E1
:1016C000696E697469616C697A65642E004572722D
:1016D0003A207574663820666F6E74206E6F7420C1
:1016E000696E697469616C697A65642E004572720D
:1016F0003A207574663820666F6E74206E6F7420A1
:10170000696E697469616C697A65642E00506C65F4
:10171000617365207265736574005052494E54457B
:10172000522048414C544544007F80FFC0FFC0FF19
:10173000C07F807F80FFC0FFC0FFC03F001E000C45
:1017400000FFFFFF0E000E000E000E000E000E0048
:101750000E000E007FC03F801F000E00040004003A
:101760000E001F003F807FC00E000E000E000E0016
:101770000E000E000E000E0000FE0003FF80078327
:10178000C00E01C00E00E01C00E07F00E03E00E063
:101790001C00E00800E00000E00001C00E01C00FE6
:1017A000078007FF0001FC0001FC0007FF000F0796
:1017B000800E01C00001C00000E00800E01C00E055
:1017C0003E00E07F00E01C00E00E00E00E01C007DC
:1017D00083C003FF8000FE0000060C00FE07022607
:1017E00003BC017FFE08FE08FE0508080600004055
:1017F000F0C88888987810050808060000C0F888A6
:1018000088888888F80505050600012030F8302012
:101810000508080600002070F820202020E00509B7
:10182000090600FF2070A8A8B88888702005060661
:10183000060001E08CEA8C8A0A0509090600FFF817
:10184000A88888888888A8F8050A0A0600FE20501B
:1018500050505088A8A8887003030306000340A0D6
:1018600040FFFFFFFFFFFFFFFFFFFFFFFFFFFFFF47
:10187000FFFFFFFFFFFFFF0000000605FF01070756
:10188000060200808080808000800303030601053B
:10189000A0A0A005060606000050F85050F850051C
:1018A00009090600FF2070A8A07028A8702005076D
:1018B00007060000C8C810204098980507070600D2
:1018C0000040A0A040A890680103030602058080A4
:1018D000800309090601FF204040808080404020AD
:1018E0000309090601FF8040402020204040800578
:1018F000070706000020A8702070A820050505062F
:1019000000012020F820200203030601FFC04080D0
:10191000050101060003F8020202060100C0C0052D
:101920000707060000081010204040800507070642
:101930000000708898A8C888700307070601004057
:10194000C040404040E005070706000070880810CE
:101950002040F8050707060000F8081030088870D6
:1019600005070706000010305090F8101005070713
:10197000060000F880F008088870050707060000D8
:10198000304080F0888870050707060000F80810CE
:1019900010202020050707060000708888708888BE
:1019A0007005070706000070888878081060020537
:1019B00005060100C0C000C0C00206060601FFC047
:1019C000C000C04080030505060101204080402082
:1019D000050303060002F800F8030505060101806F
:1019E0004020408005070706000070881020200076
:1019F000200507070600007088B8A8B880700507A2
:101A000007060000708888F88888880507070600A0
:101A100000F04848704848F0050707060000708845
:101A20008080808870050707060000F04848484815
:101A300048F0050707060000F88080F08080F80570
:101A40000707060000F88080F08080800507070601
:101A5000000070888080988870050707060000885D
:101A60008888F8888888030707060100E04040401E
:101A70004040E00507070600003810101010906085
:101A80000507070600008890A0C0A09088050707FA
:101A9000060000808080808080F80507070600002F
:101AA00088D8A8888888880507070600008888C81D
:101AB000A8988888050707060000708888888888A5
:101AC00070050707060000F08888F0808080050711
:101AD0000706000070888888A89068050707060038
:101AE00000F08888F0A0908805070706000070883D
:101AF0008070088870050707060000F82020202065
:101B000020200507070600008888888888887005D7
:101B100007070600008888888850502005070706B8
:101B2000000088888888A8A8500507070600008854
:101B300088502050888805070706000088885020B4
:101B4000202020050707060000F80810204080F834
:101B50000309090601FFE080808080808080E00525
:101B600007070600008040402010100803090906FE
:101B700001FFE020202020202020E00503030600B4
:101B8000052050880501010600FEF8030303060145
:101B90000580402005050506000070087888780556
:101BA00007070600008080F0888888F00505050694
:101BB000000070808088700507070600000808781C
:101BC000888888780505050600007088F080700513
:101BD0000707060000304840E04040400507070680
:101BE00000FE708888887808700507070600008066
:101BF00080F0888888880307070601004000C040FD
:101C00004040E00409090601FE10003010101010D9
:101C1000906005070706000080808890E0908803A8
:101C20000707060100C04040404040E005050506AA
:101C30000000D0A8A8A8A8050505060000B0C8881F
:101C400088880505050600007088888870050707E4
:101C50000600FEF0888888F080800507070600FEF1
:101C600078888888780808050505060000B0C880CF
:101C7000808005050506000078807008F0050707DC
:101C80000600002020F82020201805050506000089
:101C9000888888986805050506000088888850208F
:101CA0000505050600008888A8A85005050506005A
:101CB0000088502050880507070600FE8888885055
:101CC000204080050505060000F8102040F80309B3
:101CD000090601FF204040408040404020010909A2
:101CE0000602FF8080808080808080800309090652
:101CF00001FF804040402040404080050303060033
:101D00000248A890FF1FFFFFFFFFFFFF60000000D9
:101D10000001FF400000000000FF80000000000004
:101D20007F83CF00000C303F87FF80000C301F8680
:101D30007980000C000F8C30C7838C30E78C30CF5B
:101D4000C7CC31F38C30DCECEC33B98C30D86C6C14
:101D500033198C30D06C0C33198C30D86C0C33198F
:101D60008C30DC6C0E3B198C30CF7C079F198C308B
:101D7000C77C038F194000000000000260000000D3
:101D80000000061FFFFFFFFFFFF80000000000003B
:101D90000000000000000000000000000000000043
:101DA000000000000000000000000000000C000027
:101DB00000000000000C0000000000000012000005
:101DC00000000000002300000000000000210000CF
:101DD00000000000004C800000000000005E800059
:101DE00000000000009240000000000000A1400040
:101DF000000000000121200000000000027F900090
:101E000000000000020010000000000007FFF800C2
:101E100000000000040008000000000008000400AA
:101E20000000000008000600000000001000020092
:101E300000000000301E010000000000207F810033
:101E40000000000041FFE0800000000043FCF08043
:101E500000000000873B7840000000018EDBFC6042
:101E6000000000010FEBCC20000000021FEDB610B7
:101E7000000000021FDEB6100000000439CD7F080C
:101E80000000000436E0FF08000000087EC0BB84AC
:101E9000000000187F005D86000000107FC0ED820A
:101EA000000000203CC07301000000203B337F0194
:101EB000000000701BE77E03800000C81DEEDE04FA
:101EC000C00000880FDEDC04400001240FDF3C0965
:101ED0002000012607DBF8192000027203E7F01347
:101EE0009000025101FFE02290000489007F8024CD
:101EF00048000904801E004824000BFE400000DF5B
:101F0000F40010004000008002001FFFFFFFFFFFF1
:101F1000FE000000000000000000000000000000C3
:101F2000000000000000000000001022103C3C0EE9
:101F30001F00102210042211040010221008221188
:101F40000400102210083C1104001022101022116D
:101F5000040010221020221104001E1C1E3C3C0E06
:101F6000040000000000000000000000000000006D
:101F70000000000000000000000000000000000061
:101F80000000000000000000000000000000000051
:101F90000000000000000000000000000000000041
:101FA0000000000000000000000000000000000031
:101FB0000000000000000000000000000000000021
:101FC000000000000000000000060900FE06018974
:101FD00002FE20FFFE07FE06FE00000006000701CD
:101FE000060606020080808080008003030306014D
:101FF00003A0A0A00507070600FF5050F850F850B6
:10200000500509090600FE2070A8A07028A87020BD
:102010000608080600FF40A8481020485408050795
:10202000070600FF60909060989068010303060225
:10203000038080800207070602FF40808080808046
:10204000400207070602FF804040404040800505EF
:10205000050600008850F850880505050600002098
:1020600020F820200204040602FEC0404080050142
:1020700001060002F8020202060200C0C0040606C1
:102080000601001010204080800406060601006052
:10209000909090906003060606010040C0404040CA
:1020A000E00406060601006090102040F0040606D9
:1020B000060100F020601010E00506060600001082
:1020C000305090F810040606060100F080E0101071
:1020D000E00406060601006080E0909060040606B9
:1020E000060100F0101020404004060606010060C2
:1020F0009060909060040606060100609090701059
:1021000060020505060200C0C000C0C00207070645
:1021100002FEC0C000C04040800505050600001852
:1021200060806018050303060001F800F805050546
:10213000060000C0300830C00407070601006090A8
:1021400010604000400506060600007090A8B080B0
:1021500070050606060000205088F88888050606E7
:10216000060000F088F08888F0040606060100608A
:102170009080809060040606060100E090909090A8
:10218000E0040606060100F080E08080F004060608
:10219000060100F080E080808004060606010060F1
:1021A0009080B090600406060601009090F0909038
:1021B00090030606060100E040404040E0050606A8
:1021C000060000381010109060040606060100900A
:1021D000A0C0A09090040606060100808080808048
:1021E000F005060606000088D8A8A8888804060618
:1021F00006010090D0B09090900506060600007091
:102200008888888870040606060100E09090E080C7
:10221000800407070601FF609090D0B060100406AC
:1022200006060100E09090E090900406060601008A
:10223000609040209060050606060000F8202020EF
:1022400020200406060601009090909090600406FD
:1022500006060100909090F06060050606060000FA
:102260008888A8A8D888050606060000885020207F
:1022700050880506060600008888502020200406A5
:1022800006060100F010204080F00306060601005B
:10229000E080808080E00406060601008080402007
:1022A0001010030606060100E020202020E00503B0
:1022B000030600032050880501010600FEF8020213
:1022C000020602048040040404060100709090702D
:1022D0000406060601008080E09090E004040406F5
:1022E00001007080807004060606010010107090D6
:1022F000907004040406010060B0C0700406060675
:102300000100205040E040400406060601FE6090B7
:10231000907010600406060601008080E0909090A6
:102320000306060601004000C04040E0030808061E
:1023300001FE200060202020A040040606060100C7
:102340008080A0C0A090030606060100C040404067
:1023500040E0050404060000D0A8A8880404040690
:102360000100E090909004040406010060909060E9
:102370000406060601FEE09090E080800406060652
:1023800001FE709090701010040404060100A0D0AB
:10239000808004040406010070C030E004060606D4
:1023A00001004040E04050200404040601009090E9
:1023B0009070040404060100909060600504040617
:1023C000000088A8A85004040406010090606090F2
:1023D0000406060601FE90909070906004040406C6
:1023E0000100F02040F00307070601002040408074
:1023F0004040200107070602FF80808080808080A7
:10240000030707060100804040204040800402028C
:1024100006010350A0FFFFFFFFFFFFFFFFFFFFFFCD
:10242000FFFFFFFFFFFFFFFFFFFFFFFFFFFFFFFFBC
:10243000FFFFFFFFFFFF0000000600070106060682
:1024400002008000808080800406060601FF207064
:10245000A0A070200507070600FF304840F040406C
:10246000F8050505060000A8508850A805060606D0
:1024700000008850F820F8200107070602FF80803E
:1024800080008080800407070601FF7080609060F4
:1024900010E0030101060105A00607070600007809
:1024A0008494A494847803050506010160A060006B
:1024B000E00505050600002850A050280403030687
:1024C0000100F01010040101060102F006070706E2
:1024D00000007884B4A4A48478040101060105F006
:1024E0000403030601026090600507070600FF2051
:1024F00020F8202000F803050506010140A0204037
:10250000E0030505060101C0204020C002020206CA
:10251000020440800405050601FF9090B0D08005BC
:10252000060606000078E8E868282801010106028E
:1025300002800202020602FE408003050506010138
:1025400040C04040E003050506010140A04000E016
:10255000050505060000A0502850A0050808060043
:10256000FF40C04050703078100508080600FF405A
:10257000C04050680810380508080600FFC0204019
:1025800030F030781004070706010020002060803A
:1025900090600507070600004020205070888805DD
:1025A00007070600001020205070888805070706DE
:1025B000000020502050708888050707060000287A
:1025C00050205070888805070706000050002050F2
:1025D0007088880507070600002050205070888802
:1025E00005060606000078A0F0A0A0B804080806BA
:1025F00001FE609080809060204004070706010083
:102600004020F080E080F00407070601002040F041
:1026100080E080F00407070601002050F080E08091
:10262000F00407070601005000F080E080F0030787
:10263000070601008040E0404040E0030707060134
:10264000002040E0404040E003070706010040A0B2
:10265000E0404040E0030707060100A000E04040E2
:1026600040E00506060600007048E8484870040788
:102670000706010050A090D0B09090040707060113
:102680000040206090909060040707060100204001
:1026900060909090600407070601002050609090C1
:1026A000906004070706010050A0609090906004BD
:1026B0000707060100500060909090600505050630
:1026C000000088502050880408080601FF1070B0F0
:1026D000B0D0D0E080040707060100402090909021
:1026E00090600407070601002040909090906004DD
:1026F000070706010020509090909060040707069D
:1027000001005000909090906005070706000010AF
:1027100020885020202004060606010080E09090CA
:10272000E0800406060601006090A0A090A00407C7
:102730000706010040200070909070040707060112
:1027400000204000709090700407070601002050A0
:10275000007090907004070706010050A000709070
:1027600090700406060601005000709090700407F7
:1027700007060100205020709090700504040600A8
:102780000070A8B0780406060601FE7080807020F4
:102790004004070706010040200060B0C070040735
:1027A0000706010020400060B0C070040707060162
:1027B0000020500060B0C070040606060100500002
:1027C00060B0C070030707060100804000C04040B1
:1027D000E0030707060100204000C04040E0030777
:1027E0000706010040A000C04040E00306060601C5
:1027F00000A000C04040E004070706010030601060
:102800007090906004070706010050A000E09090CF
:1028100090040707060100402000609090600407C4
:102820000706010020400060909060040707060141
:10283000002050006090906004070706010050A03F
:1028400000609090600406060601005000609090C1
:10285000600505050600002000F8002004040406B9
:10286000010070B0D0E0040707060100402000908E
:10287000909070040707060100204000909090702F
:10288000040707060100205000909090700406068F
:102890000601005000909090700409090601FE2086
:1028A00040009090907090600408080601FE8080BF
:1028B000E09090E080800408080601FE50009090AF
:1028C00090709060536E346B3300496E766164652E
:1028D000727300427269636B6F7574004D61696E4B
:1028E000005072696E742066726F6D205344005000
:1028F00072696E742066726F6D20534400022E2E32
:10290000004D61696E005072696E740043616E63C0
:10291000656C005374617274207072696E7420006B
:102920003F00536D6F6F7468696E6700536D6F6F12
:102930007468696E67005A005A00590059005800BF
:102940005800436F7272656374696F6E00436F72F3
:1029500072656374696F6E004D61696E0046696CE3
:10296000616D656E74004261636B6C6173680053E6
:10297000746570732F6D6D004A65726B00416363FF
:10298000656C65726174696F6E0056656C6F636922
:10299000747900436F6E66696775726174696F6EF2
:1029A000004573746570732F6D6D004573746570A9
:1029B000732F6D6D005A73746570732F6D6D005AAF
:1029C00073746570732F6D6D005973746570732F18
:1029D0006D6D005973746570732F6D6D005873744D
:1029E0006570732F6D6D005873746570732F6D6D06
:1029F00000416476616E6365642053657474696E2A
:102A000067730056652D6A65726B0056652D6A65A1
:102A1000726B00567A2D6A65726B00567A2D6A6564
:102A2000726B0056792D6A65726B0056792D6A6556
:102A3000726B0056782D6A65726B0056782D6A6548
:102A4000726B00416476616E6365642053657474D3
:102A5000696E677300416D6178204500416D617852
:102A6000204500416D6178205A00416D6178205AFF
:102A700000416D6178205900416D61782059004115
:102A80006D6178205800416D6178205800412D74A7
:102A9000726176656C00412D74726176656C0041DF
:102AA0002D7265747261637400412D726574726178
:102AB000637400416363656C00416363656C00414E
:102AC0006476616E6365642053657474696E6773C0
:102AD000005654726176206D696E005654726176AC
:102AE000206D696E00566D696E00566D696E0056F8
:102AF0006D6178204500566D6178204500566D6106
:102B000078205A00566D6178205A00566D61782001
:102B10005900566D6178205900566D617820580033
:102B2000566D6178205800416476616E636564205B
:102B300053657474696E6773004C6F6164206D6DCA
:102B4000004C6F6164206D6D00556E6C6F61642088
:102B50006D6D00556E6C6F6164206D6D0041647623
:102B6000616E6365204B00416476616E6365204B46
:102B700000416476616E6365642053657474696EA8
:102B800067730044697361626C652073746570706B
:102B9000657273004D3834004175746F2D63616C3C
:102BA000696272617465004D31313720537461720E
:102BB00074696E67204175746F2D43616C69627230
:102BC0006174696F6E0A54300A4D323138205431C5
:102BD00020583433205930205A300A4732380A4DB1
:102BE000313137204C6576656C696E67205820411D
:102BF0007869730A473020583135302046393939E1
:102C0000390A473238205A300A4D313137204C6565
:102C100076656C696E6720646F6E652E0A47313287
:102C20000A4D3131372043616C6962726174696E9B
:102C3000672E2E2E0A473432350A4D3530300A4D74
:102C40003131372043616C6962726174696F6E2043
:102C500064617461207361766564004C6576656CAF
:102C600020582041786973004D313137204C65760A
:102C7000656C696E67205820417869730A47302077
:102C8000583135302046393939390A473238205AD7
:102C9000300A4D313137204C6576656C696E67209E
:102CA000646F6E652E0A004175746F20686F6D65E4
:102CB00000473238004D6F76652061786973004DAA
:102CC00061696E00457874727564657220004175A3
:102CD000746F20686F6D6500473238004D6F766500
:102CE000205A004D6F76652059004D6F766520584B
:102CF000004D6F76656D656E74004578747275640D
:102D0000657220004D6F766520302E316D6D004D5F
:102D10006F766520316D6D004D6F76652031306DB9
:102D20006D004D6F7665206178697300486F74653A
:102D30006E6420746F6F20636F6C640045787472EA
:102D40007564657220004D6F7665205A004D6F7670
:102D5000652059004D6F76652058004D6F766520CF
:102D60005A004D6F76652059004D6F7665205800EA
:102D70005761697420666F720066696C616D656E7B
:102D8000742070757267650000506C656173652012
:102D9000776169742E005072657373206275747464
:102DA0006F6E00746F20726573756D652070726947
:102DB0006E74005761697420666F720066696C6199
:102DC0006D656E74206C6F616400496E736572741A
:102DD0002066696C616D656E7400616E642070724E
:102DE00065737320627574746F6E00746F20636F07
:102DF0006E74696E756500507265737320627574C8
:102E0000746F6E00746F2068656174206E6F7A7ADB
:102E10006C65004E6F7A7A6C652068656174696EC6
:102E20006700506C6561736520776169742E2E2E82
:102E3000005761697420666F720066696C616D6528
:102E40006E7420756E6C6F616400576169742066E2
:102E50006F720066696C616D656E74206368616E87
:102E6000676500746F207374617274005061726BD7
:102E7000696E672E2E2E004368616E67696E67204B
:102E800046696C616D656E7400554E4C4F4144202F
:102E900046494C414D454E54004C4F414420464913
:102EA0004C414D454E540020204E6F7A7A6C653A65
:102EB00020002000456E642066696C616D656E744B
:102EC000206368616E6765005075726765206D6F7D
:102ED000726500004368616E67652066696C616DAC
:102EE000656E7400556E6C6F61642066696C616D0F
:102EF000656E74004C6F61642066696C616D656E0F
:102F000074004D36303020423020542564004D3757
:102F10003032203B2564004D373032205425640088
:102F20004D373031205425640050726568656174F6
:102F300020437573746F6D0050726568656174200D
:102F4000437573746F6D00507265686561742041DC
:102F50004253005072656865617420504C410042D4
:102F600061636B004E6F20534420636172640050B4
:102F700072696E742066726F6D20534400436861FD
:102F80006E67652053442063617264004D323100E6
:102F900041626F7574205072696E74657200436887
:102FA000616E67652066696C616D656E740043686B
:102FB000616E67652066696C616D656E74004D3683
:102FC000303020423000436F6E66696775726174FD
:102FD000696F6E0054656D7065726174757265001D
:102FE0004D6F76656D656E7400526573756D652005
:102FF0007072696E740054756E650053746F702042
:103000007072696E74005061757365207072696EBC
:103010007400496E666F2073637265656E00537449
:103020006F70004261636B0053746F70207072693F
:103030006E74003F005072696E742061626F72742A
:103040006564004D3234004D323520500A4D323423
:10305000005061757365207072696E740050726FF4
:103060006265205A204F666673657400426162791A
:1030700073746570205900426162797374657020C1
:103080005800466C6F7700466C6F770046616E2083
:10309000737065656420310046616E2073706565EC
:1030A0006420310042656400426564004E6F7A7AA4
:1030B0006C65004E6F7A7A6C6500537065656400CC
:1030C0005370656564004D61696E00426162797399
:1030D000746570205900426162797374657020587C
:1030E0000047616D6573005072696E74657220539C
:1030F00074617473004669726D77617265205665FC
:103100007273696F6E004D61696E002569730025E9
:10311000696D20256973002569682025696D202562
:10312000697300256964202569682025696D20255B
:10313000697300256979202569642025696820253F
:10314000696D20256973003E2000457874727564AE
:10315000656420746F74616C3A00256C642E256977
:103160006D003E20004C6F6E67657374206A6F625D
:103170002074696D653A003E2000546F74616C20C4
:103180007072696E742074696D653A00436F6D707A
:103190006C657465643A20005072696E7420436FE8
:1031A000756E743A2000436F6F6C646F776E0046E3
:1031B000616E20737065656420310046616E207316
:1031C0007065656420310042656400426564004EAC
:1031D0006F7A7A6C65004E6F7A7A6C65004D616922
:1031E0006E006F6F6F0000001FC07FF0DDD8FFF82A
:1031F0007FF044402480000031800000248044405F
:10320000107CFEFEFE04000E000E007FC0FFE0FFFB
:10321000E0FFE0FFE006000F001F8036C03FC0095E
:10322000001680294006000F001F8036C03FC016E0
:103230008020401080104008801FC037607FF05F02
:10324000D050500D80104048905FD077707FF01FB5
:10325000C0104020200F007FE0FFF0E670FFF01963
:103260008036C0C0300F007FE0FFF0E670FFF0193D
:103270008036C0198047414D45204F564552005277
:103280006573746F7265206661696C736166650051
:103290004C6F61642073657474696E677300537456
:1032A0006F72652073657474696E67730050726F16
:1032B0006265205A204F66667365740041647661CA
:1032C0006E6365642053657474696E6773004D6145
:1032D000696E0050726F6265205A204F6666736592
:1032E00074004D6F76696E672E2E2E0054415A2061
:1032F000576F726B687273652072656164792E0016
:103300005072696E74696E672E2E2E005072696E4F
:103310007420706175736564004361726420726526
:103320006D6F766564004361726420696E736572C7
:10333000746564004D33310043616E6E6F742065B7
:103340006E746572207375626469723A20002E0A89
:10335000006F70656E206661696C65642C2046693B
:103360006C653A20006175746F25632E6700657285
:10337000726F722077726974696E6720746F20664D
:10338000696C650A004E6F74205344207072696E38
:1033900074696E670A005344207072696E74696EB6
:1033A00067206279746520002E0A0044656C65749C
:1033B000696F6E206661696C65642C2046696C6576
:1033C0003A200046696C652064656C657465643AF2
:1033D0000057726974696E6720746F2066696C6546
:1033E0003A20002E0A006F70656E206661696C6578
:1033F000642C2046696C653A20002E0A006F7065C7
:103400006E206661696C65642C2046696C653A20A3
:103410000046696C652073656C65637465640A00B9
:103420002053697A653A200046696C65206F7065A3
:103430006E65643A20002066696C653A2000667209
:1034400065736800646F696E67004E6F7720004592
:103450004E4420535542524F5554494E450A00227E
:1034600020706F73002220706172656E743A2200C2
:10347000535542524F5554494E452043414C4C20E0
:103480007461726765743A2200747279696E67209C
:10349000746F2063616C6C207375622D67636F6459
:1034A000652066696C6573207769746820746F6F36
:1034B000206D616E79206C6576656C732E204D41B0
:1034C00058206C6576656C2069733A310A004D327C
:1034D00034004D32332025730053442063617264FD
:1034E000206F6B0A006F70656E526F6F742066619B
:1034F000696C65640A00766F6C756D652E696E691E
:1035000074206661696C65640A00534420696E69C1
:1035100074206661696C0A00286E6F2066696C65AC
:10352000290043616E6E6F74206F70656E20737535
:103530006264697220007C3C3E5E2B3D3F2F5B5DE8
:103540003B2C2A225C00473238205A004F46460066
:103550004F4E006563686F3A004572726F723A00B1
:103560004572726F722077726974696E6720746F2A
:1035700020454550524F4D210A005072657373200B
:10358000627574746F6E20286F72204D3130382947
:1035900020746F2068656174206E6F7A7A6C650A9A
:1035A00000507265737320627574746F6E20286F9B
:1035B00072204D3130382920746F20726573756D1B
:1035C000650A00496E736572742066696C616D6589
:1035D0006E7420616E6420707265737320627574FE
:1035E000746F6E20286F72204D313038290A004DDB
:1035F0003630303A20546F6F20636F6C6400486F30
:1036000074656E6420746F6F20636F6C640A004889
:103610006F74656E6420746F6F20636F6C640A0052
:10362000496E736572742066696C616D656E742095
:10363000616E6420707265737320627574746F6E4E
:1036400020286F72204D313038290A0063616E6383
:10365000656C00726573756D656400726573756D78
:10366000650070617573656400706F7765726F6671
:1036700066002F2F616374696F6E3A0020573A001D
:1036800020573A00486F74656E6420436F6F6C6911
:103690006E672E2E2E00486F74656E64204865613B
:1036A00074696E672E2E2E00202F002042403A00B3
:1036B00020403A00546865726D616C2052756E61ED
:1036C00077617900486F74656E6420544845524DA7
:1036D000414C2052554E41574159004245442054D7
:1036E0004845524D414C2052554E415741590020BA
:1036F0002D20496E76616C696420657874727564FA
:103700006572206E756D62657220210A00486561E0
:1037100074696E67206661696C6564004265642047
:1037200068656174696E67206661696C65640054E0
:103730006865726D616C2052756E617761790042C7
:10374000454420544845524D414C2052554E415716
:1037500041590048656174696E67206661696C65EE
:103760006400486F74656E642048656174696E67B3
:10377000206661696C656400546865726D616C20D7
:1037800052756E6177617900486F74656E6420547C
:103790004845524D414C2052554E41574159004DDC
:1037A000494E54454D50207472696767657265646F
:1037B00000486F74656E64204572723A204D494E20
:1037C00054454D50004572723A204D494E54454D76
:1037D0005020424544004D415854454D502074728C
:1037E0006967676572656400486F74656E6420453B
:1037F00072723A204D415854454D50004572723A0C
:10380000204D415854454D50204245440062656466
:10381000002C2073797374656D2073746F707065FC
:103820006421204865617465725F49443A20002331
:10383000646566696E652044454641554C545F0099
:103840004B6420004B6920004B70200000626564CF
:1038500000504944204175746F74756E6520666927
:103860006E697368656421205075742074686520E2
:103870006C617374204B702C204B6920616E642046
:103880004B6420636F6E7374616E74732066726F25
:103890006D2062656C6F7720696E746F20436F6E68
:1038A00066696775726174696F6E2E680A005049A7
:1038B00044204175746F74756E65206661696C652E
:1038C00064212074696D656F75740A0054686572AF
:1038D0006D616C2052756E6177617900486F746517
:1038E0006E6420544845524D414C2052554E41572C
:1038F00041590042454420544845524D414C2052C4
:10390000554E415741590048656174696E6720669C
:1039100061696C656400486F74656E642048656118
:1039200074696E67206661696C6564004265642035
:1039300068656174696E67206661696C65640050D2
:103940004944204175746F74756E65206661696CB9
:103950006564212054656D706572617475726520AF
:10396000746F6F20686967680A00204B643A200012
:10397000204B693A2000204B703A20000A20436C0B
:10398000617373696320504944200A002054753ADA
:103990002000204B753A2000206D61783A200020ED
:1039A0006D696E3A200020643A20002062696173DC
:1039B0003A2000504944204175746F74756E65203B
:1039C00073746172740A00504944204175746F74B5
:1039D000756E65206661696C6564212054656D7043
:1039E0006572617475726520746F6F2068696768AD
:1039F0000A001000AD0330016A0150022B01700370
:103A00000A019004F500B005E500D006D800F007E3
:103A1000CE001009C500300ABE00500BB700700C74
:103A2000B100900DAB00B00EA600D00FA200F010B8
:103A30009D001012990030139500501492007015DB
:103A40008E0090168B00B0178700D0188400F019F4
:103A50008100101B7E00301C7B00501D7900701E01
:103A60007600901F7300B0207000D0216E00F0220D
:103A70006B00102469003025660050266300702713
:103A8000610090285E00B0295C00D02A5900F02B1C
:103A90005600102D5400302E5100502F4E00703023
:103AA0004B0090314800B0324500D0334200F03432
:103AB0003E0010363B003037370050383300703945
:103AC0002E00903A2900B03B2300D03C1B00F03D73
:103AD0001100103F0100F03F00001000C90210016A
:103AE0002C014001220170011801B0010E01F0010A
:103AF00004015002FA00B002F0003003E600D003E7
:103B0000DC009004D2007005C800A006BE000008CA
:103B1000B400B009AA00D00BA000600E960060119E
:103B20008C000015820020197800C01D6E00A022B4
:103B30006400B0275A00902C500000314600E03459
:103B40003C0010383200903A2800603C1E00A03D36
:103B50001400803E0A00203F00006F70656E005424
:103B60005249474745524544003A20007A5F6D610B
:103B700078007A5F6D696E00795F6D696E00785FBD
:103B80006D696E005265706F7274696E6720656E44
:103B90006473746F70207374617475730A00456E7A
:103BA0006473746F70732025632025632025632060
:103BB000256300205A3A0020593A0020583A0065FF
:103BC0006E6473746F7073206869743A20000A53CE
:103BD000746174733A2046696C616D656E7420750A
:103BE0007365643A20002C204C6F6E6765737420F7
:103BF0006A6F623A2000546F74616C2074696D655D
:103C00003A200053746174733A20002C2046616995
:103C10006C65643A20002C2046696E69736865649F
:103C20003A20005072696E74733A200053746174C4
:103C3000733A2000496E76616C696420657874720D
:103C4000756465720A0045313A200045303A20001B
:103C50005A3A2000593A20004D53312C4D53322C02
:103C60004D53332050696E730A583A20004D6963F2
:103C7000726F737465707320756E617661696C61C3
:103C8000626C650A00205A3A0020593A0020436FBE
:103C9000756E7420583A00C23100001C260000F4F2
:103CA000190000D80F0000EB080000C004000075E8
:103CB0000200004001000024F4D43050C38E20C222
:103CC000A24017828B7011127A910D816CD90AA8CB
:103CD00061E108C7586607615143061E4B5D05C187
:103CE00045A7041A411104093D9803713931034075
:103CF00036DB0265339102D4305402802E1D0263FC
:103D00002CEE01752AC501B028A001102781018F72
:103D10002564012B244B01E0223401AC211F018DCD
:103D2000200D01801FFC00841EED00971DDF00B8F0
:103D30001CD200E61BC600201BBC00641AB200B2F5
:103D400019A8000A19A0006A189900D1179100401B
:103D5000178B00B516840031167E00B31579003A32
:103D6000157300C7146F0058146A00EE13660088BC
:103D700013630025135E00C7125B006C1257001519
:103D8000125400C111510070114F0021114B00D687
:103D90001049008D1047004610440002104200C038
:103DA0000F4000800F3E00420F3C00060F3B00CB4F
:103DB0000E3800930E37005C0E3500270E3400F3EA
:103DC0000D3200C10D3100900D3000600D2E00321B
:103DD0000D2D00050D2C00D90C2B00AE0C290085F3
:103DE0000C29005C0C2700350C27000E0C2600E87F
:103DF0000B2400C40B2400A00B23007D0B23005ACE
:103E00000B2100390B2100180B2000F80A1F00D9E4
:103E10000A1E00BB0A1E009D0A1D00800A1D0063C9
:103E20000A1C00470A1B002C0A1B00110A1A00F783
:103E3000091A00DD091900C4091900AB091900921B
:103E40000917007B091800630917004C0916003692
:103E5000091600200916000A091500F5081500E0EA
:103E6000081400CC081400B8081400A4081400902A
:103E70000813007D0812006B081300580812004652
:103E80000812003408110023081100120811000163
:103E9000081100F0071000E0071000D0071000C064
:103EA000071000B0070F00A107100091070E008354
:103EB000070F0074070F0065070E0057070E004933
:103EC000070E003B070D002E070E0020070D001304
:103ED000070D0006070D00F9060C00ED060D00E0C9
:103EE000060C00D4060C00C8060C00BC060C00B082
:103EF000060C00A4060B0099060C008D060B008230
:103F0000060B0077060B006C060B0061060A0057D3
:103F1000060B004C060A0042060A0038060A002E6C
:103F2000060A0024060A001A060A001006090007FD
:103F3000060A00FD050900F4050900EB050900E289
:103F4000050900D9050900D0050900C7050900BE0B
:103F5000050900B5050800AD050800A50509009C88
:103F6000050800940508008C050800840508007CFD
:103F7000050800740508006C050700650508005D6C
:103F8000050700560508004E0507004705070040D5
:103F900005080038050700310507002A050700233A
:103FA0000507001C050600160507000F0507000899
:103FB00005060002050700FB040600F5040700EEF5
:103FC000040600E8040600E2040700DB040600D54E
:103FD000040600CF040600C9040600C3040600BDA1
:103FE000040600B7040600B1040500AC040600A6F0
:103FF000040600A00405009B04060095040500903B
:104000000406008A04050085040500800406007A81
:1040100004050075040500700405006B04050066C6
:10402000040500610405005C040500570405005206
:104030000405004D04050048040500430405003E46
:104040000404003A04050035040500300404002C83
:1040500004050027040400230405001E0404001ABC
:1040600004040016040500110404000D04040009F2
:104070000405000404040000040400FC030400F828
:10408000030400F4030400F0030400EC030400E85C
:10409000030400E4030400E0030400DC030400D88C
:1040A000030400D4030400D0030400CC030400C8BC
:1040B000030300C503030024F404D9201BC40C5CD3
:1040C0000E9804C4095F0265077101F405F900FB4D
:1040D00004B30048048700C1036900580355000376
:1040E000034500BE023A008402310053022A00292F
:1040F00002250004022000E4011C00C8011900AFE1
:10410000011700980114008401130071011000616F
:1041100001100051010E0043010D0036010B002B70
:10412000010B0020010B00150109000C010900031F
:10413000010800FB000800F3000800EB000700E4A2
:10414000000600DE000600D8000600D2000600CC03
:10415000000500C7000500C2000500BD000400B94D
:10416000000400B5000400B1000400AD000400A983
:10417000000400A5000300A20003009F0004009BB0
:1041800000030098000300950002009300030090D4
:104190000003008D0002008B0003008800020086EF
:1041A00000020084000300810002007F0002007D05
:1041B0000002007B00020079000200770001007617
:1041C0000002007400020072000100710002006F22
:1041D0000002006D0001006C0002006A000100692D
:1041E0000002006700010066000100650001006434
:1041F0000002006200010061000100600001005F38
:104200000002005D0001005C0001005B0001005A3B
:10421000000100590001005800010057000100563C
:10422000000100550001005400010053000000533C
:104230000001005200010051000100500001004F38
:104240000001004E0000004E0001004D0001004C36
:104250000001004B0000004B0001004A0001004932
:10426000000100480000004800010047000100462E
:104270000000004600010045000000450001004428
:104280000001004300000043000100420000004222
:104290000001004100000041000100400001003F1A
:1042A0000000003F0001003E0000003E0001003D14
:1042B0000000003D0001003C0000003C0000003C0C
:1042C0000001003B0000003B0001003A0000003A02
:1042D00000010039000000390001003800000038FA
:1042E00000000038000100370000003700010036F0
:1042F00000000036000000360001003500000035E7
:1043000000000035000100340000003400000034DB
:1043100000010033000000330000003300010032D0
:1043200000000032000000320001003100000031C6
:1043300000000031000100300000003000000030BB
:104340000001002F0000002F0000002F0000002FB0
:104350000001002E0000002E0000002E0001002DA4
:104360000000002D0000002D0000002D0001002C99
:104370000000002C0000002C0000002C0001002B8D
:104380000000002B0000002B0000002B0001002A81
:104390000000002A0000002A0000002A0001002975
:1043A0000000002900000029000000290000002969
:1043B000000100280000002800000028000000285C
:1043C000000000280001002700000027000000274F
:1043D0000000002700000027000100260000002642
:1043E0000000002600000026000000260001002535
:1043F0000000002500000025000000250000002529
:10440000000000250001002400000024000000241A
:10441000000000240000002400010023000000230D
:104420000000002300000023000000230000002300
:1044300000000023000100220000002200000022F2
:1044400000000022000000220000002200010021E4
:1044500000000021000000210000002100000021D8
:1044600000000021000000210001002000000020C9
:1044700000000020000000200000002000000020BC
:1044800000000020000000200001001F0000001FAD
:104490000000001F0000001F0000001F0000001FA0
:1044A0000000001F0001001E0000001E0000001E92
:1044B0000000001E00000020204D36303320003A5E
:1044C0000A0020286D6D2900205300205A00205931
:1044D0000020580020204D343235204600426163D0
:1044E0006B6C61736820636F6D70656E7361746966
:1044F0006F6E3A0A002055004C0046696C616D658C
:104500006E74206C6F61642F756E6C6F6164206CCB
:10451000656E677468733A0A0020204D3930302088
:104520004B004C696E65617220416476616E636513
:104530003A0A0020204D383531205A005A2D507249
:104540006F6265204F6666736574002044002049E1
:104550000020204D333034205000204400204900FA
:1045600020204D3330312050005049442073657471
:1045700074696E67733A0A002046002042002048A2
:104580000020204D3134352053004D61746572692F
:10459000616C2068656174757020706172616D6511
:1045A000746572733A0A0020204D34323020530073
:1045B0004175746F20426564204C6576656C696E48
:1045C000673A0A00204500205A0020590020580070
:1045D00020540020530020204D323035204200204E
:1045E000453C6D61785F655F6A65726B3E0020587F
:1045F0003C6D61785F785F6A65726B3E20593C6DF7
:1046000061785F795F6A65726B3E205A3C6D6178B4
:104610005F7A5F6A65726B3E00416476616E6365C6
:10462000643A20423C6D696E5F7365676D656E74B8
:104630005F74696D655F75733E20533C6D696E5F95
:1046400066656564726174653E20543C6D696E5F99
:1046500074726176656C5F66656564726174653EEF
:104660000020540020520020204D323034205000D1
:10467000416363656C65726174696F6E2028756E45
:104680006974732F7332293A20503C7072696E74CA
:104690005F616363656C3E20523C72657472616356
:1046A000745F616363656C3E20543C74726176652F
:1046B0006C5F616363656C3E0A00204500205A0010
:1046C00020590020204D3230312058004D6178694A
:1046D0006D756D20416363656C65726174696F6EA1
:1046E0002028756E6974732F7332293A0A002045A9
:1046F00000205A0020590020204D3230332058002D
:104700004D6178696D756D2066656564726174656B
:10471000732028756E6974732F73293A0A005374D5
:104720006570732070657220756E69743A0A002096
:10473000204D3134392043203B20556E697473205D
:10474000696E2043656C736975730A0020204732D7
:1047500031202020203B20556E69747320696E2023
:104760006D6D0048617264636F64656420446566C2
:1047700061756C742053657474696E6773204C6F37
:10478000616465640A002823000028230000C80033
:10479000000028230000000096430000964300001C
:1047A000F0410000C8410000C8420000C8420000BB
:1047B000FA430000D243454550524F4D20496E699F
:1047C0007469616C697A65640A00290A002062795B
:1047D0007465733B2063726320002073746F72658D
:1047E000642073657474696E67732072657472698E
:1047F00065766564202800202863616C63756C61B0
:1048000074656429210A0020213D2000454550524D
:104810004F4D20435243206D69736D61746368206E
:104820002D202873746F7265642920002053697AE3
:10483000653A2000496E6465783A2000204D617227
:104840006C696E3D563637290A00454550524F4D2A
:104850002076657273696F6E206D69736D61746324
:10486000682028454550524F4D3D00290A002062DE
:10487000797465733B2063726320005365747469B7
:104880006E67732053746F7265642028000A003BC2
:1048900020454550524F4D20496E6465783A2000BE
:1048A0005570646174696E67207A6F6666736574AB
:1048B00020696E20454550524F4D3A2000454550E5
:1048C000524F4D206461746173697A65206572721C
:1048D0006F722E0A004175746F6C6576656C206688
:1048E00061696C65640A004175746F6C6576656C0E
:1048F000206661696C6564005761726E696E673A23
:1049000020486F6D696E672042756D70204469762E
:1049100069736F72203C20310A00020204486F6DF7
:1049200065202573257325732066697273740020D2
:1049300066697273740A00486F6D65200020746F99
:104940006F206C6F6E6720657874727573696F6E17
:104950002070726576656E7465640A0020636F6C02
:104960006420657874727573696F6E2070726576F5
:10497000656E7465640A0020453A00205A3A0020AA
:10498000593A00583A0000004842000048420000EE
:10499000F041FFFF010000A0400000A04000000027
:1049A000400080AC430080A2430080964300004852
:1049B000C2000088C1008095430080934300009AA4
:1049C0004300809543000048C2000088C1000000F9
:1049D000C020746F6F206C6F6E672065787472757D
:1049E00073696F6E2070726576656E7465640A0017
:1049F00020636F6C6420657874727573696F6E20C4
:104A000070726576656E7465640A00627573793AD2
:104A10002070617573656420666F7220696E7075B1
:104A2000740A00627573793A207061757365642049
:104A3000666F7220757365720A00627573793A2029
:104A400070726F63657373696E670A004D31313739
:104A50002050726F6265207375636365737366754A
:104A60006C0A0020496E76616C6964206578747206
:104A7000756465722000205A3A200020593A2000BF
:104A800042656420583A200050726F6265205A20B7
:104A90004F66667365743A20003F5A206F75742024
:104AA0006F662072616E676520282D3220746F203A
:104AB00035290A004D31343520533C696E646578E0
:104AC0003E206F7574206F662072616E67652028C6
:104AD000302D31290A00436C69636B20746F20729A
:104AE0006573756D652E2E2E00220A00556E6B6E55
:104AF0006F776E20636F6D6D616E643A20220045A2
:104B00004550524F4D204F4B0A004E6F206D6F762F
:104B1000652E004543484F00494E464F00455252CE
:104B20004F52530044525952554E00434F4D4D552C
:104B30004E49434154494F4E006F666600134B186F
:104B40004B1D4B244B2B4B44454255473A00544197
:104B50005A20576F726B686F727365204564697471
:104B6000696F6E204F46462E00205A00205900588B
:104B70000020204D61783A2000205A00205900582A
:104B80000020204D696E3A2000536F667420656ED8
:104B90006473746F70733A20005072696E7420747D
:104BA000696D653A20004D3131332053002F2F209D
:104BB000004361703A004348414D4245525F5445BD
:104BC0004D5045524154555245004D4F54494F4E5A
:104BD0005F4D4F44455300544845524D414C5F5042
:104BE000524F54454354494F4E004155544F52453E
:104BF000504F52545F53445F5354415455530050E7
:104C0000524F4D50545F535550504F525400454DE4
:104C1000455247454E43595F504152534552004318
:104C20004153455F4C494748545F425249474854B5
:104C30004E45535300544F47474C455F4C494748F6
:104C4000545300534F4654574152455F504F5745B8
:104C500052004255494C445F50455243454E540022
:104C60004C4556454C494E475F44415441005A5FBC
:104C700050524F4245004155544F4C4556454C000B
:104C80005052494E545F4A4F420050524F4752458E
:104C90005353004155544F5245504F52545F544561
:104CA0004D5000564F4C554D4554524943004545D3
:104CB00050524F4D0042494E4152595F46494C4572
:104CC0005F5452414E534645520053455249414C60
:104CD0005F584F4E5F584F4646004649524D574128
:104CE00052455F4E414D453A4D61726C696E2020D0
:104CF0004649524D574152455F56455253494F4ED2
:104D00003A322E302E302E31333120455854525500
:104D10004445525F545950453A53696E676C654536
:104D2000787472756465724165726F563220534FA4
:104D3000555243455F434F44455F55524C3A687462
:104D40007470733A2F2F636F64652E616C657068A1
:104D50006F626A656374732E636F6D2F6469666634
:104D60007573696F6E2F4D41524C494E2050524F12
:104D7000544F434F4C5F56455253494F4E3A312E94
:104D800030204D414348494E455F545950453A54AF
:104D9000415A20576F726B686F7273652045646962
:104DA00074696F6E2045585452554445525F434FC5
:104DB000554E543A3120555549443A356565373991
:104DC0003866622D343036322D346433352D383226
:104DD00032342D3565383436666662343561350ACD
:104DE000002020536D6F6F7468696E6720286D6DA9
:104DF000293A202020202020202020202020202090
:104E0000202020530020204261636B6C6173682076
:104E100044697374616E636520286D6D293A2020A2
:104E200020202020202000202846312E30203D2028
:104E300066756C6C2C2046302E30203D206E6F6ED7
:104E400065290A002020436F7272656374696F6E72
:104E500020416D6F756E742F466164652D6F75749A
:104E60003A202020202046006163746976653A0A62
:104E700000696E004261636B6C61736820436F72FE
:104E800072656374696F6E2000205A0020580020FC
:104E9000506F736974696F6E616C204572726F72C6
:104EA0003A0A002058004E6F7A7A6C652054697077
:104EB000204F757465722044696D656E73696F6EFD
:104EC000733A0A002020546F703A2000202042617B
:104ED000636B3A2000202052696768743A200020F2
:104EE000204C6566743A20004261636B6C617368A4
:104EF0003A0A00205A0020580043656E7465723AE1
:104F00000A0020204261636B3A200020205269672A
:104F100068743A200020204C6566743A20002020F6
:104F2000546F703A200053696465733A0A00426511
:104F300064204C6576656C696E6720004661696C1B
:104F4000656420746F20656E61626C6520426564E3
:104F5000204C6576656C696E670A00426564204C7A
:104F60006576656C20436F7272656374696F6E203D
:104F70004D61747269783A000A0A426564204C6592
:104F800076656C20436F7272656374696F6E204D35
:104F900061747269783A00202B000A436F7272655F
:104FA000637465642042656420486569676874209D
:104FB00076732E2042656420546F706F6C6F677932
:104FC0003A0A00202B000A42656420486569676838
:104FD0007420546F706F6772617068793A0A20208C
:104FE000202B2D2D2D204241434B202D2D2B0A20EF
:104FF00020207C20202020202020202020207C0A0F
:10500000204C207C20202020282B29202020207CA0
:1050100020520A2045207C202020202020202020F3
:1050200020207C20490A2046207C20282D29204E43
:1050300020282B29207C20470A2054207C20202057
:1050400020202020202020207C20480A2020207C96
:1050500020202020282D29202020207C20540A20B8
:1050600020207C20202020202020202020207C0A9E
:105070002020204F2D2D2046524F4E54202D2D2BD9
:105080000A2028302C30290A003474682070726F8E
:10509000626520706F696E742C2064697374616E30
:1050A00063652066726F6D20706C616E653A2000DA
:1050B000202844525952554E290047323920417513
:1050C000746F20426564204C6576656C696E67007C
:1050D0003F20284C2C522C462C4229206F757420DE
:1050E0006F6620626F756E64732E0A003F50726F98
:1050F000626520706F696E74732028592920697366
:1051000020696D706C61757369626C652028322D41
:1051100032292E0A003F50726F626520706F696EEF
:1051200074732028582920697320696D706C61752B
:105130007369626C652028322D32292E0A003F28BF
:1051400056296572626F7365206C6576656C20699F
:105150007320696D706C61757369626C65202830AD
:105160002D34292E0A0043757272656E74206669AB
:105170006C653A2000456E642066696C65206C6938
:1051800073740A00426567696E2066696C65206CFD
:105190006973740A00416476616E6365204B3D005B
:1051A0003F4B2076616C7565206F7574206F6620AB
:1051B00072616E67652028302D3130292E0A004D2E
:1051C00031313720486F7420456E64204865617422
:1051D000696E672E2E2E0A4D313034205331373010
:1051E0002054300A473238204F310A473120593293
:1051F00035205A31302046353030300A4D31313784
:10520000205265776970696E67206E6F7A7A6C6577
:105210000A54300A473120582D3136205932352072
:1052200046353030300A4D31303920523137302058
:1052300054300A4731205A310A473120582D31362F
:10524000205932352046343030300A473120582D2D
:105250003136205939352046343030300A47312034
:10526000582D3136205932352046343030300A47F7
:105270003120582D313620593935204634303030E0
:105280000A473120582D31362059323520463430E6
:1052900030300A473120582D3136205939352046D3
:1052A000343030300A473120582D313620593235CC
:1052B0002046343030300A473120582D31362059BD
:1052C00039352046343030300A473120582D3136B8
:1052D000205932352046343030300A473120582D9D
:1052E0003136205939352046343030300A473120A4
:1052F000582D3136205932352046343030300A4767
:105300003120582D3136205939352046343030304F
:105310000A4731205A31350A4D3130362053323563
:1053200035200A47302058302059300A4D31303965
:1053300020523136302054300A4D3130370A004D7A
:105340006163726F20746F6F206C6F6E672E0A003E
:1053500020466C6F773A200020643A0020693A00BA
:1053600020703A00204500205A00205900204D3975
:105370003220580043290A0061626C656420286D60
:10538000696E2074656D70200064697300656E003D
:10539000436F6C6420657874727564657320617204
:1053A000652000205400205200416363656C6572E3
:1053B0006174696F6E3A205000496E76616C696461
:1053C0002065787472756465720A0020643A002062
:1053D000693A0020703A00536C6565702E2E2E00DD
:1053E00047322F47332062616420706172616D65BE
:1053F000746572730A0050726F6265205A204F669E
:10540000667365743A2000446F6E65207361766937
:105410006E672066696C652E0A00534420726561D0
:1054200064206572726F720A00446F6E652070723C
:10543000696E74696E672066696C650A004D323961
:105440000053544F505045442E20005072696E74E2
:1054500065722073746F7070656420647565207464
:105460006F206572726F72732E204669782074689F
:1054700065206572726F7220616E6420757365209D
:105480004D39393920746F20726573746172742ECE
:10549000202854656D70657261747572652069733A
:1054A0002072657365742E205365742069742061C1
:1054B000667465722072657374617274696E6729AF
:1054C0000A004E6F20436865636B73756D207769C2
:1054D0007468206C696E65206E756D6265722C2033
:1054E0004C617374204C696E653A20004E6F204306
:1054F0006865636B73756D2077697468206C696E7D
:1055000065206E756D6265722C204C617374204C41
:10551000696E653A2000636865636B73756D206D15
:1055200069736D617463682C204C617374204C69DD
:105530006E653A20004C696E65204E756D6265722D
:10554000206973206E6F74204C617374204C696EF7
:1055500065204E756D6265722B312C204C61737421
:10556000204C696E653A20004D3131300052657330
:10557000656E643A20002042002050006F6B0022CC
:105580000A00656E7175657565696E672022005049
:105590004944204175746F74756E65206661696C4D
:1055A0006564212042616420657874727564657257
:1055B000206E756D6265720A0042656420636F6FCC
:1055C0006C696E672E2E2E004265642068656174DA
:1055D000696E672E2E2E006F6B004739310A4730F7
:1055E000205A313520463630300A4739300A4730A4
:1055F000205831373020593239302046333030305E
:105600000A4D313137205072696E742061626F72B9
:105610007465642E002020506C616E6E6572427558
:105620006666657242797465733A20002046726539
:1056300065204D656D6F72793A2000436F6D70691A
:105640006C65643A204A756E203131203230313930
:105650000A00207C20417574686F723A2028416CE2
:10566000657068204F626A6563747320496E632EAB
:105670002C204C756C7A426F7420476974205265F7
:10568000706F7369746F7279290A0000204C61731E
:105690007420557064617465643A2000322E302E97
:1056A000302E3133310A004D61726C696E00205327
:1056B0006F6674776172652052657365740A0020A5
:1056C0005761746368646F672052657365740A007C
:1056D0002042726F776E206F757420526573657407
:1056E0000A002045787465726E616C20526573659E
:1056F000740A00506F77657255700A007374617296
:10570000740A004B494C4C45442E20005072696E7F
:105710007465722068616C7465642E206B696C6CB2
:1057200028292063616C6C6564210A004B494C4C4C
:105730002063617573656420627920746F6F206DDA
:1057400075636820696E6163746976652074696D3C
:1057500065202D2063757272656E7420636F6D6DA8
:10576000616E643A20004D3130342053313730209F
:1057700054300A4D313137204C6576656C696E675F
:10578000205820417869730A47302058313530203D
:1057900046393939390A473238205A300A4D3131C1
:1057A00037204C6576656C696E6720646F6E652E78
:1057B0000A4731320A4D31303920523136300A4DE4
:1057C0003131372050726F62696E67206265640004
:1057D00070726F62655F726577697065004175749C
:1057E0006F6C6576656C206661696C6564004D312F
:1057F000313720426564206C6576656C696E672080
:105800006661696C65642E0A4730205A31300A4758
:10581000302045300A4D3330302050323520533857
:1058200038300A4D333030205035302053300A4D57
:105830003330302050323520533838300A4D333031
:1058400030205035302053300A4D33303020503224
:105850003520533838300A47342053310070726F86
:1058600062655F6661696C65640050726F74656340
:105870007465642050696E0A0025301D0C282924A7
:10588000311C0B4527232F1B0A1E4443222B1A4190
:1058900042033809FF360308060202000100B24540
:1058A0009F84AB8E4CAA94C5E400E000E200E600C1
:1058B000CB8E11241FBECFEFD1E2DEBFCDBF00E003
:1058C0000CBF14E0A0E0B2E0E4EFF3EB02E00BBFAA
:1058D00002C007900D92A034B107D9F728E1A0E4E7
:1058E000B4E001C01D92A636B207E1F71CE2C8E59C
:1058F000DCE200E006C021970109802FFE010F9431
:10590000B451CF34D10780E00807A9F70E94F338DB
:105910000D94E8590C9400001F920F920FB60F924D
:1059200011242F933F938F939F93AF93BF938091B5
:10593000410490914204A0914304B09144043091F9
:10594000400423E0230F2D3720F40196A11DB11D43
:1059500005C026E8230F0296A11DB11D2093400427
:105960008093410490934204A0934304B093440471
:105970008091450490914604A0914704B091480459
:105980000196A11DB11D8093450490934604A093F8
:105990004704B0934804BF91AF919F918F913F917D
:1059A0002F910F900FBE0F901F9018952FB7F8945E
:1059B00060914104709142048091430490914404A9
:1059C0002FBF08953FB7F894809145049091460405
:1059D000A0914704B091480426B5A89B05C02F3F6D
:1059E00019F00196A11DB11D3FBFBA2FA92F982F05
:1059F0008827820F911DA11DB11DBC01CD0142E080
:105A0000660F771F881F991F4A95D1F708958F92C7
:105A10009F92AF92BF92CF92DF92EF92FF926B0173
:105A20007C01D0DF4B015C01C114D104E104F1041D
:105A3000F1F09CD3C7DFDC01CB0188199909AA09D1
:105A4000BB09883E9340A105B10570F321E0C21A5D
:105A5000D108E108F10888EE880E83E0981EA11CA9
:105A6000B11CC114D104E104F10421F7DDCFFF9092
:105A7000EF90DF90CF90BF90AF909F908F90089560
:105A80008230910538F0880F991F880F991F05976C
:105A90000197F1F70895789484B5826084BD84B548
:105AA000816084BD85B5826085BD85B5816085BD19
:105AB000EEE6F0E0808181608083E1E8F0E0108232
:105AC000808182608083808181608083E0E8F0E073
:105AD000808181608083E1EBF0E08081846080835D
:105AE000E0EBF0E0808181608083E1E9F0E080819B
:105AF00082608083808181608083E0E9F0E0808142
:105B000081608083E1EAF0E080818260808380812F
:105B100081608083E0EAF0E0808181608083E1E25F
:105B2000F1E0808182608083808181608083E0E217
:105B3000F1E0808181608083EAE7F0E08081846029
:105B40008083808182608083808181608083808186
:105B5000806880831092C10008951F93CF93DF93D4
:105B6000182FEB0161E016D1209711F460E004C01A
:105B7000CF3FD10531F461E0812FDF91CF911F91AB
:105B800045C1E12FF0E0E55FFD4FE4914E2F50E07D
:105B9000FA013197E231F10508F09DC08827EE58EF
:105BA000FF4F8F4F0D94B45184B5806884BDC7BD3D
:105BB00097C084B5806284BDC8BD92C080918000CA
:105BC000806880938000D0938900C093880088C04B
:105BD00080918000806280938000D0938B00C0937E
:105BE0008A007EC080918000886080938000D0937E
:105BF0008D00C0938C0074C08091B0008068809349
:105C0000B000C093B3006CC08091B00080628093FC
:105C1000B000C093B40064C080919000806880930D
:105C20009000D0939900C09398005AC08091900042
:105C3000806280939000D0939B00C0939A0050C0E4
:105C400080919000886080939000D0939D00C093D5
:105C50009C0046C08091A00080688093A000809145
:105C6000A0008F7B8093A000D093A900C093A800D0
:105C700037C08091A00080628093A000D093AB00D9
:105C8000C093AA002DC08091A00088608093A000DE
:105C9000D093AD00C093AC0023C0809120018068F8
:105CA00080932001D0932901C093280119C08091CD
:105CB0002001806280932001D0932B01C0932A01A0
:105CC0000FC080912001886080932001D0932D0126
:105CD000C0932C0105C0C038D1050CF04CCF46CF85
:105CE000DF91CF911F91089590E0FC013197E2314F
:105CF000F10508F04EC08827EC57FF4F8F4F0D94E9
:105D0000B451809180008F7703C0809180008F7D97
:105D100080938000089580918000877FF9CF84B5BB
:105D20008F7702C084B58F7D84BD08958091B000C7
:105D30008F7703C08091B0008F7D8093B00008956D
:105D4000809190008F7707C0809190008F7D03C075
:105D500080919000877F8093900008958091A000AB
:105D60008F7707C08091A0008F7D03C08091A00035
:105D7000877F8093A0000895809120018F7707C0CE
:105D8000809120018F7D03C080912001877F8093C7
:105D900020010895CF93DF9390E0FC01EF5AFD4F6F
:105DA0002491FC01E956FD4F8491882361F190E034
:105DB000880F991FFC01EF5EFC4FC591D491FC0147
:105DC000E950FD4FA591B491611109C09FB7F894B6
:105DD0008881209582238883EC912E230BC062302A
:105DE00061F49FB7F8943881822F8095832388834C
:105DF000EC912E2B2C939FBF06C08FB7F894E881AF
:105E00002E2B28838FBFDF91CF9108951F93CF93BF
:105E1000DF93282F30E0F901E55FFD4F8491F90110
:105E2000EF5AFD4FD491F901E956FD4FC491CC23AF
:105E3000C1F0162F811158DFEC2FF0E0EE0FFF1F9D
:105E4000E950FD4FA591B4918FB7F894111105C099
:105E50009C91ED2FE095E92302C0EC91ED2BEC93A2
:105E60008FBFDF91CF911F910895CF93DF93282F9C
:105E700030E0F901E55FFD4F8491F901EF5AFD4FE4
:105E8000D491F901E956FD4FC491CC2389F08111D9
:105E90002BDFEC2FF0E0EE0FFF1FE352FD4FA5913B
:105EA000B491EC91ED2381E090E021F480E002C018
:105EB00080E090E0DF91CF91089508951F920F92B6
:105EC0000FB60F9211240BB60F922F933F934F935F
:105ED0005F936F937F938F939F93AF93BF93EF9352
:105EE000FF93E0910802F09109021995FF91EF915B
:105EF000BF91AF919F918F917F916F915F914F91E2
:105F00003F912F910F900BBE0F900FBE0F901F90DF
:105F100018951F920F920FB60F9211240BB60F9285
:105F20002F933F934F935F936F937F938F939F93A1
:105F3000AF93BF93EF93FF93E0910A02F0910B02AE
:105F40001995FF91EF91BF91AF919F918F917F91A3
:105F50006F915F914F913F912F910F900BBE0F90DA
:105F60000FBE0F901F9018951F920F920FB60F92B1
:105F700011240BB60F922F933F934F935F936F9320
:105F80007F938F939F93AF93BF93EF93FF93E09192
:105F90000C02F0910D021995FF91EF91BF91AF9115
:105FA0009F918F917F916F915F914F913F912F9131
:105FB0000F900BBE0F900FBE0F901F9018951F9261
:105FC0000F920FB60F9211240BB60F922F933F939F
:105FD0004F935F936F937F938F939F93AF93BF93F1
:105FE000EF93FF93E0910E02F0910F021995FF914C
:105FF000EF91BF91AF919F918F917F916F915F9141
:106000004F913F912F910F900BBE0F900FBE0F90AD
:106010001F9018951F920F920FB60F9211240BB676
:106020000F922F933F934F935F936F937F938F9331
:106030009F93AF93BF93EF93FF93E0910402F0918E
:1060400005021995FF91EF91BF91AF919F918F91AB
:106050007F916F915F914F913F912F910F900BBE68
:106060000F900FBE0F901F9018951F920F920FB6B2
:106070000F9211240BB60F922F933F934F935F9380
:106080006F937F938F939F93AF93BF93EF93FF9300
:10609000E0910602F09107021995FF91EF91BF91EF
:1060A000AF919F918F917F916F915F914F913F91B0
:1060B0002F910F900BBE0F900FBE0F901F90189551
:1060C0001F920F920FB60F9211240BB60F922F93BF
:1060D0003F934F935F936F937F938F939F93AF9370
:1060E000BF93EF93FF93E0911002F0911102199585
:1060F000FF91EF91BF91AF919F918F917F916F91A0
:106100005F914F913F912F910F900BBE0F900FBE5B
:106110000F901F9018951F920F920FB60F92112497
:106120000BB60F922F933F934F935F936F937F9391
:106130008F939F93AF93BF93EF93FF93E0911202DE
:10614000F09113021995FF91EF91BF91AF919F913B
:106150008F917F916F915F914F913F912F910F9010
:106160000BBE0F900FBE0F901F90189508951F93B0
:10617000CF93DF93EC011D821C821F821E82198641
:1061800081E0888782E28A871F861E86FE01B39699
:10619000CE01C1962FEF2193E817F907E1F711E03F
:1061A00018A3CE0113D61F8B188E198E80E48A8F08
:1061B0001B8E87EB94E39AAB89ABDF91CF911F9154
:1061C0000895DB01ED91FC911994EF92FF921F93DA
:1061D000CF93DF931F921F92CDB7DEB77C01DC0116
:1061E000D196ED91FC91D29782E069837A831995DB
:1061F00020E030E04AE069817A81C701E2DF182FB0
:10620000D701D196ED91FC91D29783E01995D701F2
:10621000D196ED91FC91D29780E01995812F0F9046
:106220000F90DF91CF911F91FF90EF9008950F9302
:106230001F93CF93DF93EC018B01E9A9FAA982E0C8
:106240001995E9A9FAA981E0199520E030E044E127
:10625000B801CE01B6DF9E012D5C3F4F47E1B8018A
:10626000CE01AFDFE9A9FAA980E0DF91CF911F91BC
:106270000F911994EF92FF921F93CF93DF93EC014C
:106280007B01E9A9FAA982E01995E9A9FAA981E0B7
:10629000199520E030E045E1B701CE0192DF182FDB
:1062A000882339F09E012D5C3F4F47E1B701CE01B5
:1062B00088DFE9A9FAA980E01995812FDF91CF91B4
:1062C0001F91FF90EF900895CF93DF931F92CDB76A
:1062D000DEB79E012F5F3F4F46E473DF89810F9049
:1062E000DF91CF910895CF93DF931F92CDB7DEB7A3
:1062F0009E012F5F3F4F47E464DF89810F90DF915C
:10630000CF91089520E030E048E45BCFCF93DF9356
:10631000EC016A817B81D8DF88836A817B81CE0131
:10632000E2DF89836A817B81CE01ECDF8B879E016E
:106330002D5C3F4F6A817B8147E1CE01DF91CF9198
:1063400040CFCF93DF93EC016A817B813EDF8823CE
:1063500019F0CE01DBDF81E0DF91CF9108958F92BC
:106360009F92AF92BF92CF92EF920F93CF93DF9312
:106370001F921F92CDB7DEB74C015B012A83498380
:10638000F6DEF401B382A282498147A32A8120A7C5
:1063900005A3E4A2C3A2C4010F900F90DF91CF9197
:1063A0000F91EF90CF90BF90AF909F908F90C9CFFB
:1063B000FC01628173813BCFCF93DF93EC01EE85CB
:1063C000FF85309709F019956A817B81CE01DF91B5
:1063D000CF9150CF0F93FC0182819381648F458FC1
:1063E000278F068F9F01245E3F4F4BE3BC01CF01F7
:1063F0000F91E7CEFC0160A30895BF92CF92DF9288
:10640000EF92FF920F931F93CF93DF936C01D62FE0
:10641000B42EC22F7801CC2369F0F701049120E05B
:106420004B2D6D2FC601D6DFFFEFEF1AFF0AC150CB
:10643000D85FF1CFDF91CF911F910F91FF90EF9037
:10644000DF90CF90BF9008958F929F92AF92BF92AE
:10645000CF92DF92EF92FF920F931F93CF93DF9330
:106460005C01C62EC42FD22ED02F220F220F220F56
:106470001ED0882379F0DC0F8D2C912CCD1751F094
:1064800087012D2D4C2F6C2DC501B7DFE80CF91CB1
:10649000CF5FF4CFDF91CF911F910F91FF90EF90DD
:1064A000DF90CF90BF90AF909F908F9008950F9303
:1064B000FC010150040F84A996A9941718F008173D
:1064C00028F402C0081750F0041740F42150260F9A
:1064D00083A995A9961720F4281720F480E007C017
:1064E000281720F481E0261710F0F8CF81E00F91F3
:1064F000089581E008952EE93FE0009729F0F90121
:106500003197F1F70197F9CF0895FC01128280814C
:106510008150838314820895FC0180819281980FB9
:1065200092832181921760F494819F5F9483938179
:10653000890F821710F08FEF820F838381E0089517
:1065400080E00895FC0191E08381861708F490E0D3
:1065500031E0461708F030E0832F892B21E052818B
:10656000451708F420E02823832F8923822B0895E0
:10657000DC01FB01108212968C9112978183159693
:106580008C9115978150828313968C918383089503
:10659000FB0141812381213029F0233031F468EF60
:1065A000640F04C0642F485F01C0642FCBCFDC01AF
:1065B00015962C9115971696ED91FC911797CF0192
:1065C000820F911D820F911D1192E817F907E1F7D3
:1065D0000895FC01A681B7818281481B85814830DE
:1065E00018F0A80FB11D4770382F3695369536959F
:1065F000562F577080E890E002C0959587955A9580
:10660000E2F7439F402D1124669566956695E62F27
:10661000F0E0E40FF11DEA0FFB1F3081222311F09F
:10662000832B02C08095832380830895FB014181E1
:10663000DC0112962C911297421760F013962C9160
:106640001397241738F0608115962C91621710F477
:106650002481BFCF0895CF92DF92FF920F931F93B3
:10666000CF93DF936C01EB01FA809B81913051F065
:1066700030F0923049F0933051F41FEF09C010E030
:1066800001E007C011E004C010E00FEF02C010E00D
:1066900000E0F7FE03C0BE01C601C8DF9881900F7D
:1066A00098839981910F9983FF0C99F7DF91CF918E
:1066B0001F910F91FF90DF90CF9008950F931F933C
:1066C000CF93DF938901FB01C281D3814233D9F09B
:1066D00058F44531E1F0473109F1443141F5CE013B
:1066E00066DFCE0112DF23C04634E1F04734E1F02B
:1066F0004B33E9F4B901CE014BDF8823C1F0B80177
:10670000CE01A9DF14C0B901CE0190DF10C0CE01C7
:1067100003DF882369F0CE014ADF09C0B901CE0149
:1067200027DF05C08D8101C08981F801808381E068
:10673000DF91CF911F910F910895CF92DF92EF9249
:10674000FF920F931F93CF93DF937C01D62FD42E0C
:10675000C22F122FC62EC20E6C2D611B183038F0BE
:106760000FEF20E04D2DC70135DE1850F5CF6C2F0F
:10677000687F6D0F2C2F277071F097E029272F5F0E
:1067800027700FEF10E001C0000F2A95EAF720E014
:106790004D2DC7011FDEDF91CF911F910F91FF900B
:1067A000EF90DF90CF900895CF92DF92EF92FF921B
:1067B0000F931F93CF93DF937C01D62ED42FC22F3C
:1067C000122FC42EC20E4C2D411B183038F00FEF83
:1067D00021E06D2DC701FEDD1850F5CF4C2F487F0D
:1067E0004D0F2C2F277071F097E029272F5F27700E
:1067F0000FEF10E001C0000F2A95EAF721E06D2DA0
:10680000C701E8DDDF91CF911F910F91FF90EF90CD
:10681000DF90CF900895EF92FF920F931F93CF9345
:10682000DF93EC01162FF42EE22E01E040DE8823E8
:1068300059F02E2D4F2D612FCE01DF91CF911F9159
:106840000F91FF90EF9079CFDF91CF911F910F9132
:10685000FF90EF900895EF92FF920F931F93CF93C5
:10686000DF93EC01162FF42EE22E022F21E01FDE23
:10687000882359F02E2D4F2D612FCE01DF91CF911E
:106880001F910F91FF90EF908FCFDF91CF911F91CC
:106890000F91FF90EF900895DF92EF92FF920F9388
:1068A0001F93CF93DF937C01162FC42FD22ED02FAE
:1068B000FEDD8823F9F02D2D4C2F612FC7013DDF20
:1068C0002D2F4C2F612FC7016FDF6FEF6D0D610F03
:1068D0002D2F4C2FC70168DF4FEF4D0F4C0F2D2D83
:1068E000612FC701DF91CF911F910F91FF90EF9022
:1068F000DF9023CFDF91CF911F910F91FF90EF9009
:10690000DF900895EF92FF920F931F93CF93DF9341
:106910007C01D62F122FC42F040F212F4C2F6D2F47
:10692000C7010BDFCF5F0C13F8CFDF91CF911F9121
:106930000F91FF90EF900895DF92EF92FF920F93E7
:106940001F93CF93DF93EC01162FF42EE22EAFDDD1
:10695000882329F02E2D4F2D612FCE01D3DFDF911B
:10696000CF911F910F91FF90EF90DF9008950895C0
:10697000FC01E60FF11D849190E0982F8827319655
:10698000E4918E0F911D0895FC0184910895FCDF20
:10699000882321F0823011F083E0089586E0089585
:1069A00080E00895FC018081089566E0E1CF68E011
:1069B000DFCF0A96FC01849108950B96FC01849127
:1069C0000895DC011496ED91FC9115973196849110
:1069D0000895BF92CF92DF92EF92FF920F931F9391
:1069E000CF93DF938C01E62EDC011496CD91DC91E0
:1069F0001597CE01C9DFF82EF80184819581C7DF94
:106A0000C82EF1E0FF1203C02FE0B22E02C0BB245B
:106A1000BA94D80114968D919C911597CADFF82EDF
:106A2000F80184819581C9DFD82ED80114968D9103
:106A30009C911597BCDFB0E6BE1538F4009729F09D
:106A4000C80FD91F91E6F92E0FC0F80184819581F6
:106A5000ACDFF0E4FE1538F4009729F0C80FD91F19
:106A600081E4F82E01C06196DE1490F4D8015096AE
:106A70001C92509753961C92539754961C9254977D
:106A800051961C92519752961C9280E090E066C0FD
:106A9000DF1460F38C2D90E0FE0124912F3F11F460
:106AA000219657C0FE104CC0D80114968D919C9130
:106AB00015976ADF9E012F5F3F4FFE01882311F07B
:106AC0008230E1F48491D80153968C935397F90165
:106AD000249154962C935497FE013396E49150964A
:106AE000EC935097FE013496E4915196EC935197B4
:106AF000FE013596E4915296EC9320C08491982F34
:106B00009F709250D80152969C93529782958F70A5
:106B100051968C935197F9012491822F8F7054963E
:106B20008C93549722952F7053962C935397FE0174
:106B30003296E491E295EF705096EC93CE010EC040
:106B4000FE013296E491EB219C012E0F311DC20F04
:106B5000D31FFD1409F48ACFF3949ECFDF91CF9118
:106B60001F910F91FF90EF90DF90CF90BF9008950D
:106B70004F925F926F927F929F92AF92BF92CF920D
:106B8000DF92EF92FF920F931F93CF93DF931F92A9
:106B9000CDB7DEB72C01C62E942E622F1ADF7C01F2
:106BA000892B09F43AC0F20184819581F0DEB82E78
:106BB000F201138904898189C80E8289981AD92C17
:106BC000D01A212F4D2D6C2DC20171DC882311F1BB
:106BD000EB0CF11C195F169516951695612E712C0C
:106BE000D914C1F03C2D57018A2D8E19811770F4EC
:106BF000F501049120E04D2D632FC2013983EADBBA
:106C0000FFEFAF1ABF0A3981385FEECFE60CF71CF1
:106C1000D394E6CFF201808901C080E00F90DF912C
:106C2000CF911F910F91FF90EF90DF90CF90BF9089
:106C3000AF909F907F906F905F904F9008950F93CB
:106C40001F93CF93DF9300D0CDB7DEB78C01DC016B
:106C50005596ED91FC9156972B834A83698319953C
:106C60004A81480F2B816981C8010F900F900F90C6
:106C7000DF91CF911F910F917BCFAF92BF92DF92A7
:106C8000EF92FF920F931F93CF93DF931F921F9268
:106C9000CDB7DEB77C01D62E042FDC015596ED91E1
:106CA000FC91569729833A831995080F2981A22EC2
:106CB0003A81B32E10E0F50121915F01222339F0D2
:106CC000402F6D2DC70154DFD80E180FF4CF812F40
:106CD0000F900F90DF91CF911F910F91FF90EF9048
:106CE000DF90BF90AF900895DF92EF92FF920F93E5
:106CF0001F93CF93DF937C01D62FD42E8901DC0123
:106D00005596ED91FC9156971995D80EC0E0F80173
:106D10002491222349F04D2D6D2FC70129DFD80F73
:106D2000C80F0F5F1F4FF3CF8C2FDF91CF911F91B3
:106D30000F91FF90EF90DF900895DC0114962D9154
:106D40003C9115972115310509F43FC057968C9158
:106D50005797F901811108C03596E4915896EC9344
:106D60005897F9013C9611C0813041F43F96E49167
:106D70005896EC935897F901709607C03D96E491A8
:106D80005896EC935897F9013E96E4915996EC93F6
:106D9000599758968C915897082E000C990B599634
:106DA0002C915997821B910927FD93955A962C9106
:106DB0005A97203441F0829FC001112426E0969515
:106DC00087952A95E1F75B968C93089520ED34E33F
:106DD000FC01368B258B0895CF92DF92EF92FF92C4
:106DE0000F931F93CF93DF938C017B016A01CB013B
:106DF000FA011995D82F882311F1682FC801E9DD10
:106E0000F801C189C195FFEFEF1AFF0AC701F6012A
:106E10001995F801882351F08089C80FC701F60140
:106E20001995D82F682FC801D4DDEDCFD03221F0CD
:106E300091898389890F01C080898C0F01C080E00E
:106E4000DF91CF911F910F91FF90EF90DF90CF9046
:106E5000089542ED54E3C0CFCF93DF93FC0124812A
:106E600035812617370741F0EC017583648365DFB0
:106E700080ED94E39E8B8D8BDF91CF910895CF931E
:106E8000DF9300D01F92CDB7DEB761157105810584
:106E9000910579F09B01AC0169833A834B835C8354
:106EA0000F94245229813A814B815C810F9498512F
:106EB00003C060E070E0CB010F900F900F900F9037
:106EC000DF91CF910895CF92DF92EF92FF920F93CF
:106ED0001F9362177307840795077CF489019A0151
:106EE0006B017C01C901B8016C197D098E099F09EC
:106EF000C6DF6C0D7D1D8E1D9F1D1F910F91FF9094
:106F0000EF90DF90CF9008954F925F926F927F92B3
:106F1000AF92BF92CF92DF92EF92FF920F931F93A7
:106F2000CF93DF93CDB7DEB729013A019B01AC01C6
:106F300024193509460957098A899B89AC89BD8975
:106F4000BC01CD016A197B098C099D090F9434514C
:106F5000A801970124193509460957090F9498513A
:106F6000CA01B9016A0D7B1D8C1D9D1DDF91CF915A
:106F70001F910F91FF90EF90DF90CF90BF90AF9057
:106F80007F906F905F904F90089580E090E008951B
:106F90000895CF92DF92EF92FF920F931F93CF93BA
:106FA000DF936C017A018B01C0E0D0E0CE15DF05E4
:106FB00089F0D8016D918D01D601ED91FC91019080
:106FC000F081E02DC6011995892B11F47E0102C0D4
:106FD0002196ECCFC701DF91CF911F910F91FF90C8
:106FE000EF90DF90CF9008956115710579F0FB0166
:106FF00001900020E9F73197AF01461B570BDC01E8
:10700000ED91FC910280F381E02D199480E090E0F5
:107010000895DC01ED91FC910190F081E02D19942F
:107020004F925F926F927F92EF92FF920F931F9316
:10703000CF93DF93CDB7DEB7A1970FB6F894DEBF3D
:107040000FBECDBF7C01FA01CB0119A2223008F49A
:107050002AE08E010F5D1F4F422E512C612C712CA6
:10706000BF01A30192010F947651F901CA010150A9
:1070700011096A3014F4605D01C0695CD8016C9339
:10708000232B242B252B61F7B801C701ADDFA19677
:107090000FB6F894DEBF0FBECDBFDF91CF911F9129
:1070A0000F91FF90EF907F906F905F904F900895B9
:1070B000CF92DF92EF92FF920F931F93CF93DF93C4
:1070C000EC016A017B012115310579F4E881F98130
:1070D0000190F081E02D642FDF91CF911F910F91EE
:1070E000FF90EF90DF90CF9019942A303105D9F4BA
:1070F00077FF18C06DE28DDF8C0144275527BA0158
:107100004C195D096E097F092AE0CE0189DF800FE5
:10711000911FDF91CF911F910F91FF90EF90DF9022
:10712000CF9008952AE0B701A601CE01DF91CF915B
:107130001F910F91FF90EF90DF90CF9071CF9A0148
:10714000AB01770F660B770BB3CFCF93CFB7F89424
:1071500080914904811127C0ECECF2E08491E6E8CB
:10716000F2E09491E82FF0E0EE0FFF1FEF5EFC4F8E
:10717000A591B491EC91E92321F461E085E30E94AB
:10718000062F61E085E30E94CA2E8CB580618CBD1C
:107190008CB580648CBD61E084E30E94CA2E61E0FE
:1071A00083E30E94CA2E809149048F5F8093490433
:1071B000CFBFCF910895CF92EF920F93FC0113AE02
:1071C00014AE15AE0496CBD80F91EF90CF900895E2
:1071D0008EBD00000DB407FEFDCF8EB5089580E092
:1071E00090E0089508950E944B2DFCDF0F949F4C72
:1071F000C0E0D0E00F94224D2097E1F30E94000000
:10720000F9CFCF93DF931F92CDB7DEB7909159049A
:10721000292F2370233041F091609260909359049C
:1072200089830E94864789810F90DF91CF910C94CA
:10723000944780915904982F9370913031F0816078
:107240008D7F809359040C948D470895CF93DF93DD
:10725000EC018991882319F00E949447FACFDF91BD
:10726000CF9108950F931F93CF938C01C62FF801F0
:1072700081918F01882331F0CC2321F00E94944723
:10728000C150F5CFCF911F910F910895CF93DF9308
:10729000FC018491EF012196882321F00E949447FC
:1072A000FE01F7CFDF91CF9108950F931F93CF93F6
:1072B000DF93CDB7DEB727970FB6F894DEBF0FBECA
:1072C000CDBF6330B1F038F46130B1F0623049F5D0
:1072D00025EB35E113C0653031F040F0663009F53B
:1072E00025EC35E10BC021EC35E108C02DEB35E193
:1072F00005C029EB35E102C021EB35E19F938F9367
:107300003F932F938E010F5F1F4F1F930F930F9487
:10731000CE56C8019BDF0F900F900F900F900F90EB
:107320000F9027960FB6F894DEBF0FBECDBFDF914A
:10733000CF911F910F9108951F93CF93DF931F92C9
:10734000CDB7DEB7182F811102C080E201C084E200
:10735000611102C090E001C092E0892B698351DF86
:107360009091590410FB92F9892F698160FB83F990
:10737000809359040F90DF91CF911F9108956091F0
:10738000590462FB992790F9891721F063FB66275E
:1073900060F9D2CF0895CF93C82F81E0F0DFC111FB
:1073A00002C082E001C083E02CDF90915904C0FB51
:1073B00094F990935904CF9108959091590492951E
:1073C00091708913E8CF0895CF93C82F80E0D7DF5D
:1073D0008C2F8F738068CF9114CFCF93C82F80E00C
:1073E000CEDF8C2F8F738064CF910BCF1F93CF9301
:1073F000DF931F92CDB7DEB7182F81E06983BFDF1F
:107400006981862F8068FDDE812F8F7080680F90E4
:10741000DF91CF911F91F5CE80E0B1DF81E0F1DE09
:107420006FE070E080E090E00C94072DCF93DF9345
:10743000C0E06C2F80E0DADFFCDED1E1D15039F022
:1074400080E00E94944780E00E949447F7CFCF5F8E
:10745000C03279F7DF91CF910895CF92DF92EF920A
:10746000FF921F93CF93DF931F921F92CDB7DEB78A
:1074700069837A83B2DFDDDE6981C62E7A81D72EF9
:1074800011E1115069F0F601E590F4908F2D0E9402
:1074900094478E2D0E94944782E0C80ED11CF1CFF4
:1074A0000F900F90DF91CF911F91FF90EF90DF90A1
:1074B000CF900895CF92DF92EF92FF920F931F9398
:1074C000CF93DF931F92CDB7DEB7982F623010F0C5
:1074D0006250985FC62EC29480EFC8228A01D12CD8
:1074E0006D2D6C0D892F998381DFA3DEF801E59066
:1074F000F4908F2D0E9494478E2D0E949447D39430
:107500000E5F1F4F998180E1D812EACF0F90DF9173
:10751000CF911F910F91FF90EF90DF90CF90089542
:10752000CF92DF92EF92FF920F931F93CF93DF934F
:10753000C42E623010F06250805F982F9170D92E67
:10754000C82FC695D62FD295D07F89EAE82E86E13E
:10755000F82E01E0F7011491602F6D0F8C2F46DF9C
:1075600068DECC2059F0D11002C0812F01C080E02C
:107570000E949447DD2029F0812F04C080E00E9402
:10758000944780E00E9494470F5FFFEFEF1AFF0AD5
:10759000053001F7DF91CF911F910F91FF90EF9090
:1075A000DF90CF9008958F929F92AF92BF92DF921B
:1075B000EF92FF920F931F93CF93DF93D82E69E141
:1075C0000F94435120E1929FC001112469E170E0C2
:1075D0000F94635180E090E85C0102C0B594A794D9
:1075E0006A95E2F711E0ED2CF12C612F8CE0FEDEC4
:1075F00020DE20E030E000E0490189E1880E911CA6
:10760000E814F90434F42E153F0534F0C0E0D0E05E
:1076100004C0CFEFDFEF01C0E501113051F01D30A4
:1076200041F0033011F4C16006C0011104C0D068FC
:1076300002C0CFEFDFEF8D2F0E9494478C2F0E9466
:1076400094470F5F940124363105B1F61F5F1E3059
:1076500061F68CE0B9DEEDDD80E20E94944729E01E
:107660002D1530F464E0C70120DE8EEA95E105C0F7
:1076700063E0C7011ADE8AEA95E1DF91CF911F919D
:107680000F91FF90EF90DF90BF90AF909F908F9001
:10769000FDCDCF93C82F85E097DECBDDC11102C0B1
:1076A000C6E001C0C4E080E00E9494478C2FCF91D7
:1076B0000C94944780E081DE69E476E180E090E01C
:1076C000CCDE69E276E180E190E0C7DE69E076E158
:1076D00080E290E0C2DE69EE75E180E390E0BDDE1D
:1076E00049E856E160E080E0E5DE49E656E161E028
:1076F00080E0E0DE49EC55E161E085E0DBDE80E042
:10770000C8CF1F93CF93DF931F92CDB7DEB7182F4B
:1077100080E1698359DE8DDD6981662351F01111A5
:1077200002C012E001C010E080E00E949447812F67
:1077300004C080E20E94944780E20F90DF91CF91D5
:107740001F910C949447CF92DF92EF92FF920F9388
:10775000CF93DF93C82F6B017A01D22F813049F08C
:1077600028F0823049F0833039F008C081E02CDE07
:1077700005C081E129DE02C089E026DE5ADD63E032
:10778000C60193DDDD2349F08AE10E94944763E05E
:10779000C7018BDD011106C015C0002399F085EAF1
:1077A00095E174DD41E04D276C2F85E0B9DE4D2F6A
:1077B0006C2F89E0DF91CF910F91FF90EF90DF90D8
:1077C000CF90AECEDF91CF910F91FF90EF90DF90F1
:1077D000CF9008950F93CF936115710589F0C1E0A3
:1077E000681779073CF49C01261B370B23303105C1
:1077F00044F406C09B01281B390B233031050CF4DF
:10780000C0E02091140221702C1711F001E001C09A
:10781000042F2C2FAB01BC0180E095DF8091140276
:10782000C0FB80F980931402CF910F9108950F93BC
:10783000CF936115710589F0C1E0681779073CF4B1
:107840009C01261B370B2330310544F406C09B01F5
:10785000281B390B233031050CF4C0E020911402B1
:1078600022FB222720F92C1711F001E001C0042F80
:107870002C2FAB01BC0181E066DF80911402C0FBBC
:1078800082F980931402CF910F910895CF93C82F5E
:1078900086E09ADDCEDC63E08C2F90E006DD85E2A9
:1078A000CF910C949447CF92DF92EF92FF920F9377
:1078B0001F93CF93DF93CDB7DEB727970FB6F8941A
:1078C000DEBF0FBECDBF8C0188E07EDDF801608198
:1078D0007181828193812CE3C22ED12CE12CF12C79
:1078E000A70196010F947651CA01B901A70196012B
:1078F0000F9476518E010F5F1F4F2436310598F497
:107900007F936F933F932F938BE995E19F938F9391
:107910001F930F930F94CE560FB6F894DEBF0FBE91
:10792000CDBF85E012C07F936F933F932F9383E980
:1079300095E19F938F931F930F930F94CE560FB69D
:10794000F894DEBF0FBECDBF86E0F801E80FF11D51
:1079500080E280836EDC66E0C80184DC27960FB687
:10796000F894DEBF0FBECDBFDF91CF911F910F9175
:10797000FF90EF90DF90CF900895CF93DF93EC01CD
:1079800086E122DD56DC63E0CE018FDC85E2DF910B
:10799000CF910C949447CF9388E116DD4ADC8BEFAE
:1079A00096E00E94F77DC82F65E18BEF96E05ADCE8
:1079B000C53128F480E20E949447CF5FF9CFCF9180
:1079C00008950E94AA7F4091280D90913A0220913B
:1079D000320D3091330D6091670270916802262755
:1079E000372760910C0D70910D0D26273727949F36
:1079F000A0011124440F452F441F550B51952427F6
:107A00003527A9014827CA0120914F04309150041D
:107A10002817390731F09093500480934F0481E088
:107A2000089580E008954F925F926F927F928F92B7
:107A30009F92AF92BF92CF92DF92EF92FF921F93ED
:107A4000CF93DF9300D01F92CDB7DEB7F82E811110
:107A500004C0B7DF882309F467C00E94AA7F182FEB
:107A60000F94F84869837A838B839C83A090670284
:107A7000B09068026091080D7091090D80910A0D17
:107A800090910B0D0F949B4E2B013C01C0900C0D5F
:107A9000D0900D0D8090320D9090330D60912E0D91
:107AA00070912F0D8091300D9091310D0F949B4E60
:107AB000DC01CB014F2DB4018DDE4F2DB601C2018B
:107AC000B6DE2091280DE22EF12C11110DC09091FF
:107AD0003A0297FD09C0929F900111247901EE0CA2
:107AE000EF2CEE1CFF08F19424E62E9DC0012F9D83
:107AF000900D112481589F4F6FEF70E00F946351E8
:107B0000862FC4DECE010196CEDEC50136DFEF281A
:107B100011F0812FBEDD61E01C141D041CF060E03B
:107B200080E001C0812FEDDD0F900F900F900F903E
:107B3000DF91CF911F91FF90EF90DF90CF90BF909A
:107B4000AF909F908F907F906F905F904F9008952F
:107B5000EBEFF6E080E09191992311F08927FBCFBC
:107B60009091510491110BC091E020914E04281383
:107B700001C090E090934D0491E090935104909156
:107B80004D04911180934E0481E0911101C080E079
:107B900008950E94AA7F982F81E020914C04291318
:107BA00002C080E0089590934C040895811103C0B1
:107BB000CFDF882311F0EFDEECCF0895CF93C82FED
:107BC0000E946C84C11104C090914B04981721F05D
:107BD00080934B04CF91E7CCCF910895CF93C82FDA
:107BE0000E948047809159048E7F809359048C2F86
:107BF0001ADF8C2FDBDF8C2FE1DF0E948047809122
:107C000059048E7F80935904CF91089561E081E0FB
:107C100093DB61E081E090DB80E0BDCB0E94804798
:107C2000809159048E7F80935904F0DFF5DBFEDBF1
:107C300041DD81E0D3DF0E948047809159048E7F2F
:107C40008093590408950E948047809159048E7F43
:107C500080935904E1DB61E081E06EDB0E948047A4
:107C6000809159048E7F8093590408950E94804723
:107C7000809159048E7F80935904C8DFCDDB61E089
:107C800081E05ADB0E948047809159048E7F809367
:107C90005904089580E0A2CF90914A04981729F0E2
:107CA00080934A048111BACFCECF0895E7E6F4E07D
:107CB00083AF64AF08954AE050E0BC0187E694E0EA
:107CC0003ECAEF92FF920F931F93CF93DF937A01F7
:107CD0006F3F71058105910509F050F487E694E046
:107CE00098D98BE694E00E94E134282F30E014C04C
:107CF000C091A204D091A3044D2F50E0EC2FF0E0EE
:107D00008B019C01BF018BE694E0ACD1C80FC093FE
:107D1000A204D093A3049C01C901DF91CF911F91CC
:107D20000F91FF90EF900895EF92FF920F931F93A2
:107D3000CF93DF938B01C7E6D4E0FBACECAC4E2DC8
:107D400050E06F2D70E09C018BE694E0E3D1F80EDB
:107D5000FBAEECAEDF91CF911F910F91FF90EF90B2
:107D60000895EF92FF920F931F93CF93DF938B01B0
:107D7000C7E6D4E0FBACECAC4E2D50E06F2D70E0CC
:107D80009C018BE694E012D2F80EFBAEECAEDF91D4
:107D9000CF911F910F91FF90EF9008950F931F9334
:107DA000CF93DF93CDB7DEB728970FB6F894DEBF39
:107DB0000FBECDBF8A0123E0660F771F2A95E1F73A
:107DC000680F791F48E050E0CE0101960F940256EB
:107DD00029813A81F801808191812817390790F033
:107DE0008217930760F09C818281981758F081E098
:107DF00090E03B812381231738F080E005C081E0CB
:107E000090E002C08FEF9FEF28960FB6F894DEBF88
:107E10000FBECDBFDF91CF911F910F910895EF92CB
:107E2000FF920F931F93CF93DF93EC018B017A01A5
:107E30008A859B858617970729F0888199810CD8B8
:107E40001B870A8788859985019689F00E811F8195
:107E5000B701888199810E942937080F111D8885F3
:107E600099858017910718F481E090E011C06E8128
:107E70008A81680F97014C81888199810E943D36E3
:107E80002E813F81280F311D3F832E8380E090E0BB
:107E9000DF91CF911F910F91FF90EF9008954F9236
:107EA0005F926F927F928F929F92AF92BF92CF928A
:107EB000DF92EF92FF920F931F93CF93DF93CDB793
:107EC000DEB72D970FB6F894DEBF0FBECDBF6C01A5
:107ED0002A013B01490158011B861C86CE010196EF
:107EE0007C0188E0F70111928A95E9F7DB01CA016C
:107EF00027E0B695A795979587952A95D1F79A8308
:107F00008983F42FFF77FD878F2F80588B838C8395
:107F10001A8619864F3F51056105710509F018F45D
:107F200060E070E026C060915C0470915D048E0199
:107F3000075F1F4F97014EEC5EE380915A049091CA
:107F40005B040E94487C97FDEBCF69857A8583E0CE
:107F5000660F771F8A95E1F780915A0490915B0430
:107F6000680F791F48E050E0C7010F9402566F81F7
:107F700078856115710519F44B86B60106C0C616E1
:107F8000D70619F08D8580688B87AE01455F5F4FFE
:107F9000C401F50119952D960FB6F894DEBF0FBEFA
:107FA000CDBFDF91CF911F910F91FF90EF90DF90A8
:107FB000CF90BF90AF909F908F907F906F905F9089
:107FC0004F9008956F927F928F929F92AF92BF923F
:107FD000CF92DF92EF92FF920F931F93CF93DF9395
:107FE00000D01F92CDB7DEB76C017B013A01590179
:107FF000480119821A821B821C82AE014F5F5F4FBB
:10800000B301C7010E94A87C7C0149815A816B8120
:108010007C81411551056105710529F084019501A7
:10802000C6013DDFE6CF0F900F900F900F90DF91CC
:10803000CF911F910F91FF90EF90DF90CF90BF9065
:10804000AF909F908F907F906F90089521E0209344
:108050005E04EAE5F4E0918380837383628380E0C9
:1080600090E008957F92AF92BF92CF92DF92EF920D
:10807000FF920F931F93CF93DF93CDB7DEB72C976B
:108080000FB6F894DEBF0FBECDBF6C01762EF72F72
:10809000842FE52FB901A801D6011496AD90BC90AC
:1080A000159790915E0491110AC02DEE36E1482F8C
:1080B000672DC6010E94743680E090E019C0DA8214
:1080C000C9827B82FC838D83EE8318861F82FA86A9
:1080D000E9861C861B860FE01FE39E012F5F3F4F42
:1080E000C501DDDEB501C6010E942C378F81988560
:1080F0002C960FB6F894DEBF0FBECDBFDF91CF91A7
:108100001F910F91FF90EF90DF90CF90BF90AF90B5
:108110007F900895CF92DF92EF92FF920F931F937B
:10812000CF93DF93CDB7DEB72C970FB6F894DEBFB1
:108130000FBECDBF7C01C901F701C480D58020915D
:108140005E04211108C02DEC36E1C7010E9474368F
:1081500080E090E01CC0FA82E9826B837C834D83CF
:108160005E8318861F821A8709871C861B860FE08C
:108170001FE39E012F5F3F4F42E45CE7BC01C60155
:1081800021DFB601C7010E942C378F8198852C967C
:108190000FB6F894DEBF0FBECDBFDF91CF911F9118
:1081A0000F91FF90EF90DF90CF900895CF92DF92E4
:1081B000EF92FF920F931F93CF93DF93CDB7DEB76C
:1081C0002C970FB6F894DEBF0FBECDBF7C01C9015E
:1081D000F701C480D58020915E04211108C02DEAEA
:1081E00036E1C7010E94743680E090E01CC0FA823C
:1081F000E9826B837C834D835E8318861F821A8796
:1082000009871C861B860FE01FE39E012F5F3F4FEF
:1082100045E45CE7BC01C601D5DEB601C7010E949A
:108220002C378F8198852C960FB6F894DEBF0FBE41
:10823000CDBFDF91CF911F910F91FF90EF90DF9015
:10824000CF900895CF93DF93EC01262F4CAD6BAD0B
:1082500004960E941F362BAD082E000C990B820F3E
:10826000911D8BAF81E090E0DF91CF9108950F9346
:108270009CE0899F802D112421E0280F2093660423
:10828000845F8093650490E0029640919F0450E0E3
:108290008417950714F480E033C0822F90E020917A
:1082A000A10430E082179307B4F76623A9F061E0D8
:1082B0008BE694E00E94FA31409166044E5F0BE039
:1082C00020E860E08BE694E00E949C3460E08BE65E
:1082D00094E00E94FA3105C061E08BE694E00E94D0
:1082E000FA316091650480919F046817A0F2909123
:1082F00066048091A104891770F280E0D7DC81E0E8
:108300000F910895CF93DF93FC0185ADEF01249683
:10831000811105C081E085AFCE010E94A131CE015F
:10832000DF91CF910C94D8316FEF7FEF1ACD6FEFC3
:108330007FEFFACC4FEF5FEFC4CC482F50E0209195
:108340006404022E000C330B4217530781F0809314
:108350006404813031F468EC7FE18BE694E00C94A6
:108360002C3768ED77E18BE694E00C942C37089578
:10837000EF92FF920F938AE8E82E8DE1F82E00E449
:1083800028E040E060E08BE694E00E9424326BE25B
:1083900073E08BE694E00E942C3723E433E041E164
:1083A00069E38BE694E00E943D366BE97BE08BE667
:1083B00094E00E942C3720E533E04CE16AE38BE641
:1083C00094E00E943D3666EF7EE08BE694E00E94EA
:1083D0002C3720E633E049E26BE38BE694E00E9421
:1083E0003D3666EF7EE08BE694E00E942C372CE66B
:1083F00033E04EE36DE38BE694E00E943D362EE6DB
:1084000033E04EE362E48BE694E00E943D3668ED93
:1084100077E18BE694E00F91FF90EF900C942C376E
:1084200087E694E06FDF61E080E0A2DF8BE694E016
:108430000E94DC318111F7CF64EC79E080E090E0BC
:108440000C947D9CEF92FF920F9385E0E82E8DE1D6
:10845000F82E03E127E047E064E28BE694E00E9417
:10846000243283E06ADF2EE633E04BE265E28BE6FE
:1084700094E00E943D3628E733E047E367E08BE66F
:1084800094E00F91FF90EF900C943D3687E694E0D6
:1084900039DFD8DF8BE694E00E94DC318111F9CF1F
:1084A00064EC79E080E090E00C947D9CB9DFEECF45
:1084B00060E070E088EC9FE1C9CD1F93CF93DF931C
:1084C000D5DBC0916C04C695C69587E694E01ADFAB
:1084D000DC2FDD0F1D2F1C0F83E02FDF6C2F80E0C2
:1084E000E5DB8BEF96E023DF6D2F80E0DFDB8AE1B9
:1084F00097E11ADF612F80E0D9DB8DE097E114DF8F
:108500008BE694E00E94DC318111E6CFDF91CF91C0
:108510001F9108950895CF93E62F6CE0869F602DFC
:10852000112481E0860F80936604645F6093650484
:10853000462F50E04E5F5F4F20919F0430E042177E
:1085400053070CF445C090E02091A10430E082175D
:1085500093070CF03DC0CE2F8EE3A8DB65E470E0FE
:1085600080E090E0E7DE61E36C0F062E000C770BF5
:10857000880B990BDFDE60E270E080E090E0DADEED
:1085800060912E0D70912F0D8091300D9091310DD5
:108590000F949B4ECB010E94169DC9DE6FE270E0E6
:1085A00080E090E0C7DE0E94AA7F811109C085E0CB
:1085B000C89FF0011124E55EF24F8481811108C04B
:1085C0008091320D9091330D0E94169DCF91AFCEC8
:1085D000CF910895CF92DF92EF92FF920F931F9366
:1085E000CF93DF931F921F92CDB7DEB77B01622F2F
:1085F00049833DDE4981882309F440C0442309F1C1
:1086000001151105F1F4C7010E94187E25E130E043
:10861000281B310937FF02C02F5F3F4F3595279543
:1086200030E82158822F830F87FD0CC060E270E094
:1086300080E090E02A8339837DDE398131502A81C0
:10864000F1CF30E8C32ED12CB601C7018ADB760109
:10865000E81AF90A0115110511F41E2D06C0FF24B0
:10866000B701C80161DB1E2D181B173038F060E21E
:1086700070E080E090E05EDE181BF7CF0F900F9067
:10868000DF91CF911F910F91FF90EF90DF90CF90EE
:1086900008950F93CF93DF93982F862FEA01692FC8
:1086A000E6DD882309F162E770E0CE015ADBC2E71C
:1086B000C81BC73038F060E270E080E090E03ADE3E
:1086C000C81BF7CF609165048AE7F0DA602F000FCE
:1086D000770B880B990B2EDE60E270E080E090E073
:1086E000DF91CF910F9126CEDF91CF910F91089519
:1086F000CF92DF92EF92FF920F931F93CF93DF936E
:10870000982F862F6A017901692FB1DD882309F43A
:1087100042C0C701002321F00E94187E182F03C019
:108720000E94F77D182FC3E1D0E0C11BD1098C2F27
:10873000880FC80FCC0FD0E0BE01C60112DBC81BEA
:108740006AE370E080E090E0F5DDC73038F060E289
:1087500070E080E090E0EEDDC81BF7CF8AEF189F55
:10876000802D1124609165048058A0DAC701002390
:1087700049F0DF91CF911F910F91FF90EF90DF9023
:10878000CF90D2CDDF91CF911F910F91FF90EF90BD
:10879000DF90CF90CCCDDF91CF911F910F91FF90C3
:1087A000EF90DF90CF900895BF92CF92DF92EF923B
:1087B000FF920F931F93CF93DF936C017B010E9475
:1087C000187EC82FC7010E94F77D082F10E08C2F5C
:1087D00090E023E130E0201B310BBB24B394281739
:1087E00039071CF0B12CC5E201C0CFE12C2F30E0DD
:1087F000A9014E5F5F4F80919F0490E04817590791
:1088000044F0295031098091A10490E08217930728
:10881000C4F5D0E0E114F10409F43AC06AE370E071
:1088200080E090E087DDBB2081F0C45F80919F04F1
:10883000C81770F12C2F30E0295031098091A10424
:1088400090E0821793071CF423C0DD2309F124E193
:1088500030E0201B310B822F880F820F6C2F880F86
:1088600025DA60E270E080E090E064DDC701DF912E
:10887000CF911F910F91FF90EF90DF90CF90BF901D
:1088800056CD6C2F80E012DAC6014EDDD1E0C2CFAA
:10889000DF91CF911F910F91FF90EF90DF90CF90DC
:1088A000BF900895CF92DF92EF92FF920F931F93A4
:1088B000CF93DF931F92CDB7DEB7182F7A01D22E58
:1088C000CA0169830E94187E082F812F880F810FAB
:1088D000C82ECC0C1CE06981169F100D1124DD20E0
:1088E000C1F061E08BE694E00E94FA31202F220F64
:1088F000200F220F2E5F0BE047EF410F6FEF6C0D43
:108900008BE694E00E949C3460E08BE694E00E9449
:10891000FA31612F8C2DCAD9C70106DDDD2071F037
:1089200061E08BE694E00F90DF91CF911F910F9162
:10893000FF90EF90DF90CF900C94FA310F90DF9181
:10894000CF911F910F91FF90EF90DF90CF900895FE
:10895000AF92BF92DF92EF92FF920F931F93CF934C
:10896000DF93EC015B01D42EC901B801A7010E947D
:10897000407F91E02D2D2927A50164E081E092DF61
:10898000CE010E94187E2D2DAE0164E094E1981B6B
:10899000892FDF91CF911F910F91FF90EF90DF9082
:1089A000BF90AF907FCFEF92FF920F93CF93DF9363
:1089B000D82FC62F7901682F8C2F59DC8823D9F046
:1089C000002329F062E070E080E090E0B3DC2D2F1E
:1089D0004C2F64E1C7010E948F7E68E770E0A4D944
:1089E000C8E7C81BC73038F060E270E080E090E074
:1089F000A1DCC81BF7CFDF91CF910F91FF90EF90D3
:108A000008958F929F92AF92BF92CF92DF92EF9292
:108A1000FF920F936B017C01809060049090610441
:108A2000A0906204B0906304A50194010F942C4EB1
:108A3000882301F120E030E0A901C701B6010F94BD
:108A40002C4E882351F0A5019401C701B6010F9463
:108A50002C4E87FD04C081E003C080E001C08FEF91
:108A600080935F04C0926004D0926104E09262043B
:108A7000F092630480919F04813128F48091A104D5
:108A8000833008F048C080919F04853128F480919C
:108A9000A104843108F04FC080919F048F3308F007
:108AA00057C08091A1048F3208F452C080915F04B6
:108AB00040E3481B8EE5E82E87E1F82E0DE022E02A
:108AC0006AE58BE694E00E94243280915F0441E3E2
:108AD000481B94E4E92E97E1F92E22E065E08BE64D
:108AE00094E00E94243228E7E22E27E1F22E00E1F2
:108AF00023E04FE262E18BE694E00E94243238EA00
:108B0000E32E37E1F32E23E04FE267E68BE694E0B5
:108B10000E9424321DC080915F0444E0481B59E24A
:108B2000E52E57E1F52E0CE022E062E48BE694E0BE
:108B30000E942432A8CF41E4E42E47E1F42E01E064
:108B400023E044E16CE38BE694E00E942432A4CF5E
:108B50000F91FF90EF90DF90CF90BF90AF909F90DC
:108B60008F900895CF92EF920F93CF93DF93C7E644
:108B7000D4E01B821A8280E993E099838883CC2415
:108B8000CA94EE24EA9406E427E448E465E172E03E
:108B9000CE010E94DB388CE993E099838883DF91D2
:108BA000CF910F91EF90CF9008959091050194701F
:108BB0009093030187FD76C0A3989091050190954D
:108BC0009470909303019091050194709093030128
:108BD000982F990F86FD72C0A3988091050180950A
:108BE0008470809303018091050184708093030158
:108BF000292F220F96FD60C0A398809105018095D2
:108C00008470809303018091050184708093030137
:108C1000922F990F26FD4EC0A39880910501809553
:108C20008470809303018091050184708093030117
:108C3000292F220F96FD3CC0A398809105018095B5
:108C400084708093030180910501847080930301F7
:108C5000922F990F26FD2AC0A39880910501809537
:108C600084708093030180910501847080930301D7
:108C7000292F220F96FD18C0A39880910501809599
:108C800084708093030180910501847080930301B7
:108C900026FD16C0A398809105018095847080936D
:108CA00003010895A39A89CFA39AE7CFA39AD5CFBA
:108CB000A39AC3CFA39AB1CFA39A9FCFA39A8DCFE4
:108CC000A39A809105018095847080930301089593
:108CD0002F923F925F927F929F92AF92BF92CF92DC
:108CE000DF92EF92FF920F931F93CF93DF937C015C
:108CF0001B01942E69018AE0481709F47BC0A5E1A5
:108D00004A134EC0DB011296ED91FC91139712812C
:108D1000C681D781A49A88E28A950000E9F700EE1F
:108D2000010F80E1582E510E98E2792E88EF3DDF39
:108D3000872D8A950000E9F7103208F046C0812F90
:108D40008077806832DF812F8295807F2EDF872DAC
:108D50008A950000E9F780E828DF80E026DF872D8C
:108D60008A950000E9F78AEF20DF872D8A950000B9
:108D7000E9F75E01B0E1AB0EB11C8881807F15DFA1
:108D800089918295807F11DFCA15DB05B1F7872DA8
:108D90008A950000E9F71F5F0F5F1511C7CFA498F0
:108DA0009601492DB101C701DF91CF911F910F911C
:108DB000FF90EF90DF90CF90BF90AF909F907F900B
:108DC0005F903F902F900C945E33802F8077806867
:108DD000ECDE802F8295807FE8DE872D8A9500006B
:108DE000E9F780E8E2DE80E8E0DE872D8A95000082
:108DF000E9F7B9CF9C9AA4989B9AA3988091040113
:108E00008460809304018091050180958470809333
:108E10000301A49AC8E28C2F8A950000E9F788E73D
:108E200090E00E947B3288EFC0DE8C2F8A95000094
:108E3000E9F780E2BADE80E0B8DE8C2F8A95000088
:108E4000E9F780E0B2DE80E8B0DE8C2F8A95000082
:108E5000E9F780E0AADE80E1A8DE8C2F8A95000089
:108E6000E9F78FE090E00E947B3280E29EDE80E4B2
:108E70009CDE8C2F8A950000E9F780E296DE80E682
:108E800094DECA950000E9F710E0D8E208E2812FED
:108E9000807780688ADE812F8295807F86DE8D2FA5
:108EA0008A950000E9F780E880DE80E07EDE8D2F85
:108EB0008A950000E9F78AEF78DE8D2F8A95000009
:108EC000E9F7C0E280E071DE80E06FDE9D2F9A95C9
:108ED0000000E9F7C150B1F788EF67DE802F8A956F
:108EE0000000E9F71F5F103209F0D1CF80E05DDEAE
:108EF00080EC5BDE88E28A950000E9F7A49850CF09
:108F0000A49A88E28A950000E9F7089588EF4DDE7B
:108F100088E28A950000E9F708958AEF46DE88E244
:108F20008A950000E9F70895CF93C82F807F3DDE32
:108F30008C2F8295807F39DE88E28A950000E9F7E0
:108F4000CF910895CF93DF931F921F92CDB7DEB7D5
:108F500089839A830E94347920E040E060E070E0E9
:108F600089819A810F900F90DF91CF910C94D979DC
:108F70000F93CF93DF9361E081E00E94DD7AD0917F
:108F8000C906C0E0D11117C08091C806811104C084
:108F90000E94D97E811165C080912302882309F443
:108FA00057C081E09091C806911180E004E024E070
:108FB0004CED58E24BC0D130C1F48091C8068130ED
:108FC00021F40E94D97E811154C08091230288230C
:108FD00009F43EC081E09091C806913009F080E02C
:108FE00003E02EE343ED58E231C0D230B9F4809172
:108FF000C806823021F40E94D97E811143C080913D
:109000002302882329F181E09091C806923009F06B
:1090100080E003E02EE34AEC58E218C0D330C1F4FC
:109020008091C806833021F40E94D97E811133C01B
:1090300080912302882361F081E09091C8069330EB
:1090400009F080E003E02EE344EC58E26C2F21DBD2
:10905000CF5FDF5FC53009F095CF84E08093C7060E
:1090600021C00E94077A80919506882309F494CF45
:1090700019C082E79FE666DF80919506882309F490
:10908000A4CF10C081E894E75DDF80919506882326
:1090900009F4B5CF07C082E498E754DF80919506C4
:1090A000882331F2DF91CF910F910895CF92DF9213
:1090B000EF92FF920F931F9380915709811103C084
:1090C00089E999E002C087E599E020E2C22E29E211
:1090D000D22E7C0103E119E227E03AE74DE758E49C
:1090E0006CE079E286E099E20E94D57B1F910F91B6
:1090F000FF90EF90DF90CF90089589E999E00E946A
:10910000CF880E94007A0C944C840E946B8D21E0E1
:1091100030E0811102C020E030E03093F00620936F
:10912000EF061092C90681E08093950683E0809354
:1091300023020895CF92DF92EF92FF920F931F9335
:10914000CF93DF930E94698E6C0161E081E00E9401
:10915000DD7AC091C906D0E081E0C81AD108C111FA
:1091600017C08091C806811104C00E94D97E811168
:1091700095C080912302882359F081E09091C80620
:10918000911180E004E024E041E059E26D2F81DAA2
:1091900069E979E080E299E00E945D948091990903
:1091A0008F3201F18091A60983FF1CC0C130C1F448
:1091B0008091C806813021F40E94D97E811176C049
:1091C00080912302882361F081E09091C80691305C
:1091D00009F080E000E22EE34DEF58E26D2F59DAFE
:1091E00092E001C091E080912302882309F44EC0EF
:1091F000760111E01C0F8FEFE816F80609F446C05F
:10920000C9133FC060E070E0C7010E94448A90919A
:10921000A6098091C80694FF1CC08C134EC00E9402
:10922000D97E882309F449C089E999E00E94158D07
:109230001092C90682E090E09093F0068093EF06CA
:1092400081E0809395061092F20683E080932302DA
:1092500052C08C1304C00E94D97E81113DC0809100
:109260002302882361F081E09091C8069C1380E07E
:1092700000E02FE538E141EE58E26D2F94DB912FAD
:1092800001C09F5F81E0E81AF108B5CFDF5FCF5FD3
:10929000D53009F064CF9093C7062DC00E94077A9D
:1092A00080919506882309F464CF25C02EDF809134
:1092B0009506882309F484CF1EC080912302882359
:1092C000F1F281E09091C8069C1380E001E02FE567
:1092D00038E14FEE58E2D1CF0E94347920E040E0EF
:1092E00060E070E086E598E40E94D9798091950667
:1092F000882309F4B4CFDF91CF911F910F91FF9094
:10930000EF90DF90CF900895CF93DF93EC01CB01E6
:10931000BA010F94CE4E0F94A04E6883DF91CF9187
:109320000895CF93DF93EC01CB01BA010F94CE4E99
:109330002FE632E143E85AE30F946A506883798359
:109340008A839B83DF91CF91089564E879E481EB70
:1093500099E40C941C7A61E979E48EEC99E40C941C
:109360001C7A0F94CE4E0F94A04E862F0C94C19C65
:10937000CF93DF9300D01F92CDB7DEB769837A8396
:109380008B839C8360E2CE0101960E94549F0F90D4
:109390000F900F900F90DF91CF9108950F94CE4EC4
:1093A0002FE632E143E85AE30F946A50E1CF2F925F
:1093B0003F924F925F926F927F928F929F92AF9265
:1093C000BF92CF92DF92EF92FF920F931F93CF93B2
:1093D000DF93CDB7DEB729970FB6F894DEBF0FBE87
:1093E000CDBF1C0179876887CA01B901E982FA8279
:1093F0000B831C83DE82CD82AF8220E030E04AE71F
:1094000054E40F946A506B017C0120E030E040E0AE
:1094100057EC0F942F5018162CF0C12CD12CE12CA6
:1094200027ECF22EC701B6010F949B4E2B013C0195
:1094300020E030E04AE754E469817A818B819C81A5
:109440000F946A504B015C0120E03EEF4FEF56E471
:109450000F942C4E87FD07C0812C9EEF992EAA24D5
:10946000AA9496E4B92E20E030E04AE754E4E88577
:10947000F98560817181828193810F946A506B01BB
:109480007C01C301B2010F94CE4E9B01AC01C70118
:10949000B6010F94524D0F94A04E69837A838B834B
:1094A0009C83C501B4010F949B4E7B018C01E41891
:1094B000F50806091709FF81FF938D809E808BEACE
:1094C000A82E89E4B82EC980DA80A30192016885AC
:1094D0007985C1010E945B790F9029960FB6F894A7
:1094E000DEBF0FBECDBFDF91CF911F910F91FF90D7
:1094F000EF90DF90CF90BF90AF909F908F907F9034
:109500006F905F904F903F902F9008958F929F9211
:10951000AF92BF92CF92DF92EF92FF920F931F9381
:10952000CF93DF9361E081E00E94DD7AD091C9069C
:10953000C0E0D11119C08091C806811104C00E94F9
:10954000D97E8111C4C080912302882309F4B6C05A
:1095500081E09091C806911180E004E024E048E5A4
:1095600059E26C2F96D8AAC0D130E1F48091C80698
:10957000813021F40E94D97E8111B1C080912302F3
:10958000882309F49BC011E08091C806813009F05E
:1095900010E08091A30C0E94C19C00E09C0142E479
:1095A00059E289C0D23009F58091C806823021F491
:1095B0000E94D97E8111B4C080912302882309F4CE
:1095C0007DC011E08091C806823009F010E0609102
:1095D000A40C7091A50C8091A60C9091A70CC8DEEC
:1095E00000E09C014EE359E266C0D33009F580915A
:1095F000C806833021F40E94D97E8111AAC08091CF
:109600002302882309F45AC011E08091C8068330F0
:1096100009F010E06091A80C7091A90C8091AA0C3F
:109620009091AB0CA5DE00E09C014AE359E243C0F7
:10963000D43001F58091C806843021F40E94D97E8F
:109640008111A0C0809123028823C1F111E0809193
:10965000C806843009F010E06091AC0C7091AD0C3C
:109660008091AE0C9091AF0C83DE00E09C0146E34C
:1096700059E221C0D53011F58091C806853021F41A
:109680000E94D97E811197C0809123028823B1F076
:1096900011E08091C806853009F010E06091270242
:1096A000709128028091290290912A0261DE00E0E7
:1096B0009C0142E259E26C2F812F1AD8CF5FDF5F05
:1096C000C53009F036CF86E08093C7068CC00E9473
:1096D000077A80919506882309F435CF84C081E00C
:1096E0000E94CE7EC090A30CD12C1F92812C912C75
:1096F00045EAA42E49E4B42EE12CF12C8701EA942A
:1097000020E030E0A90163EA7CE08DE499E20E9468
:109710005B790F9080919506882309F42FCF63C061
:1097200081E00E94CE7EA12CC12CD12C16E6E12E28
:10973000FE2C0EE111E420E030E0A90164EA7CE0B7
:1097400080E499E234DE80919506882309F434CFD1
:109750004AC081E00E94CE7EA12CC12CD12C16E6FD
:10976000E12EFE2C0EE111E420E030E0A90168EAD0
:109770007CE08CE399E21BDE80919506882309F456
:109780003ECF31C081E00E94CE7EA12CC12CD12CD5
:1097900016E6E12EFE2C0EE111E420E030E0A901F6
:1097A0006CEA7CE088E399E202DE809195068823EA
:1097B00009F448CF18C081E00E94CE7EA12CC12CB4
:1097C000D12C16E6E12EFE2C0EE111E420E030E073
:1097D000A90167E272E08CE299E2E9DD80919506E9
:1097E000882309F451CFDF91CF911F910F91FF9002
:1097F000EF90DF90CF90BF90AF909F908F900895A3
:10980000CF93DF93EC01CB01BA010F94CE4E2AE047
:1098100037ED43E25CE30F946A50688379838A836F
:109820009B83DF91CF910895CF93DF93EC01CB0120
:10983000BA010F94CE4E688379838A839B83DF912C
:10984000CF910895CF93DF93EC01CB01BA010F9430
:10985000CE4E20E030E048EC51E40F946A5068832B
:1098600079838A839B83DF91CF910895CF93DF9390
:10987000EC01CB01BA010F94CE4E20E030E048EC71
:1098800052E40F946A50688379838A839B83DF91C3
:10989000CF910895CF93DF93EC01CB01BA010F94E0
:1098A000CE4E20E030E048EC51E40F946A500F9423
:1098B000A04E688379838A839B83DF91CF9108953B
:1098C000CF93DF93EC01CB01BA010F94CE4E20E091
:1098D00030E048EC52E40F946A500F94A04E688335
:1098E00079838A839B83DF91CF910895CF93DF9310
:1098F000EC01CB01BA010F94CE4E2AE037ED43E2E2
:109900005CE30F946A50688379838A839B83DF9139
:10991000CF910895CF93DF93EC01CB01BA010F945F
:10992000CE4E2DEC3CEC4CEC5DE30F946A5068831A
:1099300079838A839B83DF91CF91089560E07CE4F3
:109940008FEE9CE40C941C7A64E17CE487EA9DE44D
:109950000C941C7A66E37CE489E29DE40C941C7A06
:1099600062E27CE48CE09DE40C941C7A6AE47CE482
:109970008AEE90E50C941C7A60E67CE483E69DE434
:109980000C941C7A66E77CE486E49DE40C941C7AD3
:109990006AE87CE482ED9CE40C941C7A0D949504B6
:1099A0000D94DC04CF93DF9300D01F92CDB7DEB7C8
:1099B0000F94CE4E2DEC3CEC4CEC5DE30F946A50D2
:1099C00069837A838B839C83CE0101960E94F6A1E2
:1099D0000F900F900F900F90DF91CF910895CF933C
:1099E000DF9300D01F92CDB7DEB70F94CE4E2AE0A2
:1099F00037ED43E25CE30F946A5069837A838B838B
:109A00009C83CE0101960E94169E0F900F900F909E
:109A10000F90DF91CF910895CF93DF9300D01F92E5
:109A2000CDB7DEB70F94CE4E20E030E048EC51E4E5
:109A30000F946A5069837A838B839C83CE0101964D
:109A40000E949DA00F900F900F900F90DF91CF91EB
:109A50000895CF93DF9300D01F92CDB7DEB70F9458
:109A6000CE4E20E030E048EC52E40F946A50698317
:109A70007A838B839C83CE0101960E949DA00F90D8
:109A80000F900F900F90DF91CF910895CF93DF93B8
:109A900000D01F92CDB7DEB70F94CE4E2AE037ED3F
:109AA00043E25CE30F946A5069837A838B839C83DF
:109AB000CE0101960E9455A10F900F900F900F902C
:109AC000DF91CF910895CF93DF9300D01F92CDB750
:109AD000DEB70F94CE4E20E030E048EC52E40F9415
:109AE0006A500F94A04E0F94CC4E69837A838B8377
:109AF0009C83CE0101960E949DA00F900F900F9025
:109B00000F90DF91CF910895CF92DF92EF92FF9265
:109B10006B017C0120E030E0A9010F942C4E87FD01
:109B200005C020E030E040E05FE304C020E030E02A
:109B300040E05FEBC701B6010F94534D0F949B4E6D
:109B4000CB01FF90EF90DF90CF900C94169D0F9477
:109B5000CE4EDACFCF93DF9300D01F92CDB7DEB7D2
:109B60000F94A04E0F94CC4E69837A838B839C8391
:109B7000CE0101960E949DA00F900F900F900F9024
:109B8000DF91CF9108956F927F928F929F92AF92C3
:109B9000BF92CF92DF92EF92FF920F931F93CF93DA
:109BA000DF9300D01F92CDB7DEB761E081E00E9465
:109BB000DD7A6090C906712C61101AC08091C806C8
:109BC000811104C00E94D97E811159C18091230264
:109BD000882309F44BC181E09091C806911180E07F
:109BE00004E024E04FEB5AE2672D0E9449433EC156
:109BF00081E068122CC08091C806813021F40E9457
:109C0000D97E811144C180912302882309F42EC199
:109C100011E08091C806813009F010E08091E40ED7
:109C20009091E50EA091E60EB091E70E89839A839C
:109C3000AB83BC83CE0101960E949DA000E09C01F5
:109C400043EB5AE2672D812F0E9478430FC182E0D7
:109C500068122CC08091C806823021F40E94D97EFF
:109C600081114DC180912302882309F4FFC011E0C6
:109C70008091C806823009F010E08091E80E909142
:109C8000E90EA091EA0EB091EB0E89839A83AB8323
:109C9000BC83CE0101960E949DA000E09C014FE98B
:109CA0005AE2672D812F0E947843E0C083E068125A
:109CB0002CC08091C806833021F40E94D97E811186
:109CC00056C180912302882309F4D0C011E080910D
:109CD000C806833009F010E08091EC0E9091ED0EF3
:109CE000A091EE0EB091EF0E89839A83AB83BC8373
:109CF000CE0101960E949DA000E09C014DE85AE231
:109D0000672D812F0E947843B1C084E0681227C07C
:109D10008091C806843021F40E94D97E81115FC1F0
:109D200080912302882309F4A1C011E08091C80624
:109D3000843009F010E06091B00E7091B10E809106
:109D4000B20E9091B30E0F94CC4E04DF00E09C0154
:109D50004FE75AE2672D812F0E94784387C085E044
:109D6000681227C08091C806853021F40E94D97EF0
:109D7000811171C180912302882309F477C011E019
:109D80008091C806853009F010E06091B40E7091A2
:109D9000B50E8091B60E9091B70E0F94CC4EDADED0
:109DA00000E09C0141E75AE2672D812F0E94784331
:109DB0005DC086E0681227C08091C806863021F415
:109DC0000E94D97E811183C180912302882309F4E6
:109DD0004DC011E08091C806863009F010E0609116
:109DE000B80E7091B90E8091BA0E9091BB0E0F947F
:109DF000CC4EB0DE00E09C0143E65AE2672D812F95
:109E00000E94784333C087E0681230C08091C80652
:109E1000873021F40E94D97E81118EC18091230266
:109E2000882321F111E08091C806873009F010E005
:109E30006091BC0E7091BD0E8091BE0E9091BF0ED0
:109E40000F94CC4E0F94A04E0F94CC4E69837A831E
:109E50008B839C83CE0101960E949DA000E09C0113
:109E600045E55AE2672D812F0E94784373946394ED
:109E700085E07812A1CE88E08093C70698C10E9441
:109E8000077A80919506882309F4A0CE90C181E0DD
:109E90000E94CE7E2AE037ED43E25DE36091E40E5E
:109EA0007091E50E8091E60E9091E70E0F946A5046
:109EB00020E030E040E85FE30F94524D0F94A04E55
:109EC0001F92812C912C50EBA52E5CE4B52E6B01DA
:109ED00017E7E12E1FE0F12E00E010E021E030E076
:109EE00040E050E064EE7EE089EB9AE20E945B790C
:109EF0000F9080919506882309F485CE58C181E0A2
:109F00000E94CE7E2AE037ED43E25CE36091E80EEA
:109F10007091E90E8091EA0E9091EB0E0F946A50C9
:109F200020E030E040E85FE30F94524D0F94A04EE4
:109F30001F92812C912C3AEAA32E3CE4B32E6B01A4
:109F40001DEDE12E13E0F12E00E010E021E030E005
:109F500040E050E068EE7EE089EA9AE20E945B7998
:109F60000F9080919506882309F47CCE20C181E072
:109F70000E94CE7E2AE037ED43E25DE36091EC0E75
:109F80007091ED0E8091EE0E9091EF0E0F946A504D
:109F900020E030E040E85FE30F94524D0F94A04E74
:109FA0001F92812C912C90EBA92E9CE4B92E6B0171
:109FB00017E7E12E1FE0F12E00E010E021E030E095
:109FC00040E050E06CEE7EE086E99AE20E945B7928
:109FD0000F9080919506882309F473CEE8C081E044
:109FE0000E94CE7E6091B00E7091B10E8091B20E43
:109FF0009091B30E0F94CC4E2AE037ED43E25DE32F
:10A000000F946A5020E030E040E850E40F94524D45
:10A010000F94A04E1F92BEEC8B2EBCE49B2E16EB31
:10A02000A12E1CE4B12E6B0114E7E12E1FE0F12EEE
:10A0300000E010E024E030E040E050E060EB7EE043
:10A0400086E89AE20E945B790F90809195068823BA
:10A0500009F466CEACC081E00E94CE7E6091B40E61
:10A060007091B50E8091B60E9091B70E0F94CC4EB4
:10A070002AE037ED43E25DE30F946A5020E030E0E0
:10A0800040E850E40F94524D0F94A04E1F92EEEC16
:10A090008E2EECE49E2EF6EBAF2EFCE4BF2E6B0171
:10A0A00014E7E12E1FE0F12E00E010E024E030E0A4
:10A0B00040E050E064EB7EE088E79AE20E945B7942
:10A0C0000F9080919506882309F454CE70C081E0EA
:10A0D0000E94CE7E6091B80E7091B90E8091BA0E3A
:10A0E0009091BB0E0F94CC4E2AE037ED43E25DE336
:10A0F0000F946A500F94A04E1F923EEC832E3CE4C6
:10A10000932E46EBA42E4CE4B42E6B0118E7E12EFF
:10A110001FE0F12E00E010E020E030E0A90168EB44
:10A120007EE08AE69AE20E945B790F908091950624
:10A13000882309F449CE3BC081E00E94CE7E609125
:10A14000BC0E7091BD0E8091BE0E9091BF0E0F940B
:10A15000CC4E2AE037ED43E25CE30F946A5020E0F6
:10A1600030E040E85FE30F94524D0F94A04E1F92F1
:10A170008EEC882E8CE4982E9CEBA92E9CE4B92EB4
:10A180006B011DEDE12E13E0F12E00E010E021E067
:10A1900030E040E050E06CEB7EE08CE59AE20E941B
:10A1A0005B790F9080919506882309F437CE0F9044
:10A1B0000F900F900F90DF91CF911F910F91FF9013
:10A1C000EF90DF90CF90BF90AF909F908F907F9057
:10A1D0006F9008950F94CE4E20E030E048EC51E4AB
:10A1E0000F946A50B7CC0F931F93CF93DF9361E026
:10A1F00081E00E94DD7AC091C906D0E0C1111AC089
:10A200008091C806811104C00E94D97E8111CCC002
:10A2100080912302882309F461C081E09091C806EF
:10A22000911180E004E024E043E959E26D2F0E949F
:10A23000494354C0C130D9F48091C806813021F41B
:10A240000E94D97E8111B8C080912302882309F42D
:10A2500045C081E09091C806913009F080E003E0AC
:10A260002EE34AE859E26D2F0E94494337C0C230BD
:10A27000D1F48091C806823021F40E94D97E8111E8
:10A28000A5C080912302882349F181E09091C806FE
:10A29000923009F080E003E02EE34DE759E26D2FA4
:10A2A0000E9449431BC0C330C9F48091C806833063
:10A2B00021F40E94D97E811193C0809123028823CA
:10A2C00069F081E09091C806933009F080E003E0E6
:10A2D0002EE348E759E26D2F0E9449430E94C2795C
:10A2E00081111DC0C430E9F48091C806843021F486
:10A2F0000E94D97E81117EC080912302882309F4B7
:10A3000083C081E09091C806943009F080E003E0BA
:10A310002EE34FE659E26D2F0E94494375C014E0C9
:10A3200001C015E0C1131BC08091C8068C1304C086
:10A330000E94D97E81116AC080912302882371F026
:10A3400081E09091C8069C1380E003E02EE346E68E
:10A3500059E26D2F0E9449431C2F01C01C2F81E040
:10A36000810FC81318C08091C8068C1304C00E94C6
:10A37000D97E811155C080912302882361F081E04C
:10A380009091C8069C1380E003E02EE34DE559E26E
:10A390006D2F0E944943DF5FCF5FD53009F02ECF8C
:10A3A0001E5F1093C70645C00E94077A80919506EC
:10A3B000882309F42DCF3DC08CED93E50E94A24780
:10A3C00080919506882309F43FCF33C083EC9DE448
:10A3D0000E94A24780919506882309F452CF29C094
:10A3E00084EA95E50E94A24780919506882309F4A6
:10A3F00064CF1FC088ED97E50E94A2478091950623
:10A40000882309F479CF15C015E0A9CF86E89AE42E
:10A410000E94A24780919506882309F48DCF09C038
:10A4200089EA92E50E94A24780919506882309F463
:10A43000A2CFDF91CF911F910F9108952F923F925C
:10A440004F925F926F927F928F929F92AF92BF9244
:10A45000CF92DF92EF92FF920F931F93CF93DF93F0
:10A4600000D000D0CDB7DEB71C017E836D832901FB
:10A470003A01460120E030E040E057ECB201C30170
:10A480000F942F5018162CF0412C512C612C27ECD6
:10A4900001C0272DB201862D922F0F949B4E2B01C8
:10A4A0003C0120E03EEF4FEF56E4B701C8010F94A6
:10A4B0002C4E87FD06C0B12C9EEFF92E0FEF16E44F
:10A4C00001C0BE2CC301B2010F94CE4E9B01AC0162
:10A4D000ED81FE8160817181828193810F94524D63
:10A4E0000F94A04E69837A838B839C836B2D7F2D81
:10A4F000C8010F949B4E7B018C01E418F5080609F6
:10A500001709AF9284EAA82E8CE4B82EC980DA80AD
:10A51000A30192016D817E81C1010E945B790F9040
:10A5200026960FB6F894DEBF0FBECDBFDF91CF9158
:10A530001F910F91FF90EF90DF90CF90BF90AF9061
:10A540009F908F907F906F905F904F903F902F9053
:10A5500008956F927F928F929F92AF92BF92CF9207
:10A56000DF92EF92FF920F931F93CF93DF9300D070
:10A570001F92CDB7DEB761E081E00E94DD7A609086
:10A58000C906712C61101AC08091C806811104C0DF
:10A590000E94D97E811198C080912302882309F4FA
:10A5A0008AC081E09091C806911180E004E024E027
:10A5B00041E75BE2672D0E9449437DC081E068125C
:10A5C0002CC08091C806813021F40E94D97E81116F
:10A5D00083C080912302882309F46DC011E080912B
:10A5E000C806813009F010E08091220E9091230E70
:10A5F000A091240EB091250E89839A83AB83BC83EE
:10A60000CE0101960E94169E00E09C014DE55BE2A2
:10A61000672D812F0E9478434EC082E0681225C0CA
:10A620008091C806823021F40E94D97E811182C0B7
:10A6300080912302882309F43EC011E08091C8066E
:10A64000823009F010E060917C0C70917D0C80915B
:10A650007E0C90917F0C58DA00E09C0149E45BE2AB
:10A66000672D812F0E94784326C083E0681223C0A3
:10A670008091C806833021F40E94D97E811172C076
:10A68000809123028823B9F011E08091C8068330BD
:10A6900009F010E06091800C7091810C8091820C27
:10A6A0009091830C31DA00E09C0149E35BE2672D75
:10A6B000812F0E9478437394639485E0781262CF6F
:10A6C00084E08093C70665C00E94077A8091950652
:10A6D000882309F461CF5DC020E030E048EC52E40B
:10A6E0006091220E7091230E8091240E9091250E80
:10A6F0000F946A500F94A04E1F92812C912C2EE93A
:10A70000A22E2CE4B22E6B01EE24EA941FE7F12E68
:10A7100000E010E020E030E0A90162E27EE087E6A0
:10A720009BE20E945B790F9080919506882309F443
:10A7300050CF2FC081E00E94CE7EA12CC12CD12C05
:10A74000E12CF12C08E413E420E030E0A9016CE7EF
:10A750007CE083E59BE272DE80919506882309F414
:10A7600067CF17C081E00E94CE7EA12CC12CD12CD6
:10A77000E12CF12C08E413E420E030E0A90160E8CA
:10A780007CE081E49BE25ADE80919506882309F4FF
:10A7900077CF0F900F900F900F90DF91CF911F9177
:10A7A0000F91FF90EF90DF90CF90BF90AF909F9070
:10A7B0008F907F906F900895AF92CF92DF92EF923B
:10A7C000FF920F931F93CF93DF9361E081E00E948C
:10A7D000DD7AD091C906C0E0D1111AC08091C806B7
:10A7E000811104C00E94D97E811103C1809123028E
:10A7F000882309F4F5C081E09091C806911180E0AA
:10A8000004E024E047E25BE26C2F0E944943E8C089
:10A81000D13029F58091C806813021F40E94D97E7B
:10A820008111EFC080912302882309F4D9C011E07F
:10A830008091C806813009F010E06091D40E7091CB
:10A84000D50E8091D60E9091D70E5ED900E09C0176
:10A8500049E15BE26C2F812F0E947843C1C0D23066
:10A8600029F58091C806823021F40E94D97E811199
:10A87000E2C080912302882309F4B2C011E08091E4
:10A88000C806823009F010E06091D80E7091D90EA0
:10A890008091DA0E9091DB0E37D900E09C014BE0FD
:10A8A0005BE26C2F812F0E9478439AC0D33029F548
:10A8B0008091C806833021F40E94D97E8111D5C0D1
:10A8C00080912302882309F48BC011E08091C8068F
:10A8D000833009F010E06091DC0E7091DD0E809104
:10A8E000DE0E9091DF0E10D900E09C014DEF5AE290
:10A8F0006C2F812F0E94784373C0D43029F580914A
:10A90000C806843021F40E94D97E8111C8C080918C
:10A910002302882309F464C011E08091C8068430C2
:10A9200009F010E06091E00E7091E10E8091E20E6E
:10A930009091E30EE9D800E09C014FEE5AE26C2FB3
:10A94000812F0E9478434CC0D53029F58091C806EC
:10A95000853021F40E94D97E8111BBC080912302F1
:10A96000882309F43DC011E08091C806853009F0C4
:10A9700010E06091F00E7091F10E8091F20E9091C6
:10A98000F30EC2D800E09C0145EE5AE26C2F812FF5
:10A990000E94784325C0D63019F58091C8068630CC
:10A9A00021F40E94D97E8111ADC0809123028823B9
:10A9B000B9F011E08091C806863009F010E060918E
:10A9C000F40E7091F50E8091F60E9091F70E9CD8D2
:10A9D00000E09C0141ED5AE26C2F812F0E947843E8
:10A9E000CF5FDF5FC53009F0F7CE87E08093C70601
:10A9F000A1C00E94077A80919506882309F4F6CEBB
:10AA000099C081E00E94CE7EA12CC12CD12CE12CDA
:10AA100010ECF12E09E714E420E030E040E85FE3B9
:10AA200064ED7EE080E29BE209DD8091950688235B
:10AA300009F4F8CE7FC081E00E94CE7EA12CC12C0B
:10AA4000D12CE12C10ECF12E09E714E420E030E0E9
:10AA500040E85FE368ED7EE082E19BE2EFDC80911D
:10AA60009506882309F405CF65C081E00E94CE7E5B
:10AA7000A12CC12CD12CE12C10ECF12E09E714E40F
:10AA800020E030E040E85FE36CED7EE084E09BE2B4
:10AA9000D5DC80919506882309F412CF4BC081E064
:10AAA0000E94CE7EA12CC12CD12CE12C10ECF12ED9
:10AAB00009E714E420E030E040E85FE360EE7EE088
:10AAC00086EF9AE2BBDC80919506882309F41FCFBC
:10AAD00031C081E00E94CE7EA12CC12CD12CE12C72
:10AAE00010ECF12E09E714E420E030E0A90160EF5A
:10AAF0007EE08AEE9AE2A2DC80919506882309F432
:10AB00002DCF18C081E00E94CE7EA12CC12CD12C6B
:10AB1000E12C10ECF12E09E714E420E030E0A9016B
:10AB200064EF7EE08BED9AE289DC809195068823C4
:10AB300009F43BCFDF91CF911F910F91FF90EF90E0
:10AB4000DF90CF90AF9008956F927F928F929F92F7
:10AB5000AF92BF92CF92DF92EF92FF920F931F932B
:10AB6000CF93DF9300D01F92CDB7DEB761E081E0D5
:10AB70000E94DD7A6090C906712C61101AC0809124
:10AB8000C806811104C00E94D97E8111C2C0809183
:10AB90002302882309F4B5C081E09091C806911181
:10ABA00080E004E024E043E45AE2672D0E94494338
:10ABB000A8C081E0681226C08091C806813021F4C7
:10ABC0000E94D97E8111ADC080912302882309F4AF
:10ABD00098C011E08091C806813009F010E06091C2
:10ABE000800E7091810E8091820E9091830E0E9452
:10ABF000844D00E09C0143E35AE2672D812F0E94BF
:10AC000078437FC082E0681226C08091C8068230F7
:10AC100021F40E94D97E81119EC080912302882355
:10AC200009F46FC011E08091C806823009F010E08D
:10AC30006091840E7091850E8091860E9091870EA2
:10AC40000E94844D00E09C0143E25AE2672D812F6F
:10AC50000E94784356C083E068122CC08091C806D9
:10AC6000833021F40E94D97E81118FC0809123020C
:10AC7000882309F446C011E08091C806833009F0AA
:10AC800010E08091880E9091890EA0918A0EB0916B
:10AC90008B0E89839A83AB83BC83CE0101960E947D
:10ACA00055A100E09C0143E15AE2672D812F0E94EB
:10ACB000784327C084E0681224C08091C80684309D
:10ACC00021F40E94D97E811198C0809123028823AB
:10ACD000C1F011E08091C806843009F010E0609165
:10ACE0008C0E70918D0E80918E0E90918F0E0E9421
:10ACF000844D00E09C0143E05AE2672D812F0E94C1
:10AD000078437394639485E0781237CF7092C706C6
:10AD10008DC00E94077A80919506882309F437CF69
:10AD200085C081E00E94CE7EA12CC12CD12CE12CCB
:10AD300010E8F12E07E714E420E030E040E85FE39C
:10AD400060E87EE08BE39AE279DB809195068823C8
:10AD500009F43ACF6BC081E00E94CE7EA12CC12CB9
:10AD6000D12CE12C10E8F12E07E714E420E030E0CC
:10AD700040E85FE364E87EE08BE29AE25FDB80918B
:10AD80009506882309F449CF51C081E00E94CE7E08
:10AD900020E030E048EC52E46091880E7091890E1A
:10ADA00080918A0E90918B0E0F946A5020E030E0D3
:10ADB00040E251E40F94524D0F94A04E1F92812C0B
:10ADC000912C92ECA92E9CE4B92E6B0115EFE12E8B
:10ADD0001FE7F12E00E010E02AE030E040E050E014
:10ADE00068E87EE08BE19AE20E945B790F908091A7
:10ADF0009506882309F43ACF19C081E00E94CE7EDF
:10AE0000A12CC12CD12CE12C10E8F12E07E714E481
:10AE100020E030E040E85FE36CE87EE08BE09AE21F
:10AE20000DDB80919506882309F44FCF0F900F908A
:10AE30000F900F90DF91CF911F910F91FF90EF90A6
:10AE4000DF90CF90BF90AF909F908F907F906F904A
:10AE500008952F923F924F925F926F927F928F92BE
:10AE60009F92AF92BF92CF92DF92EF92FF920F9399
:10AE70001F93CF93DF93CDB7DEB729970FB6F89422
:10AE8000DEBF0FBECDBF1C0179876887CA01B9013B
:10AE9000E982FA820B831C83DE82CD82AF8220E0BE
:10AEA00030E040E251E40F946A506B017C0120E0F5
:10AEB00030E040E057EC0F942F5018162CF0C12CC6
:10AEC000D12CE12C27ECF22EC701B6010F949B4E3A
:10AED0002B013C0120E030E040E251E469817A81BD
:10AEE0008B819C810F946A504B015C0120E03EEF06
:10AEF0004FEF56E40F942C4E87FD07C0812C9EEF38
:10AF0000992EAA24AA9496E4B92E20E030E040E2DB
:10AF100051E4E885F98560817181828193810F9484
:10AF20006A506B017C01C301B2010F94CE4E9B01AC
:10AF3000AC01C701B6010F94524D0F94A04E698326
:10AF40007A838B839C83C501B4010F949B4E7B0154
:10AF50008C01E418F50806091709FF81FF938D801D
:10AF60009E8088ECA82E8CE4B82EC980DA80A301DC
:10AF7000920168857985C1010E945B790F902996BD
:10AF80000FB6F894DEBF0FBECDBFDF91CF911F91FA
:10AF90000F91FF90EF90DF90CF90BF90AF909F9078
:10AFA0008F907F906F905F904F903F902F9008957B
:10AFB0009F92AF92BF92CF92DF92EF92FF920F9348
:10AFC0001F93CF93DF9300D01F92CDB7DEB761E020
:10AFD00081E00E94DD7A9090C906B12C91101AC0D0
:10AFE0008091C806811104C00E94D97E8111D4C00D
:10AFF00080912302882309F4C7C081E09091C8069C
:10B00000911180E004E024E041EF59E26B2D0E94B1
:10B010004943BAC081E098122CC08091C8068130A3
:10B0200021F40E94D97E8111BFC080912302882320
:10B0300009F4AAC011E08091C806813009F010E03F
:10B040008091C40E9091C50EA091C60EB091C70E0E
:10B0500089839A83AB83BC83CE0101960E94F6A1BB
:10B0600000E09C014DED59E26B2D812F0E94784349
:10B070008BC082E098122CC08091C806823021F4E7
:10B080000E94D97E8111ACC080912302882309F4EB
:10B090007BC011E08091C806823009F010E08091F9
:10B0A000C80E9091C90EA091CA0EB091CB0E8983A3
:10B0B0009A83AB83BC83CE0101960E94F6A100E087
:10B0C0009C0149EC59E26B2D812F0E9478435CC0B2
:10B0D00083E098122CC08091C806833021F40E942E
:10B0E000D97E811199C080912302882309F44CC034
:10B0F00011E08091C806833009F010E08091CC0EF9
:10B100009091CD0EA091CE0EB091CF0E89839A83EF
:10B11000AB83BC83CE0101960E94F6A100E09C01A6
:10B1200045EB59E26B2D812F0E9478432DC084E0BE
:10B1300098122AC08091C806843021F40E94D97EDA
:10B14000811186C0809123028823F1F011E0809163
:10B15000C806843009F010E08091D00E9091D10E95
:10B16000A091D20EB091D30E89839A83AB83BC8316
:10B17000CE0101960E94F6A100E09C0141EA59E24D
:10B180006B2D812F0E947843B394939485E0B8127D
:10B1900025CFB092C70677C00E94077A80919506A6
:10B1A000882309F425CF6FC081E00E94CE7EA12CB8
:10B1B00060EDC62E6CE4D62EE12C1CE3F12E0CE1E2
:10B1C00016E420E030E040EA50E464EC7EE087EEF4
:10B1D00099E23FDE80919506882309F426CF53C07B
:10B1E00081E00E94CE7EA12C40EDC42E4CE4D42EF2
:10B1F000E12C1CE3F12E0CE116E420E030E040EA03
:10B2000050E468EC7EE083ED99E223DE80919506C0
:10B21000882309F439CF37C081E00E94CE7EA12C6B
:10B2200020EDC22E2CE4D22EE12C1CE3F12E0CE1F9
:10B2300016E420E030E040EA50E46CEC7EE08FEB76
:10B2400099E207DE80919506882309F44CCF1BC054
:10B2500081E00E94CE7EA12C80EDC82E8CE4D82EF9
:10B26000E12C1CE3F12E0CE116E420E030E040EA92
:10B2700050E460ED7EE08BEA99E2EBDD809195068B
:10B28000882309F45FCF0F900F900F900F90DF91FC
:10B29000CF911F910F91FF90EF90DF90CF90BF90D3
:10B2A000AF909F9008950F93CF93DF9361E081E07B
:10B2B0000E94DD7AC091C906D0E0C11118C080910A
:10B2C000C806811104C00E94D97E8111B5C0809149
:10B2D0002302882361F081E09091C806911180E0FB
:10B2E00004E024E041EF5CE26D2F0E94494380912D
:10B2F000010E8770873009F058C0C130D9F48091B1
:10B30000C806813021F40E94D97E81119DC08091B0
:10B310002302882309F4C0C081E09091C8069130CF
:10B3200009F080E003E02EE34AEE5CE26D2F0E941C
:10B330004943B2C0C230D9F48091C806823021F4AA
:10B340000E94D97E81118AC080912302882309F44A
:10B35000A3C081E09091C806923009F080E003E03C
:10B360002EE343EE5CE26D2F0E94494395C0C3304B
:10B37000D1F58091C806833021F40E94D97E8111D5
:10B3800077C080912302882309F486C081E09091E0
:10B39000C806933009F080E003E02EE34CED5CE258
:10B3A0006D2F0E94494384E03EC0C130F1F480918A
:10B3B000C806813021F40E94D97E811163C080913A
:10B3C0002302882309F46AC081E09091C806913075
:10B3D00009F080E000E22EE34EEC5CE26D2F0E946B
:10B3E000494382E020C084E001C082E0C8131BC052
:10B3F0008091C8068C1304C00E94D97E811150C070
:10B4000080912302882371F081E09091C8069C13FB
:10B4100080E003E02EE344EC5CE26D2F0E944943A0
:10B420008C2F01C08C2FDF5FCF5FD53009F045CF67
:10B430008F5F8093C7063DC00E94077A8091950672
:10B44000882309F444CF35C08AEE9DE50E94A247C7
:10B4500080919506882309F45ACF2BC08FEE9DE585
:10B460000E94A24780919506882309F46DCF21C0E0
:10B4700084EF9DE50E94A24780919506882309F4F8
:10B4800080CF17C088ED9CE20E9459798091950683
:10B49000882309F494CF0DC084E0C5CF82E0C3CFE8
:10B4A00089EF9DE50E94A24780919506882309F4C3
:10B4B000A7CFDF91CF910F910895CF92DF92EF92B6
:10B4C000FF92CF93C82F0E94D62C6B017C0124EAF7
:10B4D00030E74DE75FE36091E0067091E10680910F
:10B4E000E2069091E3060F942C4E87FD05C04AEFCB
:10B4F00050E060E070E003C040E050E0BA01C40EEC
:10B50000D51EE61EF71EC092DC06D092DD06E09244
:10B51000DE06F092DF06C0932402CF91FF90EF90F9
:10B52000DF90CF9008952F923F924F925F926F924B
:10B530007F928F929F92AF92BF92CF92DF92EF92C3
:10B54000FF921F93CF93DF93CDB7DEB728970FB647
:10B55000F894DEBF0FBECDBF1C01162F0E94D97E0E
:10B56000882329F01092F7060E94077ADAC020910A
:10B57000EF063091F0063E832D83232B09F49DC006
:10B58000E4E01E9FC001112498878F83FC01E359DA
:10B59000FD4F80809180A280B38020E030E04AE7B8
:10B5A00054E4C501B4010F94524D2B013C0120E03D
:10B5B00030E04AE754E4C501B4010F94534D6B01E8
:10B5C0007C01809162028823B9F1113029F198F051
:10B5D000123091F540905A0250905B0260905C02EC
:10B5E00070905D02C0905E02D0905F02E0906002B9
:10B5F000F090610221C040904A0250904B0260904E
:10B600004C0270904D02C0904E02D0904F02E090DC
:10B610005002F090510210C04090520250905302DC
:10B620006090540270905502C0905602D09057021C
:10B63000E0905802F09059022D813E81B901330FFC
:10B64000880B990B0F94CE4E2091E0063091E106C5
:10B650004091E2065091E3060F946A509B01AC01C1
:10B66000C501B4010F94534DEF81F885E359FD4FA7
:10B670005F0160837183828393832D813E8137FFD5
:10B680000CC0A30192010F942C4E87FF11C0F5014D
:10B6900040825182628273820BC0A70196010F948F
:10B6A0002F5018162CF4F501C082D182E282F38269
:10B6B000812F03DF81E0809323021092F006109225
:10B6C000EF0680912302882361F124E0129FF001AC
:10B6D0001124E359FD4F80819181A281B381898337
:10B6E0009A83AB83BC832DEC3CEC4CEC5DE3609126
:10B6F000E0067091E1068091E2069091E3060F94D6
:10B700002F5087FD05C0CE0101960E94DC9E05C02A
:10B7100060E2CE0101960E94549FBC01C1010E94CB
:10B72000D44328960FB6F894DEBF0FBECDBFDF918D
:10B73000CF911F91FF90EF90DF90CF90BF90AF908F
:10B740009F908F907F906F905F904F903F902F9041
:10B75000089560E089E69DE2E6CE61E082E69DE242
:10B76000E2CE62E08BE59DE2DECECF93DF9300D0A8
:10B770001F92CDB7DEB70E94D97E882329F01092A0
:10B78000F7060E94077A57C06091EF067091F006A5
:10B790006115710569F1072E000C880B990B0F9448
:10B7A000CE4E2091E0063091E1064091E2065091A4
:10B7B000E3060F946A509B01AC016091790270918D
:10B7C0007A0280917B0290917C020F94534D60939A
:10B7D000790270937A0280937B0290937C0283E0DB
:10B7E0006CDE81E0809323021092F0061092EF0647
:10B7F000809123028823F9F02091A7053091A805B4
:10B800004091A9055091AA056091790270917A0240
:10B8100080917B0290917C020F94524D69837A83D0
:10B820008B839C83CE0101960E94DC9EBC018AEF33
:10B830009CE20E94D4430F900F900F900F90DF91E5
:10B84000CF91089521E02093F7066093E00670936E
:10B85000E1068093E2069093E30620E040E060E09A
:10B8600070E08091A5059091A6050C94D97960E0CF
:10B8700070E080E291E4E6CF60E070E080E89FE372
:10B88000E1CF6DEC7CEC8CEC9DE3DCCFFF920F9371
:10B890001F93CF93DF93F82E7093A6056093A505B1
:10B8A00061E081E00E94DD7AD091C906C0E091E0BC
:10B8B00081E0F81659F1F81628F082E0F81609F43C
:10B8C00049C06CC0D111D3C0992389F08091C806BA
:10B8D00018166CF02091EF063091F0062F5F3F4F65
:10B8E0003093F0062093EF068F5F8093C806809117
:10B8F0002302882309F42CC100E010E021E041E09C
:10B9000064E57DE28C2F0E94EA4222C1D111AFC0D2
:10B91000992389F08091C80618166CF02091EF06E3
:10B920003091F0062F5F3F4F3093F0062093EF06E3
:10B930008F5F8093C80680912302882309F408C191
:10B9400000E010E021E041E06DE47DE28C2F0E94F8
:10B95000EA42FEC0D1118BC0992389F08091C806BC
:10B9600018166CF02091EF063091F0062F5F3F4FD4
:10B970003093F0062093EF068F5F8093C806809186
:10B980002302882309F4E4C000E010E021E041E054
:10B9900066E47DE28C2F0E94EA42DAC0409179028F
:10B9A00050917A0260917B0270917C024093A705CE
:10B9B0005093A8056093A9057093AA05D11122C0E0
:10B9C000992389F08091C80618166CF02091EF0633
:10B9D0003091F0062F5F3F4F3093F0062093EF0633
:10B9E0008F5F8093C80680912302882309F4E8C002
:10B9F00000E010E021E041E06CE37DE28C2F0E944A
:10BA0000EA42DEC083E0F81232C060912E0D7091E0
:10BA10002F0D8091300D9091310D2091F60C211158
:10BA200026C00F949B4E2091360230913702621748
:10BA30007307ECF4D130C9F48091C806813021F449
:10BA40000E94D97E81118EC080912302882369F0E3
:10BA500081E09091C806913009F080E004E024E094
:10BA60004CE25DE26C2F0E94494382E072C0D1300B
:10BA7000D9F48091C806813021F40E94D97E8111C9
:10BA800079C080912302882309F462C081E09091FB
:10BA9000C806913009F080E004E024E042E25DE273
:10BAA0006C2F0E94494354C0D230D9F48091C8060B
:10BAB000823021F40E94D97E811164C080912302DA
:10BAC000882309F445C081E09091C806923009F0BE
:10BAD00080E003E02EE348E15DE26C2F0E944943E1
:10BAE00037C0D330D1F48091C806833021F40E944E
:10BAF000D97E811151C080912302882349F181E0D0
:10BB00009091C806933009F080E003E02EE34FE007
:10BB10005DE26C2F0E9449431BC0D430C9F4809170
:10BB2000C806843021F40E94D97E81113FC08091E3
:10BB30002302882369F081E09091C806943009F0CF
:10BB400080E003E02EE344E05DE26C2F0E94494375
:10BB500085E0CF5FDF5F90E0C53009F0A9CE80932C
:10BB6000C70632C00E94077A80919506882309F49F
:10BB70006BCF2AC00E94077A80919506882309F42A
:10BB800080CF22C087E39CE50E94A2478091950662
:10BB9000882309F493CF18C08CE39CE50E94A24748
:10BBA00080919506882309F4A6CF0EC081E49CE518
:10BBB0000E94A24780919506882309F4B8CF04C05B
:10BBC00083E0F812C5CF21CFDF91CF911F910F9164
:10BBD000FF9008954FEF69EA7BE580E057CE4FEF85
:10BBE0006DEA7BE581E052CE4FEF61EB7BE582E0D1
:10BBF0004DCE4FEF65EB7BE583E048CE0F93CF93BF
:10BC0000DF9361E081E00E94DD7AD091C906C0E057
:10BC1000D1111AC08091C806811104C00E94D97E3A
:10BC20008111A9C080912302882309F49BC081E07F
:10BC30009091C806911180E004E024E04FEB5CE2B3
:10BC40006C2F0E9449438EC0D130D9F48091C80630
:10BC5000813021F40E94D97E811195C08091230208
:10BC6000882309F47FC081E09091C806913009F0E3
:10BC700080E003E02EE345EB5CE26C2F0E94494339
:10BC800071C0D230D9F48091C806823021F40E946C
:10BC9000D97E811182C080912302882309F462C079
:10BCA00081E09091C806923009F080E000E22EE336
:10BCB00047EA5CE26C2F0E94494354C0D330D9F468
:10BCC0008091C806833021F40E94D97E81116FC013
:10BCD00080912302882309F445C081E09091C80631
:10BCE000933009F080E000E22EE34BE55CE26C2F3C
:10BCF0000E94494337C0D430D1F48091C8068430C3
:10BD000021F40E94D97E81115CC080912302882396
:10BD100049F181E09091C806943009F080E000E29A
:10BD20002EE348E95BE26C2F0E9449431BC0D530EB
:10BD3000C9F48091C806853021F40E94D97E811112
:10BD40004AC080912302882369F081E09091C8065F
:10BD5000953009F080E000E22EE343E85BE26C2FCF
:10BD60000E944943CF5FDF5FC53009F051CF86E0C5
:10BD70008093C70639C00E94077A80919506882370
:10BD800009F450CF31C083E599E50E94A247809124
:10BD90009506882309F462CF27C081EB9CE20E94BC
:10BDA000597980919506882309F475CF1DC088E6DE
:10BDB0009CE20E94597980919506882309F488CFE6
:10BDC00013C087EA9BE20E945979809195068823E7
:10BDD00009F49BCF09C084E99BE20E9459798091C4
:10BDE0009506882309F4ADCFDF91CF910F91089587
:10BDF000CF93DF93EC01CB01BA010F94CE4E0F9499
:10BE00009B4E79836883DF91CF91089568EF7EE53B
:10BE10008FE89FE50C941C7A0F931F93CF93DF93C9
:10BE200061E081E00E94DD7AC091C906D0E081E046
:10BE3000C11122C0882389F08091C80618166CF0C1
:10BE40002091EF063091F0062F5F3F4F3093F006C0
:10BE50002093EF068F5F8093C8068091230288238A
:10BE600009F441C000E010E020E041E063ED7EE233
:10BE70008D2F0E94EA4237C0C130D1F48091C806AC
:10BE8000813021F40E94D97E811137C08091230234
:10BE9000882349F181E09091C806913009F080E053
:10BEA00000E22EE348EC5EE26D2F0E9449431BC086
:10BEB000C230C9F48091C806823021F40E94D97E34
:10BEC000811122C080912302882369F081E0909142
:10BED000C806923009F080E000E22EE344EB5EE217
:10BEE0006D2F0E944943DF5FCF5F80E0D53009F0BE
:10BEF0009FCF83E08093C7060DC0C093840C8091D0
:10BF00009506882319F206C0C093840C809195068B
:10BF10008823C1F2DF91CF911F910F9108950F9463
:10BF2000CE4E0F949B4ECB010C94169DEF92FF9238
:10BF30000F931F93CF93DF93CDB7DEB72B970FB639
:10BF4000F894DEBF0FBECDBF7C014091AC05842FBD
:10BF5000042E000C990B2091AD05223051F02330B6
:10BF600019F022E03FE20AC047FF06C02EE03FE2A0
:10BF700005C020E23FE202C027E13FE29F934F93DA
:10BF80003F932F938E010F5F1F4F1F930F930F94BB
:10BF9000CE5640913402509135024F5051099701CD
:10BFA0000F900F900F900F900F900F904E155F0510
:10BFB0000CF49A013093330D2093320D80E00E94EF
:10BFC0009CB6C8010E94C77B2B960FB6F894DEBFC3
:10BFD0000FBECDBFDF91CF911F910F91FF90EF90DA
:10BFE0000895E091AC0587E1E802F0011124E65DD7
:10BFF000F24F808591859ACF7F928F929F92AF92D8
:10C00000BF92CF92DF92EF92FF920F931F93CF9345
:10C01000DF93782E8093AD056093AC0561E081E0FD
:10C020000E94DD7AD091C906C0E081E0D1112EC016
:10C03000882389F08091C80618166CF02091EF06CD
:10C040003091F0062F5F3F4F3093F0062093EF06BC
:10C050008F5F8093C80680912302882309F494C0DF
:10C0600022E0721649F033E0731203C064EE7EE200
:10C0700005C064ED7EE202C064EF7EE200E010E005
:10C0800021E041E08C2F0E94EA427EC0D130D9F4F9
:10C090008091C806813021F40E94D97E81117DC033
:10C0A00080912302882309F46FC081E09091C80633
:10C0B000913009F080E004E024E04FE55FE26C2F6E
:10C0C0000E94494361C0D230D9F48091C8068230C1
:10C0D00021F40E94D97E811168C0809123028823B7
:10C0E00009F452C081E09091C806923009F080E0D6
:10C0F00000E22EE343E55FE26C2F0E94494344C017
:10C10000D330D1F48091C806833021F40E94D97EC7
:10C11000811156C0809123028823B1F181E0909172
:10C12000C806933009F080E000E22EE347E45FE2C6
:10C130006C2F0E94494328C0D43031F58091C80645
:10C14000843021F40E94D97E811145C08091230260
:10C150008823D1F011E08091C806843009F010E006
:10C160002091AC0537E12303F0011124E65DF24F85
:10C17000808591850E94169D00E09C0149E25FE266
:10C180006C2F812F0E947843CF5FDF5F80E0C53046
:10C1900009F04CCFC093C7065BC00E94077A80911C
:10C1A0009506882309F47CCF53C08091B405909103
:10C1B000B505BCDE80919506882309F48ECF48C072
:10C1C0008091B6059091B705B1DE809195068823E0
:10C1D00009F4A0CF3DC081E00E94CE7E0091AC0565
:10C1E00027E1020380011124F801E65DF24F60852A
:10C1F0007185072E000C880B990B0F94CE4E20E012
:10C2000030E040EF52E40F94524D0F94A04EF801ED
:10C21000EE5CF24F1F9281EF882E8FE5982E96E00C
:10C22000A92E9FE5B92E6B011AEAE12EF12C00E050
:10C2300010E028E730E040E050E0BF0188E39FE2F3
:10C240000E945B790F9080919506882309F47ECF38
:10C25000DF91CF911F910F91FF90EF90DF90CF90E2
:10C26000BF90AF909F908F907F90089560E081E0A5
:10C27000C3CE8F929F92AF92BF92CF92DF92EF92F6
:10C28000FF920F931F93CF93DF934C015B016A01E1
:10C2900060E085E00E94DD7AD091C906F12C82E051
:10C2A000E82ED1111AC080912302882321F18091B8
:10C2B0002602823041F0833019F469E87EE205C03D
:10C2C00067E77EE202C069E97EE200E010E021E07B
:10C2D00041E08F2D0E94EA420EC0D13061F480917E
:10C2E0002302882341F000E010E020E041E0B401A7
:10C2F0008F2D0E94EA42A114B10481F0D23081F462
:10C3000080912302882309F46EC000E010E020E051
:10C3100041E0B5018F2D0E94EA4265C0C2E001C034
:10C32000C3E0C114D10491F0DC130FC0809123024B
:10C33000882351F000E010E020E041E0B6018F2DAD
:10C340000E94EA42CD2F01C0CD2FCF5F21E030E027
:10C35000A114B10411F420E030E081E090E0C114B8
:10C36000D10411F480E090E0820F931F029781F0D6
:10C37000DC130DC080912302882349F000E010E017
:10C3800020E041E062EB7EE28F2D0E94EA42CF5F27
:10C39000DC1314C080912302882371F000E010E0C8
:10C3A00021E040E067EA7EE28F2D0E94EA42609140
:10C3B000AB058F2D0E948B42E0922302F394DF5F46
:10C3C00085E0F8126ECFCF5FC093C706DF91CF91A3
:10C3D0001F910F91FF90EF90DF90CF90BF90AF90A3
:10C3E0009F908F900895C3E0C114D10409F0ADCFA0
:10C3F000ADCF40E050E060E070E08CE69EE239CFE7
:10C4000043E65EE263E57EE28AE49EE232CF40E00C
:10C4100050E06AE37EE281E39EE22BCF40E050E011
:10C4200062E27EE283E19EE224CF40E050E064E0FD
:10C430007EE287EF9DE21DCF4BEE5DE26AED7DE28D
:10C440008AEC9DE216CF40E050E06CEB7DE283EB9E
:10C450009DE20FCF40E050E063EA7DE286E99DE295
:10C4600008CF40E050E069E87DE288E89DE201CF36
:10C4700040E050E069E77DE280E79DE2FACE61119D
:10C48000609326024093AB05082E000C990BAA0B73
:10C49000BB0B8C309105A0F5FC018827EA56FF4FB5
:10C4A0008F4F0D94B45180E092E61FC087E092E672
:10C4B0001CC08AE292E619C08CE192E616C083E2C3
:10C4C00092E613C088E392E610C081E392E60DC0C5
:10C4D00085E192E60AC08EE092E607C01092840CD5
:10C4E0008CE09FE502C089EF91E6009749F021E0DA
:10C4F0002093F70620E040E060E070E00C94D979EA
:10C500000C94007A10925E18109288028091A6090D
:10C5100080628093A6090E9441B16FEF85E390E3AA
:10C520000E9439810C94007ACF92DF92EF92FF92B1
:10C530000F931F9383E3C82E80E3D82EE12CF12CB8
:10C5400008E210E327E03AE742E852E663E270E3EC
:10C550008EE190E30E94D57B1F910F91FF90EF90A9
:10C56000DF90CF9008959091A60993FB882780F9DA
:10C5700093FF06C081E09091D607911101C080E041
:10C580000895F1DF882339F08091A60982FB88277E
:10C5900080F991E08927089581E590E30E94D47A9B
:10C5A00040E061E080E06BDF87E490E30D94613D63
:10C5B000E8DF882321F083E490E30F94613D0C943D
:10C5C00039B1EF92FF920F931F93CF93DF9361E006
:10C5D00081E00E94DD7AC091C90610E0C11118C047
:10C5E0008091C806811104C00E94D97E8111AAC120
:10C5F00080912302882361F081E09091C806911117
:10C6000080E004E024E042E150E3612F0E944943CE
:10C610008091A60982FBDD27D0F982FD06C0D1E01A
:10C6200090915318913009F0D0E083FBEE24E0F8AC
:10C6300083FF03C098DFF82E01C0F12CDD2309F43D
:10C6400058C0C130D9F48091C806813021F40E94CD
:10C65000D97E81117FC180912302882309F48BC187
:10C6600081E09091C806913009F080E000E22EE36D
:10C6700046E050E3612F0E9449437DC1C230D9F4A6
:10C680008091C806823021F40E94D97E811169C14F
:10C6900080912302882309F46EC181E09091C8063D
:10C6A000923009F080E003E02EE34BEF5FE2612F70
:10C6B0000E94494360C1C33009F047C08091C80659
:10C6C000833021F40E94D97E811157C180912302C9
:10C6D000882309F450C181E09091C806933009F095
:10C6E00080E003E02EE346EF5FE2612F0E944943C2
:10C6F00042C180915318823029F043DF811102C07A
:10C70000D1E004C0C13009F442C1D2E0CD131BC056
:10C710008091C8068C1304C00E94D97E811159C132
:10C7200080912302882371F081E09091C8069C13C8
:10C7300080E003E02EE340EE5FE2612F0E94494378
:10C74000DC2F01C0DC2FDF5F01C0D4E0CD131BC0A4
:10C750008091C8068C1304C00E94D97E811143C108
:10C7600080912302882371F081E09091C8069C1388
:10C7700080E003E02EE344ED5FE2612F0E94494335
:10C78000DC2F01C0DC2F81E08D0FC81318C0809111
:10C79000C8068C1304C00E94D97E81112EC18091DD
:10C7A0002302882361F081E09091C8069C1380E009
:10C7B00003E02EE346EC5FE2612F0E94494382E0F2
:10C7C0008D0F4091320D5091330D9091F60C9111D7
:10C7D00007C0209136023091370242175307DCF030
:10C7E000C81333C08091C8068C1304C00E94D97E40
:10C7F00081110DC180912302882339F181E090914C
:10C80000C8069C1380E000E22EE34EEA5FE2612F4F
:10C810000E9449431AC0C81318C08091C8068C13DF
:10C8200004C00E94D97E8111FCC08091230288231C
:10C8300061F081E09091C8069C1380E003E02EE354
:10C840004EE95FE2612F0E944943DD5FCD1318C0BE
:10C850008091C8068C1304C00E94D97E8111EBC060
:10C8600080912302882361F081E09091C8069C1397
:10C8700080E003E02EE340E95FE2612F0E9449433C
:10C8800091E09D0FEE2009F43BC0F11053C0C91395
:10C8900018C08091C8068C1304C00E94D97E8111F3
:10C8A000D4C080912302882361F081E09091C80672
:10C8B0009C1380E000E22EE34DE75FE2612F0E94CF
:10C8C000494382E08D0FC81318C08091C8068C13AD
:10C8D00004C00E94D97E8111C2C0809123028823A6
:10C8E00061F081E09091C8069C1380E003E02EE3A4
:10C8F0004FE65FE2612F0E94494393E09D0F1AC00B
:10C90000C91316C08091C8068C1302C00E94D97E3C
:10C9100080912302882361F081E09091C8069C13E6
:10C9200080E000E22EE344E65FE2612F0E9449438B
:10C9300092E09D0F1F5FCF5F153009F04FCE9093AF
:10C94000C70696C00E94077A80919506882309F44D
:10C950004FCE8EC021DE80919506882309F47BCED0
:10C9600087C084E992E60E94A247809195068823B9
:10C9700009F48ECE7DC0D4E006CF86E996E60E940B
:10C98000A24780919506882309F4A0CE71C08091BA
:10C99000C806813021F40E94D97E811112C0809195
:10C9A00023028823A1F081E09091C806913009F01C
:10C9B00080E000E22EE349EE5FE2612F0E944943EE
:10C9C00006C0F6DD80919506882349F351C0D2E078
:10C9D000BACE8EEF9DE50E94A247809195068823EE
:10C9E00009F49ECE45C08CE29BE60E94A24780914E
:10C9F0009506882309F4B4CE3BC088E498E70E94EA
:10CA0000A24780919506882309F4C9CE31C08EEBE8
:10CA10009FE20E94597980919506882309F4EACE15
:10CA200027C086E391E60E94A2478091950688235D
:10CA300009F4FBCE1DC08CE79AE60E94A2478091C4
:10CA40009506882309F40CCF13C08CE89FE20E945E
:10CA5000597980919506882309F423CF09C08AE982
:10CA600098E40E94A24780919506882309F435CF67
:10CA7000DF91CF911F910F91FF90EF9008956091FA
:10CA8000260D70E080E00C94BBB160918102709142
:10CA90008202072E000C880B990B0F94CE4E2AE0D1
:10CAA00037ED43E25CE30F946A5060937D0270932C
:10CAB0007E0280937F02909380020895CF93DF934C
:10CAC000EC01CB01BA010F94CE4E0F94A04E6883B7
:10CAD000DF91CF91089580E00C949CB66EE575E6E9
:10CAE00084E795E60C941C7A0F94CE4E0F94A04EDA
:10CAF000862F0C94F09CEF92FF920F931F93CF938D
:10CB0000DF9300D01F92CDB7DEB7082F7B010E94C4
:10CB1000D97E882329F01092F7060E94077A3BC03D
:10CB20006091EF067091F0066115710551F0109259
:10CB3000F0061092EF0681E080932302802F0E947E
:10CB40007CAA80912302882331F184E0089F800130
:10CB500011240057114F60916E0C70916F0C072ECD
:10CB6000000C880B990B0F94CE4E9B01AC01F80181
:10CB700060817181828193810F946A5069837A8385
:10CB80008B839C8360E2CE0101960E94EC9FBC01E6
:10CB9000C7010E94D4430F900F900F900F90DF9128
:10CBA000CF911F910F91FF90EF90089566ED70E384
:10CBB00080E0A1CF6BEC70E381E09DCF20E040E00E
:10CBC00060E070E00E94D97981E08093F7061092CE
:10CBD0006F0C10926E0C089586ED95E6EFCF8AEDFE
:10CBE00095E6ECCF2F923F924F925F926F927F9299
:10CBF0008F929F92AF92BF92CF92DF92EF92FF926D
:10CC00000F931F93CF93DF93CDB7DEB729970FB65E
:10CC1000F894DEBF0FBECDBF1C017987688769011C
:10CC20001A830983EB82BA01550F880B990B0F9475
:10CC3000CE4E4B015C0120E030E040E057EC0F9419
:10CC40002F5018162CF0812C912CA12C27ECB22EF1
:10CC5000C501B4010F949B4E2B013C01B601DD0CC4
:10CC6000880B990B0F94CE4E4B015C0120E03EEFF8
:10CC70004FEF56E40F942C4E87FD07C0812C9EEF9A
:10CC8000992EAA24AA9496E4B92EE885F9856081A4
:10CC90007181072E000C880B990B0F94CE4E6B01FF
:10CCA0007C01C301B2010F94CE4E9B01AC01C701C0
:10CCB000B6010F94524D0F94A04E6C837D838E83EA
:10CCC0009F83C501B4010F949B4E7B018C01E41836
:10CCD000F50806091709FB81FF9389809A8086E091
:10CCE000A82E8FE5B82ECC80DD80A3019201688547
:10CCF0007985C1010E945B790F9029960FB6F8944F
:10CD0000DEBF0FBECDBFDF91CF911F910F91FF907E
:10CD1000EF90DF90CF90BF90AF909F908F907F90DB
:10CD20006F905F904F903F902F9008958F929F92B9
:10CD3000AF92BF92CF92DF92EF92FF920F931F9329
:10CD4000CF93DF9361E081E00E94DD7AD091C90644
:10CD5000C0E0D1111AC08091C806811104C00E94A0
:10CD6000D97E811121C180912302882309F413C146
:10CD700081E09091C806911180E004E024E046EC47
:10CD800050E36C2F0E94494306C1D13011F58091C8
:10CD9000C806813021F40E94D97E81110DC1809195
:10CDA0002302882309F4F7C011E08091C80681307E
:10CDB00009F010E080916702909168020E94169D30
:10CDC00000E09C014AEB50E36C2F812F0E947843D6
:10CDD000E2C0D23011F58091C806823021F40E9461
:10CDE000D97E8111FBC080912302882309F4D3C02E
:10CDF00011E08091C806823009F010E08091320D78
:10CE00009091330D0E94169D00E09C014CEA50E386
:10CE10006C2F812F0E947843BEC0D33011F58091D2
:10CE2000C806833021F40E94D97E8111ECC0809124
:10CE30002302882309F4AFC011E08091C806833033
:10CE400009F010E080910C0D90910D0D0E94169D3F
:10CE500000E09C0144EA50E36C2F812F0E9478434C
:10CE60009AC0D43001F58091C806843021F40E9424
:10CE7000D97E8111DDC080912302882309F48BC003
:10CE800011E08091C806843009F010E08091260DF1
:10CE90000E94F09C00E09C014CE850E36C2F812F35
:10CEA0000E94784378C0D53011F58091C80685304E
:10CEB00021F40E94D97E8111DEC080912302882353
:10CEC00009F469C011E08091C806853009F010E0CE
:10CED00080918102909182020E94169D00E09C0147
:10CEE00042E850E36C2F812F0E94784354C0D63023
:10CEF000D9F48091C806863021F40E94D97E811130
:10CF0000CCC080912302882309F445C081E0909130
:10CF1000C806963009F080E003E02EE347E750E3CF
:10CF20006C2F0E94494337C0D730D1F48091C80696
:10CF3000873021F40E94D97E8111B9C080912302EB
:10CF4000882349F181E09091C806973009F080E08C
:10CF500003E02EE34CE650E36C2F0E9449431BC0D4
:10CF6000D830C9F48091C806883021F40E94D97E57
:10CF70008111A7C080912302882369F081E09091FC
:10CF8000C806983009F080E003E02EE34DE550E359
:10CF90006C2F0E944943CF5FDF5FC53009F0D9CEC7
:10CFA00089E08093C70696C00E94077A8091950613
:10CFB000882309F4D8CE8EC0E12C00E010E027EEE3
:10CFC00033E04AE050E067E672E080EC90E30ADE8E
:10CFD00080919506882309F4E2CE7CC081E00E940E
:10CFE000CE7EE12C0BE615E622E231E040E050E097
:10CFF00062E37DE083EB90E3F5DD80919506882385
:10D0000009F4F1CE67C081E00E94CE7EE12C09EEEA
:10D0100016EB2CE830E040E050E06CE07DE088EA80
:10D0200090E3E0DD80919506882309F400CF52C09B
:10D0300081E00E94CE7EC090260DD12C1F928FE3FE
:10D04000882E85E6982E9EE6A92E95E6B92EE12C2F
:10D05000F12C8701EA9420E030E0A90166E27DE04E
:10D0600088E990E30E945B790F9080919506882370
:10D0700009F401CF2FC0E12C05E415E627EE33E0DB
:10D080004AE050E061E872E087E890E3ABDD809130
:10D090009506882309F411CF1DC08CEE95E60E94F9
:10D0A000A24780919506882309F42BCF13C08FEEF9
:10D0B00095E60E94A24780919506882309F43ECF09
:10D0C00009C083E49BE70E94A247809195068823CC
:10D0D00009F450CFDF91CF911F910F91FF90EF9006
:10D0E000DF90CF90BF90AF909F908F9008950E9457
:10D0F000D97E882321F01092F7060E94077A0C94BB
:10D1000022420E94D97E882341F020E040E060E086
:10D1100070E087E798E60E94D97961E080E00C949E
:10D12000B8414F925F926F927F92AF92BF92CF922F
:10D13000DF92EF92FF92CF93DF93EB01FC016081CE
:10D140007181828193812CE3C22ED12CE12CF12CB0
:10D15000A70196010F947651B62EA72ECA01B901E8
:10D16000A70196010F9476516B017C01CA01B901A8
:10D1700028E130E040E050E00F9476512B013C0173
:10D18000C9016DE671E00F944F5161157105D9F039
:10D19000AF92BF92DF92CF925F924F929F938F9305
:10D1A0007F936F9383E391E39F938F93DF93CF9369
:10D1B0000F94CE568DB79EB70E960FB6F8949EBFBD
:10D1C0000FBE8DBF61C00097C9F0AF92BF92DF92D2
:10D1D000CF925F924F929F938F9383E291E39F93BD
:10D1E0008F93DF93CF930F94CE56EDB7FEB73C9657
:10D1F0000FB6F894FEBF0FBEEDBF46C041145104F8
:10D2000061047104B9F0AF92BF92DF92CF925F9246
:10D210004F9287E191E39F938F93DF93CF930F9486
:10D22000CE568DB79EB70A960FB6F8949EBF0FBE26
:10D230008DBF2AC0C114D104E104F104A9F0AF925A
:10D24000BF92DF92CF928FE091E39F938F93DF9312
:10D25000CF930F94CE56EDB7FEB738960FB6F8942D
:10D26000FEBF0FBEEDBF10C0AF92BF928BE091E347
:10D270009F938F93DF93CF930F94CE560F900F9081
:10D280000F900F900F900F90DF91CF91FF90EF9044
:10D29000DF90CF90BF90AF907F906F905F904F9056
:10D2A00008952F923F924F925F926F927F928F924A
:10D2B0009F92AF92BF92CF92DF92EF92FF920F9325
:10D2C0001F93CF93DF93CDB7DEB76F970FB6F89468
:10D2D000DEBF0FBECDBF0E94D97E882319F00E9409
:10D2E000077AF1C02090550D3090560D8091570D62
:10D2F0009091580D9F8F8E8F8091590D90915A0D5E
:10D30000A0915B0DB0915C0D8A8F9B8FAC8FBD8F10
:10D3100040905D0D50905E0D60905F0D7090600DBF
:10D320008090610D9090620DA090630DB090640D9F
:10D3300060E085E00E94DD7AE090C906F12CDE0114
:10D3400011966D01E1100DC0809123028823E1F058
:10D35000C1010E944C9D8C0120E040E068E971E32E
:10D3600010C0B1E0EB1210C080912302882361F05D
:10D370008E8D9F8D0E944C9D8C0120E040E06CE8DA
:10D3800071E38F2D0E94EA428A8D9B8DAC8DBD8DFD
:10D390008E8B9F8BA88FB98FB601CE014696C1DECA
:10D3A00092E0E9120BC0809123028823B1F000E0E3
:10D3B00010E020E040E06AE771E30CC0A3E0EA126D
:10D3C0000CC080912302882341F0860120E040E0D8
:10D3D00067E771E38F2D0E94EA424E8A5F8A688E6A
:10D3E000798EB601CE0146969CDEB4E0EB120BC0FE
:10D3F000809123028823B1F000E010E020E040E0BB
:10D4000065E671E30CC085E0E8120CC08091230250
:10D41000882341F0860120E040E062E671E38F2D31
:10D420000E94EA4220E030E048EC52E4C501B40139
:10D430000F94334E0F949B4ECB016AE070E00F9433
:10D4400063519F938F9320E030E04AE754E4C50195
:10D45000B4010F94334E0F949B4E9F938F937F9301
:10D460006F93AAE5B1E3BF93AF93DF92CF920F948E
:10D47000CE560FB6F894DEBF0FBECDBFB6E0EB12AE
:10D480000BC0809123028823B1F000E010E020E07F
:10D4900040E06AE471E30CC087E0E8120CC08091C0
:10D4A0002302882341F0860120E040E067E471E335
:10D4B0008F2D0E94EA42F394E39495E0F91242CF53
:10D4C00088E08093C7066F960FB6F894DEBF0FBE54
:10D4D000CDBFDF91CF911F910F91FF90EF90DF9023
:10D4E000CF90BF90AF909F908F907F906F905F9004
:10D4F0004F903F902F9008950F93CF93DF9361E06B
:10D5000081E00E94DD7AD091C906C0E0D11117C038
:10D510008091C806811104C00E94D97E811166C025
:10D5200080912302882309F458C081E09091C806B5
:10D53000911180E004E024E046E051E34BC0D1309B
:10D54000C1F48091C806813021F40E94D97E8111F6
:10D5500055C080912302882309F43FC081E0909157
:10D56000C806913009F080E003E02EE345EF50E378
:10D5700031C0D230B9F48091C806823021F40E94C3
:10D58000D97E811145C080912302882331F181E049
:10D590009091C806923009F080E003E02EE347EE58
:10D5A00050E318C0D530C9F48091C806853021F405
:10D5B0000E94D97E811136C080912302882369F0B0
:10D5C00081E09091C806953009F080E003E02EE3F9
:10D5D00041EE50E36C2F0E944943CF5FDF5FC530BF
:10D5E00009F094CF86E08093C70624C00E94077A92
:10D5F00080919506882309F493CF1CC081E898E6B2
:10D600000E94A24780919506882309F4A2CF12C0F8
:10D6100081E599E60E94A24780919506882309F446
:10D62000B2CF08C088EB97E40E94A247809195068C
:10D63000882311F2DF91CF910F91089560E070E09F
:10D6400080E00E94BBB160E070E081E00E94BBB16D
:10D650000E9436B70C94007A8F929F92AF92BF923D
:10D66000CF92DF92EF92FF920F931F93CF93DF93AE
:10D6700061E081E00E94DD7AD091C906C0E0D1115D
:10D680001AC08091C806811104C00E94D97E811100
:10D69000ABC080912302882309F474C081E090918B
:10D6A000C806911180E004E024E04DED51E36C2FB9
:10D6B0000E94494367C0D13011F58091C80681307E
:10D6C00021F40E94D97E811197C080912302882382
:10D6D00009F458C011E08091C806813009F010E0CB
:10D6E0008091320D9091330D0E94169D00E09C01B7
:10D6F0004FEC51E36C2F812F0E94784343C0D2300E
:10D7000009F58091C806823021F40E94D97E8111EA
:10D7100099C0809123028823A9F111E08091C80665
:10D72000823009F010E080910C0D90910D0D0E9457
:10D73000169D00E09C0147EC51E36C2F812F0E9465
:10D74000784320C0D330F1F48091C806833021F4AF
:10D750000E94D97E81119BC080912302882391F081
:10D7600011E08091C806833009F010E08091260D09
:10D770000E94C19C00E09C014FEA51E36C2F812F75
:10D780000E9478438091320D9091330D20910C0DC1
:10D7900030910D0D232B11F4892BE9F0D430C9F40D
:10D7A0008091C806843021F40E94D97E811192C0F4
:10D7B00080912302882369F081E09091C80694301B
:10D7C00009F080E000E22EE346EA51E36C2F0E946C
:10D7D000494385E001C084E0CF5FDF5FC53009F0D9
:10D7E0004ECF8093C7067CC00E94077A8091950631
:10D7F000882309F44ECF74C081E00E94CE7EC09091
:10D80000320DD090330D1F926BE6862E65E6962E74
:10D8100076E0A72E7FE5B72E12E2E12EFF24F394E7
:10D8200000E010E020E030E0A90162E37DE086ED59
:10D8300091E30E945B790F9080919506882309F40B
:10D8400044CF4EC081E00E94CE7EC0900C0DD0909F
:10D850000D0D1F9239EE832E36EB932E46E0A42E4B
:10D860004FE5B42E1CE8E12EF12C00E010E020E0A2
:10D8700030E0A9016CE07DE08BEC91E30E945B79E4
:10D880000F9080919506882309F443CF29C081E049
:10D890000E94CE7EC090260DD12C1F928FE3882E41
:10D8A00085E6982E95EAA92E99E4B92EE12CF12C63
:10D8B0008701EA9420E030E0A90166E27DE08BEB8D
:10D8C00091E30E945B790F9080919506882309F47B
:10D8D00043CF06C0B3DE80919506882309F468CF54
:10D8E000DF91CF911F910F91FF90EF90DF90CF903C
:10D8F000BF90AF909F908F90089580E095E29093B5
:10D90000BD058093BC058CE491E09093B9058093AC
:10D91000B80580EC9EEF9093BB058093BA0590917B
:10D92000C10580E2890F863740F080EF890F20E43F
:10D9300031E03093BB052093BA051092BE05809369
:10D94000BF058FEF8093C00508958F929F92BF927D
:10D95000CF92DF92EF92FF920F931F93CF93DF93BB
:10D960001F92CDB7DEB7E1D7882309F4D6C18091E5
:10D97000EF06863214F085E202C087FD80E0282F92
:10D98000082E000C330B3093F0062093EF06982FEF
:10D99000990F890F8093C10580911106882309F49E
:10D9A000BCC12091BA053091BB050091BE05109114
:10D9B000BF05020F131FE090BC05F090BD058091DC
:10D9C000B8059091B905E80EF91E01304FE714072C
:10D9D00068F03195219531093093BB052093BA0544
:10D9E0006CED70E085E090E00F947448F7FE15C090
:10D9F0008091B8059091B905919581959109909381
:10DA0000B9058093B80568E171E085E090E00F9476
:10DA1000744881E08093C00517C081E0E81680E477
:10DA2000F80694F06BE470E084EF91E00F94744892
:10DA30008091CB0581508093CB05882311F05DDF69
:10DA40006CC11092110669C12091B8053091B905D9
:10DA5000C7019A508130934108F098C08F2D9927C3
:10DA600087FD9A950A9765E070E00F946351812FC6
:10DA700017FF02C087E0810F482F459545954595D2
:10DA800081E090E0A0E0B0E004C0880F991FAA1FD9
:10DA9000BB1F4A95D2F7FB01EE0FFF1FEE53FA4F63
:10DAA000408151818A0108231923012B09F419C1EE
:10DAB00080959095842395239183808384E090E0E2
:10DAC000861B970B4091120650911306840F951FE9
:10DAD00090931306809312068091CA05815080931B
:10DAE000CA05811103C082E080931106932F90959F
:10DAF000991F9927991F8091C005881F8827881F23
:10DB00009817F1F03195219531093093B90520939B
:10DB1000B80520E130E040E050E060EF7FEF8FEFAC
:10DB20009FEF0E9463372091BA053091BB05620FC9
:10DB3000731F7093BB056093BA0560E773E021C063
:10DB40008091BA059091BB0591958195910990932B
:10DB5000BB058093BA0520E130E040E050E060EF83
:10DB60007FEF8FEF9FEF0E9463372091B8053091D0
:10DB7000B905620F731F7093B9056093B80560E82B
:10DB800072E085E090E00F947448ABC01216130663
:10DB90000CF0A7C0FDE3FF1A41E0E41642E0F406F2
:10DBA00008F09FC08091C105181B103108F099C082
:10DBB0003195219531093093B9052093B80560E777
:10DBC00073E083E090E00F9474488FEF8093C0057A
:10DBD00021E012300CF020E08EEF810F8C30A0F0AD
:10DBE0008091BA059091BB0541E050E018161906E6
:10DBF00014F040E050E030E04217530709F055C000
:10DC000091958195910927C0143050F520E030E0BE
:10DC1000A90160EC7FEF8FEF9FEF0E9463372091A7
:10DC2000BA053091BB05620F731F7093BB056093FB
:10DC3000BA0561157E4F34F480E09EEF9093BB05EA
:10DC40008093BA058091BA059091BB0581309240CE
:10DC500064F180E092E09093BB058093BA0525C003
:10DC60001C301CF120E430E040E050E060E070E067
:10DC7000CB010E9463372091BA053091BB05620F3A
:10DC8000731F7093BB056093BA0561157E4F34F422
:10DC900080E09EEF9093BB058093BA058091BA0512
:10DCA0009091BB0581309240A4F68091110682309C
:10DCB000C1F480E48093CA058FEF9FEF9093C30572
:10DCC0008093C2059093C5058093C4059093C705C2
:10DCD0008093C6059093C9058093C80581E0809321
:10DCE00011062091BE053091BF058091BA05909133
:10DCF000BB05820F931F9093BF058093BE052091B3
:10DD0000BC053091BD058091B8059091B905820F91
:10DD1000931F9093BD058093BC0561E08BE694E072
:10DD20000E94FA3180919F048E3130F080919F04DF
:10DD30008E3308F456C05AC08091A1048A30B0F3E3
:10DD400082ECE82E85E0F82E9AE0892E912CB82CF2
:10DD500080919F0490E094012C5F3F4F2817390772
:10DD60005CF442E0E40EF11C85E0880E911CEEE1CB
:10DD70008E16910461F7DACF8091A104881588F39B
:10DD800030E0C12CD12CF70180819181A0E0B0E07E
:10DD90000C2C04C0B695A795979587950A94D2F751
:10DDA00080FD07C0FFEFCF1ADF0A385F303859F720
:10DDB000D8CF00E010E0A801480D591D80919F04C4
:10DDC00090E0481759073CF08091A10490E0841737
:10DDD00095070CF055C00F5F1F4F0430110559F720
:10DDE000E1CF8091A1048C3308F055C080911106D9
:10DDF0008823B1F08091BD05482F582F550F550B42
:10DE00009A0133272F5F3F4F80919F0490E028179E
:10DE100039073CF08091A104841708F04DC001C07F
:10DE20009DD580919F048B30D0F469E080E00E9402
:10DE3000563E80911206909113060E945B3E69E067
:10DE40008EE60E94563E2091CB0583E090E0821B37
:10DE500091096FEF7FEF8E519E4C0E94B13E0E9460
:10DE6000D97E882391F10F90DF91CF911F910F916F
:10DE7000FF90EF90DF90CF90BF909F908F90ABC5B9
:10DE800027E04B2D400F632F8BE694E039830E94EF
:10DE90000B343981A0CF20E14DE36091C1058BE6C1
:10DEA00094E00E940B3420E14CE36091C1058BE6C5
:10DEB00094E00E940B349ACF6091BF0502E022E00B
:10DEC0008BE694E00E944C34ACCF0F90DF91CF9161
:10DED0001F910F91FF90EF90DF90CF90BF909F9098
:10DEE0008F90089565EA7CE682E064D588E38093AC
:10DEF000C10583E08093CB0580E48093CA05E2EC02
:10DF0000F5E0118210821382128215821482178228
:10DF10001682F3DC82E190E09093F0068093EF06A6
:10DF200008958F929F92AF92BF92CF92DF92EF921D
:10DF3000FF92CF937091E405AFEDB5E020E030E0C3
:10DF400090E080E0622FCD902F5F3F4FC110722F85
:10DF50008C296295607F40E050E0D12CE12CF12CBF
:10DF600046015701042E04C0B694A7949794879451
:10DF70000A94D2F780FE08C0E92FF0E0E053FA4F90
:10DF8000C62FC42BC0839F5F4F5F5F4F4530510545
:10DF900039F723303105B1F67093E40540E050E0E5
:10DFA00020E090E0A0E0B0E06C017D01042E04C010
:10DFB000F694E794D794C7940A94D2F7C0FE05C0AC
:10DFC0002093E6052AE335E007C02E504F5F5F4FF0
:10DFD0004530510549F7F4CF422F3150A0F0225F70
:10DFE0006C017D01032E04C0F694E794D794C79486
:10DFF0000A94D2F7C0FEF0CF4093E5058091E30587
:10E00000823069F403C02093E505F8CF8091E705DD
:10E01000181614F08CEF01C084E08093E705CF91CF
:10E02000FF90EF90DF90CF90BF90AF909F908F9038
:10E03000089580E090E0FC01E651FA4F12820396C9
:10E040008E319105C1F708951092E9058AE0809319
:10E05000E80583E08093E7058FE08093E305EFED2B
:10E06000F5E08FE18083818382835BDFE2CF1F93C2
:10E07000CF93DF93EC01162FDCDF80910E068093A7
:10E080000B0687E380930C0686E080930D066AE01A
:10E0900070E088EE93E00F94744890910F069150D1
:10E0A00090930F06992351F010920A06188310924C
:10E0B0000E061092F0061092EF0601C01882DF9152
:10E0C000CF911F9108955F926F927F928F929F924E
:10E0D000AF92BF92CF92DF92EF92FF920F931F9376
:10E0E000CF93DF9384E0809323028091F10688230D
:10E0F00009F467C28091EF069091F0068E31910588
:10E1000014F08DE190E097FF02C080E090E09093E2
:10E11000F0068093EF06880F991F880F991F2091B2
:10E120000E06422F022E000C550B4817590774F4A7
:10E130002D5FAC01421B510927FD5395423051051B
:10E140001CF020930E0602C080930E0620910E064E
:10E15000422F022E000C550B841795077CF4235098
:10E16000422F022E000C550B481B590B4230510513
:10E170001CF020930E0602C080930E0680911106BB
:10E18000882309F41EC22091CE05222349F09091E4
:10E19000CF05920F9093CF05933F14F41092CE05C4
:10E1A000823070F0815080931106823011F44CDF80
:10E1B00008C2843609F005C281E08093110601C2CD
:10E1C0008091CD058F5F8093CD054091E30590E070
:10E1D000242F30E035952795281739070CF0ACC06F
:10E1E0009091CC0581E089278093CC051092CD05D4
:10E1F000442309F4A1C09091E7058091E905890FB6
:10E200002091E605821724F02091E5052817D4F423
:10E2100091959093E7052091E8052B5F2093E80501
:10E220008093E9058091E4053AE08302C00111245E
:10E23000820F911D27FD9A95C99724F064E181E131
:10E2400096E015DF9091E9058091E705890F8093AD
:10E25000E9058091E305882309F46EC024E130E0EC
:10E2600040E050E060E070E0CB010E946337672B34
:10E27000682B692B09F060C0ECEEF5E0C0E0D0E05F
:10E280008081811153C0CE01880F991FC80FD91FFB
:10E29000C651DA4F209709F44FC02091E30530E0D2
:10E2A0002F5F3F4F032E000C440B550B60E070E0D6
:10E2B000CB010E946337FB01E053FA4F4081242FCA
:10E2C00030E0B4E035952795BA95E1F7F901E655C8
:10E2D000FC4F808190E04F705091E9056EE0469FC1
:10E2E000500D1124452FFC01E955FC4F5081450F7D
:10E2F000FC01EC55FC4F90819695842F890F888303
:10E300008091E80582502F5F3F4F9AE0299F800D52
:10E310001124898322E030E040E050E060E070E0CA
:10E32000CB010E9463376E5F6A8306C021963396E5
:10E33000CA30D10509F0A4CF90910A06992341F083
:10E3400080910906890F8093090687FD10920A06BD
:10E3500080910A06882309F4A2C020910906E09161
:10E36000E8052E170CF49BC0022E000C330B0E2E6A
:10E37000000CFF0BCF014D96821793070CF48FC052
:10E38000E0900806CE2D0E2C000CDD0B1091E90557
:10E39000CE01811B910917FD93956EE070E00F94FB
:10E3A0006351F62E653008F07AC02E1B3F0BC90171
:10E3B00002966AE070E00F946351062F633008F014
:10E3C0006EC0812C912C540183940F2C04C0880CB6
:10E3D000991CAA1CBB1C0A94D2F7A62F660FBB0B74
:10E3E000BD0161527A4FFB019081892F882109F488
:10E3F00056C0FD01E655FC4FE0814E2F50E0812FC5
:10E40000FEE0FF9E800D11249A0129553C4FF90131
:10E41000F080F80EEF140CF442C0FA01EC55FC4FFA
:10E420001081412F50E04F0D511DF7FC5A95C41734
:10E43000D507ACF510920A06282D20952923FB015B
:10E44000208323E030E02A1B3B0B80911206909141
:10E450001306280F391F30931306209312066AE023
:10E4600070E088E290E00F9474482091E805FAE0AB
:10E470000F9F200D1124912F96958F2D890F855078
:10E4800080930B0620930C0684E080930D06809108
:10E49000E30581508093E305882321F042DDCCEE33
:10E4A000D5E011C084E180931106C3DDF8CFFE01F1
:10E4B0008291890F8083803454F01882239626E05D
:10E4C000CA30D207E1F098819923C1F3F0CF8733A6
:10E4D000ACF3FE013297208180910E06281774F369
:10E4E000022E000C330B082E000C990B0A96821793
:10E4F000930724F368E781E196E0B9DDDFCF8091EF
:10E50000CE05811124C024EF31E040E050E060E00E
:10E5100070E0CB010E946337672B682B692BB9F43D
:10E5200022E030E040E050E060E070E0CB010E948B
:10E530006337672B682B692B09F091C18FEF8093AC
:10E54000CE05813009F48DC18FE78093CF0580918E
:10E550000A068823B1F18091CE05882391F180913C
:10E560000906873074F5209108068091CF05281799
:10E5700044F1022E000C330B082E000C990B0C9664
:10E5800082179307F4F01092CE0510920A0680913C
:10E590001206909113060A96909313068093120622
:10E5A0006AE070E088E290E00F9474488091CF05B3
:10E5B0008F5F80930B0681E080930C0684E080934C
:10E5C0000D068091F90682FF04C08091E20581501A
:10E5D00001C08AE08093E2050E94D97E8823C1F0C1
:10E5E00080911106811103C01092E20511C08130A3
:10E5F00079F480910A0681110BC080910E068B5F21
:10E600008093080684E3809309068CEF80930A06C2
:10E610008091E205811101C0DED161E08BE694E0DA
:10E620000E94FA31C091E8054C2F0C2E000C550BBE
:10E630008091E4059A016AE08602200D311D1124C3
:10E640002250310980919F0490E0821793072CF0AB
:10E650008091CE05811165C069C08091A10490E0D0
:10E6600084179507ACF37AEA672E73E0772EEFED07
:10E670008E2EE5E09E2EFEE15F2E5C0EF301C19032
:10E680003F012C2F0C2E000C330BA901495F5F4F6B
:10E6900080919F0490E0481759073CF4C65FFFEF54
:10E6A0008F1A9F0AC511EACFD3CF8091A10490E0C1
:10E6B000821793079CF3D091E90516E41D0FA12C56
:10E6C000B12CD12CCC0CDD1CF401808190E0A0E0B9
:10E6D000B0E00A2C04C0B695A795979587950A9443
:10E6E000D2F780FF17C08091CC057601E80EF11CAF
:10E6F000C70164E0880F991F6A95E1F79C012B5EC2
:10E700003D4C790108E022E04C2F6D2F8BE694E020
:10E710000E942432D25F3FEFA31AB30AD113D4CFA1
:10E72000BDCF80919F04883008F49DC08091110670
:10E73000882369F090919F049F3348F49091A1043D
:10E74000973328F0823008F49CC081FD9AC08091F4
:10E750000A068823B1F040910906242F042E000CEC
:10E76000330BB9016D5F7F4F80919F0490E0681774
:10E7700079073CF08091A10490E0821793070CF098
:10E780008EC0C0E0D0E0FE01E651FA4F82818823BE
:10E7900099F04181842F042E000C990B20919F0445
:10E7A00030E08217930744F002972091A10430E0F3
:10E7B000281739070CF07BC02396CE31D10519F705
:10E7C00080910D068823B1F040910C06242F042E71
:10E7D000000C330BB9016A5F7F4F80919F0490E07A
:10E7E000681779073CF08091A10490E082179307A5
:10E7F0000CF065C080911106811101C0AFD08091ED
:10E800009F048A3008F06DC069E080E00E94563EA7
:10E8100080911206909113060E945B3E80910F0634
:10E82000882309F45EC0C1E040E1C42ED12C809160
:10E830000F068C1708F455C0B6016C1B7109660FE2
:10E84000660F660F50E0E52E52E3F52E05E021E05D
:10E8500041E08BE694E00E942432CF5FE8CF81E074
:10E860006ECE83EF72CE28EEE22E21E3F22E05E08B
:10E8700022E042E06091CF058BE694E00E942432D2
:10E8800055CF95E0E92E92E3F92E08E022E047E328
:10E8900060910E068BE694E00E94243258CF24E06B
:10E8A000609108068BE694E00E942B346ACF4250B8
:10E8B00023E060818BE694E00E942B347DCF82EFD1
:10E8C000E82E81E3F82E07E022E060910B068BE64C
:10E8D00094E00E94243280910D06815080930D06B1
:10E8E00089CFDF91CF911F910F91FF90EF90DF9033
:10E8F000CF90BF90AF909F908F907F906F905F90E0
:10E90000089563E670E784E155D083E080930F06B5
:10E910008AE08093E20510920A0696DB10920E06BA
:10E920001092F0061092EF0608958091F106882368
:10E9300019F082E08093100684E080932302809196
:10E940001106882349F0909110068FEF890F80936C
:10E95000100681E019160CF080E008950F93809165
:10E960009F04853228F58091A1048B3108F160E085
:10E970008BE694E00E94FA3109E028E34BE164E27F
:10E980008BE694E00E949C3461E08BE694E00E9468
:10E99000FA310E94AA7F882359F063E285E20E943F
:10E9A000563E6FEF7FEF85E792E30F910C94B13EF7
:10E9B0000F910895FB011092130610921206809396
:10E9C000110620E040E060E070E0CF01F2D481E089
:10E9D0008093F70608951092F70619C580911406E2
:10E9E0009091160689130DC0809115069091170617
:10E9F000891714F02FEF01C021E0820F80931506D4
:10EA000008C0891714F02FEF01C021E0820F809316
:10EA10001406891319C02091780621502093780696
:10EA200030E0832F90E0DC01AA0FBB1FAC5EB94F32
:10EA3000880F991FFC01EA5EF94F808191818D93C7
:10EA40009C933F5F231768F70895EF92FF921F93FF
:10EA5000CF93DF931091780620917F06E22E022E4D
:10EA6000000CFF0830918006C32F032E000CDD0B35
:10EA7000E7E1F6E040E0411709F446C0CF01039713
:10EA8000DC019C91BF0161507109DB018C919813ED
:10EA90001DC0692F092E000C770B61507109C61734
:10EAA000D70711F039132DC09081BF016250710951
:10EAB000DB018C91582F98170CF4592F25170CF166
:10EAC00089170CF4892F8217E4F020C0BF0162502F
:10EAD0007109DB015C91652F052E000C770B6150ED
:10EAE0007109E616F70611F025130BC0582F981779
:10EAF0000CF4592F35172CF089170CF4892F831734
:10EB00002CF44F5F3296B7CF80E001C081E0DF91F7
:10EB1000CF911F91FF90EF90089528E130E040E001
:10EB200050E060E070E0CB010E94633760938006A4
:10EB30002AE030E040E050E060E070E0CB010E946D
:10EB4000633760937F0681DF8111E7CF089590914D
:10EB50008106811102C08FEF01C081E0980F937090
:10EB600090938106E0917806EF5FE0937806F0E0FD
:10EB7000EE0FFF1FEC5EF94F80917C068083809141
:10EB80007A0681830895CF9380E091E090937C068C
:10EB900080937B0680E095E090937A0680937906D7
:10EBA0001092810610927806E4E1F6E01082C5E04A
:10EBB000C18381E0CCDFC0937E061092F0061092F4
:10EBC000EF0610927D06CF910895EF92FF920F937A
:10EBD0001F93CF93DF9380917806843008F4B1C0FF
:10EBE00090E0FC01EE0FFF1FEE5EF94F2081EC017B
:10EBF000CC0FDD1FCC5ED94F68810297261719F024
:10EC0000F12C31966BC0E12C219631964E2D50E0BF
:10EC1000481759070CF095C0BA01660F771F8B0192
:10EC20000C5E194FD801FC90DB01AA5EB94F3C91F4
:10EC3000F316E9F0432FF3160CF44F2D24179CF133
:10EC40003F150CF43F2D321774F1DB01AC5EB94F68
:10EC500011965C9141E0308153170CF040E031E0B7
:10EC6000688165170CF430E04317E9F06CC02F1190
:10EC70001AC06881408111965C91D80111963C912F
:10EC8000A42F64170CF4A62F732F35170CF4752FCF
:10EC90007A174CF046170CF4462F53170CF4352F07
:10ECA00043170CF050C0E394B1CFEA01CC0FDD1F45
:10ECB0008E010C5E194FD80111967C91DE01AA5E7F
:10ECC000B94F11963C911197731709F14081532F59
:10ECD00073170CF4572F45173CF4F3944F2D50E065
:10ECE0004817590714F32DC037170CF4372F341772
:10ECF000A4F3CC5ED94F588141E052170CF040E0AC
:10ED000031E065170CF430E0431739F31CC0308153
:10ED10003713E3CF4C91D8013C91762F26170CF492
:10ED2000722F532F34170CF4542F5717B4F2562F59
:10ED300062170CF4522F43170CF4342F53176CF254
:10ED400002C080E001C081E0DF91CF911F910F915F
:10ED5000FF90EF900895CF92DF92EF92FF920F9382
:10ED60001F93CF93DF931F92CDB7DEB7DEDD8823ED
:10ED700009F480C080917B0690917C06392F4091E8
:10ED8000790650917A0620918106213061F02CF4A9
:10ED9000211116C0CA01C3970AC0223031F02330B6
:10EDA00079F4C39709C0C39607C0CA01C39690936C
:10EDB0007A068093790604C090937C0680937B0644
:10EDC00010917C0600917A06311303C0051709F4EF
:10EDD00051C0183110F40A3048F01092110668E260
:10EDE00070E080E991E00F94744844C0E0917806A7
:10EDF000F0E0EE0FFF1FEC5EF94F1083018380916E
:10EE0000EF0690917D06282F291B39F080937D060F
:10EE100081E012160CF080E09ADE80917E06882355
:10EE200021F0815080937E0601C0D8DDCEDE8111B5
:10EE3000D4CF8091800618131DC080917F060813DF
:10EE400019C06CED70E085E090E00F94744868E1C3
:10EE500071E085E090E00F947448809112069091E3
:10EE600013060196909313068093120682E0809316
:10EE70007E0653DE61E08BE694E00E94FA318091D9
:10EE80009F04893050F467E080E00E94563E8091F4
:10EE90001206909113060E945B3E06E32CE749E0C0
:10EEA00062E08BE694E00E944C34F12C809178066D
:10EEB00020919F04F81608F071C0EF2DF0E0AF012B
:10EEC000440F551FDA01AC5EB94F9C91FA01EA5E1E
:10EED000F94F8081981345C091811196EC901E2DB9
:10EEE000E9160CF4192F85E01802B0011124625FB5
:10EEF0007F4F30E0621773070CF44EC09E150CF480
:10EF0000E92E9E2DE5E09E0290011124265F3F4FE1
:10EF10008091A10490E028173907F4F58E2D880F11
:10EF2000880F8E0D7BE0780FCA018C5E994F6C01C3
:10EF30001E1594F1272F072E000C330BA9014D5FEE
:10EF40005F4F80919F0490E0481759073CF08091F3
:10EF5000A10490E0821793070CF04CC0E3947B5F10
:10EF6000E7CF11963C91432F440F440F340F4BE0F1
:10EF7000D42ED30E4D2D0D2C000C550BBA016D5F08
:10EF80007F4F30E0621773073CF02091A10430E01E
:10EF9000241735070CF03FC0F39488CF40917F06CB
:10EFA000842F880F880F480F455F642F042E000CB4
:10EFB000770BFB013396822F90E0E817F9073CF0BE
:10EFC0008091A10490E0861797070CF043C08091D0
:10EFD0001106811101C0C2DCECD6882309F448C0B7
:10EFE0000F90DF91CF911F910F91FF90EF90DF90E5
:10EFF000CF90F1CCF6016081862F880F880F680FC3
:10F000006C5F04E024E0472F8BE694E079830E9454
:10F010009C347981A3CFE82E98170CF4E92EC82EE2
:10F0200089170CF4C92E1E2D110F110F1E0D50E063
:10F030001C5FCE140CF4B0CF612F650F04E024E008
:10F040004D2D8BE694E059830E949C34E3945981C2
:10F050005B5FEFCF60918006862F880F880F680F67
:10F060006C5F04E024E08BE694E00E944C34AFCF68
:10F070000F90DF91CF911F910F91FF90EF90DF9054
:10F08000CF9008956BEA76E781E094DC7CDD45CD96
:10F090000F931F93CF93DF9361E081E08ED2D091E5
:10F0A000C906C0E0D11116C08091C806811103C005
:10F0B00080D681119AC080912302882309F43CC034
:10F0C00081E09091C806911180E004E024E04EECCC
:10F0D00052E32FC0D130B1F48091C806813019F4C9
:10F0E00068D6811189C080912302882329F181E0AB
:10F0F0009091C806913009F080E003E02EE34CEBDC
:10F1000052E317C0D230C1F48091C806823019F49E
:10F1100050D681117BC080912302882369F081E061
:10F120009091C806923009F080E003E02EE34DEAAA
:10F1300052E36C2F0E94494325D1182FD330D1F4CC
:10F140008091C806833019F434D6811169C080914A
:10F150002302882309F476C081E09091C806933099
:10F1600009F080E000E22EE34EE952E36C2F0E94AA
:10F17000494368C0811168C0D430B1F48091C80699
:10F18000843019F416D6811152C08091230288234D
:10F1900019F181E09091C806943009F080E000E216
:10F1A0002EE340E952E315C0D530B1F48091C80692
:10F1B000853009F443C080912302882369F081E0FF
:10F1C0009091C806953009F080E000E22EE34FE709
:10F1D00052E36C2F0E94494386E0CF5FDF5FC5306A
:10F1E00009F060CF8093C7063AC011D1809195068F
:10F1F000882309F460CF33C083EF90E50E94A247D3
:10F2000080919506882309F46ECF29C083E49BE79B
:10F210000E94A24780919506882309F47CCF1FC0E5
:10F22000BED280919506882309F491CF18C0BAD236
:10F2300080919506882309F4A8CF11C0BAD5811111
:10F2400005C0B9CF112341F284E0C7CF0E945FDA35
:10F2500081E005D280919506882309F4ACCFDF9137
:10F26000CF911F910F910895E0919606E63000F539
:10F2700081E08E0F809396068091EF069091F006C4
:10F28000A0E0B0E03091C9062091C70648E0E49FB5
:10F29000F0011124E956F94F4091EA065091EB062E
:10F2A0005183408382839383A483B58336832783EA
:10F2B00008950D94613D2F923F924F925F926F920D
:10F2C0007F928F929F92AF92BF92CF92DF92EF92F6
:10F2D000FF920F931F93CF93DF9300D000D0CDB751
:10F2E000DEB71C012B833C834D835E8369837A8365
:10F2F000BBDF83E080932302309294062092930632
:10F3000069817A8170939206609391062B813C818A
:10F310004D815E8120938D0630938E0640938F063B
:10F3200050939006E0928906F0928A0600938B062D
:10F3300010938C06D092F006C092EF06B092EB06C6
:10F34000A092EA0690928806809287068C8D809320
:10F35000860626960FB6F894DEBF0FBECDBFDF91AE
:10F36000CF911F910F91FF90EF90DF90CF90BF90C2
:10F37000AF909F908F907F906F905F904F903F9055
:10F380002F9008958091FE0E9091FB0E891B8F7037
:10F3900071F49091A60992FB882780F992FD08C02C
:10F3A00081E090915318913019F080E0089581E048
:10F3B0000895E091EA06F091EB06E817F907F9F0F5
:10F3C0009093EB068093EA067093F0066093EF0645
:10F3D0004093C9062093C70689539E4721F4109293
:10F3E000F706109296060E948A4282E080932302DA
:10F3F00081E0809395061092F2061092820608959D
:10F4000020E040E060E070E089E39EE7D2CFE09149
:10F410009606EE2381F0E150E093960688E0E89F9F
:10F42000F0011124E956F94F2781468160E070E030
:10F4300080819181BECFE4CFCF93DF93FC01EB01BC
:10F440008091EF069091F00697FF04C01092F006AD
:10F450001092EF064091890650918A0660918B06C2
:10F4600070918C068091EF069091F006092E000CA9
:10F47000AA0BBB0B481759076A077B0724F4509364
:10F48000F0064093EF06809123028823D1F020916B
:10F49000EF063091F00680918D0690918E06A09136
:10F4A0008F06B0919006BC01CD01620F731F811DC4
:10F4B000911D1995BC0180919306909194060E942C
:10F4C000D4438091E406811108C080918606882388
:10F4D00081F180912302882361F1809191069091BE
:10F4E0009206009791F02091EF063091F00640913E
:10F4F0008D0650918E0660918F0670919006420F96
:10F50000531F611D711DFE011995E0918706F09151
:10F510008806309741F080918606811103C0809162
:10F52000E4068111199545D4882319F0DF91CF9114
:10F530006ECFDF91CF9108950F931F93CF93DF93F9
:10F5400080912302882359F060918306709184068C
:10F5500000E010E020E041E081E00E94EA4280917A
:10F56000850681111CC081E080938506C091EA0662
:10F57000D091EB0620E040E060E070E08CE99AE793
:10F5800018DF0E944AF51092850620E040E060E016
:10F5900070E0CE01DF91CF911F910F910ACFDF91E3
:10F5A000CF911F910F910895009711F482EE92E38D
:10F5B0009093840680938306BFCF282F1092E9068C
:10F5C0008091EF069091F0068130904820F01092E3
:10F5D000F0061092EF068091F106882331F08091B9
:10F5E000EF068093C806109295068091C7061816FC
:10F5F000BCF4082E000C990B821B91092091C806BF
:10F60000022E000C330B2817390754F097FF02C065
:10F6100080E090E08093C8069093F0068093EF0618
:10F620008091C8066623C1F09091C906891714F429
:10F630008093C9062091C906022E000C330B2C5F63
:10F640003F4F482F082E000C550B2417350734F474
:10F6500084508093C90608958093C906089588232D
:10F6600061F063E972E084E690E00F9474486AEB1D
:10F6700072E084E690E00D94744868EB71E084E1F8
:10F6800090E00D947448CF92DF92EF92FF92CF9367
:10F69000DF938FD3882359F00E9451D61092F7063A
:10F6A000DF91CF91FF90EF90DF90CF90B0CE81E0CF
:10F6B0008093F706C091EF06D091F006209709F4E9
:10F6C00042C01092F0061092EF06BE010D2E000C03
:10F6D000880B990B0F94CE4E2091980E3091990E75
:10F6E00040919A0E50919B0E0F946A502091D90D23
:10F6F0003091DA0D4091DB0D5091DC0D0F94534D9C
:10F700006B017C0120E030E040E050EC0F942F5082
:10F7100087FD19C020E030E040EA50E4C701B6019F
:10F720000F942C4E18167CF0BE0182E00E947CAA39
:10F73000C092D90DD092DA0DE092DB0DF092DC0D83
:10F7400082E080932302809123028823C9F089ED0F
:10F750009DE00E94789DBC0183ED92E30E94D4431A
:10F760006091D90D7091DA0D8091DB0D9091DC0DD7
:10F77000DF91CF91FF90EF90DF90CF900C940145F7
:10F78000DF91CF91FF90EF90DF90CF90089521E02F
:10F79000209385060F94663D1092850608950E9479
:10F7A0008CD65DCF0E9403E55ACF4F925F926F9245
:10F7B0007F928F929F92AF92BF92CF92DF92EF9201
:10F7C000FF920F931F93CF93DF931F921F92CDB79A
:10F7D000DEB72C014A0139015801870176012091D9
:10F7E000EF063091F0062115310559F081E012162F
:10F7F00013060CF080E0809382061092F0061092BF
:10F80000EF0669837A83D5D2D82E69817A818111F6
:10F8100004C080912302882311F195014091820652
:10F82000C2010E94A844DD20D1F080918206882385
:10F8300011F0F40101C0F3010F900F90DF91CF910F
:10F840001F910F91FF90EF90DF90CF90BF90AF90FE
:10F850009F908F907F906F905F904F9019940F9032
:10F860000F90DF91CF911F910F91FF90EF90DF905C
:10F87000CF90BF90AF909F908F907F906F905F9050
:10F880004F900895FC0180810895FC0184910895B2
:10F890004F925F926F927F928F929F92AF92BF92A0
:10F8A000CF92DF92EF92FF920F931F93CF93DF934C
:10F8B0006C017B015A012901672B31F08824839464
:10F8C000912CC0E0D0E019C0F8011182108227C04D
:10F8D0003701680C791C76946794E3012197A201A3
:10F8E000BE01C601F50119951816190654F0892BA9
:10F8F000C9F04301FFEF8F1A9F0AE814F90440F79B
:10F9000002C07E01FACFCE15DF0530F4CE0102969B
:10F910008816990620F02196F801D183C0838FEFD5
:10F920009FEF05C0F801D183C08380E090E0DF91B4
:10F93000CF911F910F91FF90EF90DF90CF90BF90EC
:10F94000AF909F908F907F906F905F904F900895B1
:10F950008F929F92AF92BF92CF92DF92EF92FF92DF
:10F960000F931F93CF93DF93EC016B017A01FB019F
:10F97000199587FD06C0082F10E020E030E02196A1
:10F9800020C1982F907E903CC1F4082F0F7110E099
:10F9900020E030E04801590186E0880C991CAA1C3F
:10F9A000BB1C8A95D1F7CE010196F60119958F738C
:10F9B00095018401082B229604C1982F907F903ED8
:10F9C00019F58F70882E912CA12CB12C16E0880C83
:10F9D000991CAA1CBB1C1A95D1F7CE010196F60101
:10F9E00019958F73882A06E0880C991CAA1CBB1CE9
:10F9F0000A95D1F7CE010296F60119958F739501FC
:10FA00008401082B2396DDC0982F987F903F81F5C5
:10FA10008770882E912CA12CB12CF6E0880C991CB3
:10FA2000AA1CBB1CFA95D1F7CE010196F6011995D7
:10FA30008F73882AA6E0880C991CAA1CBB1CAA9567
:10FA4000D1F7CE010296F60119958F73882AB6E098
:10FA5000880C991CAA1CBB1CBA95D1F7CE01039641
:10FA6000F60119958F7395018401082B2496A9C07E
:10FA7000982F9C7F983FE9F58370882E912CA12CBC
:10FA8000B12C56E0880C991CAA1CBB1C5A95D1F7C6
:10FA9000CE010196F60119958F73882A66E0880CCD
:10FAA000991CAA1CBB1C6A95D1F7CE010296F601DF
:10FAB00019958F73882A76E0880C991CAA1CBB1CA8
:10FAC0007A95D1F7CE010396F60119958F73882A9E
:10FAD000E6E0880C991CAA1CBB1CEA95D1F7CE0164
:10FAE0000496F60119958F7395018401082B2596CC
:10FAF00068C0982F9E7F9C3F09F04AC08170882E75
:10FB0000912CA12CB12C86E0880C991CAA1CBB1C42
:10FB10008A95D1F7CE010196F60119958F73882A3F
:10FB200096E0880C991CAA1CBB1C9A95D1F7CE01B3
:10FB30000296F60119958F73882A26E0880C991C85
:10FB4000AA1CBB1C2A95D1F7CE010396F601199584
:10FB50008F73882A36E0880C991CAA1CBB1C3A9526
:10FB6000D1F7CE010496F60119958F73882A46E0E5
:10FB7000880C991CAA1CBB1C4A95D1F7CE0105968E
:10FB8000F60119958F7395018401082B269619C0EB
:10FB9000982F907C903849F4082F007C003871F43D
:10FBA0002196CE01F6011995F7CF082F0E7F0D3F54
:10FBB00028F02196CE01F6011995F7CF00E010E06C
:10FBC0009801E114F10429F0F701008311832283E5
:10FBD0003383CE01DF91CF911F910F91FF90EF9072
:10FBE000DF90CF90BF90AF909F908F9008951F931C
:10FBF000CF93DF9300D01F92CDB7DEB710E0AE01F8
:10FC00004F5F5F4F62E47CE7A3DE49815A816B81DD
:10FC10007C81452B462B472B11F01F5FF0CF812FA6
:10FC20000F900F900F900F90DF91CF911F9108953B
:10FC30001F93CF93DF9300D01F92CDB7DEB710E0B4
:10FC4000AE014F5F5F4F65E47CE782DE49815A81F8
:10FC50006B817C81452B462B472B11F01F5FF0CF2A
:10FC6000812F0F900F900F900F90DF91CF911F91E8
:10FC700008951092E9068091E4061092E406882324
:10FC800049F020E040E060E070E081EE92E691DB38
:10FC90000C94584220916702309168024091EF061F
:10FCA0005091F006C901840F951F2436310551F497
:10FCB0004730510514F006972CC04A3F5F4F34F58A
:10FCC000069627C02436310524F485369105F4F4D0
:10FCD00004C08436910524F419C08A3091053CF0A3
:10FCE000883E43E094072CF087EE93E002C08AE060
:10FCF00090E02817390741F09093680280936702DB
:10FD00001092F0061092EF060C944A3E84E690E0C2
:10FD1000E7CF8A30910524F78AE090E0EDCFCF93CA
:10FD2000DF931F92CDB7DEB780915709811103C0D1
:10FD300089E999E02FC0211103C087E599E02AC025
:10FD40008DE0815048F0440F411DE82FF0E0E75668
:10FD5000F64F90814927F5CF8091DB068417A9F0F3
:10FD60004093DB0687E599E0698341DF90E0698194
:10FD7000861B910997FF02C080E090E08093EC061B
:10FD80001092ED0688E0809325028091ED0690E0C8
:10FD9000895A964F0F90DF91CF9108958093E9068D
:10FDA0001092E5061092E6061092E7061092E80619
:10FDB00008958091E4061092E40608959F92AF9210
:10FDC000BF92CF92DF92EF92FF920F931F93CF9348
:10FDD000DF9300D01F92CDB7DEB78C017B015A01B3
:10FDE0006901FB0180816CE0689F600D1124F801BE
:10FDF0008081982F990F890F880F0E94563EA11479
:10FE0000B10471F19B2C8CE0B82EAE014F5F5F4FB7
:10FE1000B6018A2D992D9CDDA82E992E69817A81B3
:10FE20008B819C816115710581059105C9F04FEFAA
:10FE30005FEF0E94613EF80130813F5F353110F481
:10FE40003083E3CFF8011082F70130813F5F3083C8
:10FE50006B2DB39E600D112480E00E94563ED5CFDD
:10FE60000F900F900F900F90DF91CF911F910F91F6
:10FE7000FF90EF90DF90CF90BF90AF909F9008954C
:10FE8000BF92CF92DF92EF92FF920F931F93CF9387
:10FE9000DF931F921F92CDB7DEB76C017B018A0101
:10FEA000C7DEB82E0115110519F0C801C1DE01C069
:10FEB00080E01A821982E114F104C1F44B2D50E064
:10FEC00090E09A01280F391F263131057CF425E195
:10FED00030E0241B350B281B390B37FF02C02F5F86
:10FEE0003F4F359527952A8381E0898325E43CE7B8
:10FEF000A601BE016F5F7F4FCE0102965FDFE11466
:10FF0000F10481F08A81882321F01A8289818F5F30
:10FF1000898322E43CE7A701BE016F5F7F4FCE01DA
:10FF200002964CDF0115110549F025E43CE7A801D4
:10FF3000BE016F5F7F4FCE01029640DF0F900F90A2
:10FF4000DF91CF911F910F91FF90EF90DF90CF90B5
:10FF5000BF900895CF92DF92EF92FF920F931F937D
:10FF60000E94D62C0091D7061091D8062091D90670
:10FF70003091DA066B017C01C01AD10AE20AF30A59
:10FF8000F7FC13C02091D60620952093D606DC01FD
:10FF9000CB018A549C4FAF4FBF4F8093D7069093AD
:10FFA000D806A093D906B093DA0681E09091D606E0
:10FFB000911101C080E01F910F91FF90EF90DF90B1
:10FFC000CF900895CF9393E09093230281111092E4
:10FFD000F9060E94D62CDC01CB018C509E4FAF4F0E
:10FFE000BF4F8093F3069093F406A093F506B09369
:10FFF000F60668E873E182E090E00F947448C6E08A
:020000021000EC
:10000000C15049F00F94134862E070E080E090E046
:100010000E94072DF5CFCF910895AF92BF92CF9256
:10002000DF92EF920F931F93CF93DF9300D01F9235
:10003000CDB7DEB7809124028F3F09F444C00E94FF
:10004000D62C0091DC061091DD062091DE06309161
:10005000DF06DC01CB01801B910BA20BB30BB7FDBC
:1000600032C09091FB0E8091FE0E8F5F8F709817BB
:1000700051F1E091240284E0E802F0011124E355FB
:10008000FC4F20E030E040E752E4608171818281E2
:1000900093810F94334E69837A838B839C83A12C45
:1000A000B12C6501E12C8E010F5F1F4F29E732E073
:1000B00045E752E061E772E08DE692E00F94B0020E
:1000C0008FEF809324020F900F900F900F90DF918D
:1000D000CF911F910F91EF90DF90CF90BF90AF9095
:1000E00008950F931F930E94D62C0091F306109150
:1000F000F4062091F5063091F606DC01CB01801B59
:10010000910BA20BB30BB7FD0FC08091030185FBD0
:10011000992790F981E089279091030196FF8260E9
:10012000629B84608093F9068091F90681709091BA
:10013000F90691FD82609091CA06891741F18130DC
:10014000A9F028F0823041F0833059F01EC0913080
:1001500089F09230A9F019C0992361F0933081F0B1
:1001600014C0913069F0923081F404C0992341F0B9
:10017000933059F49091EE069F5F9093EE0605C080
:100180009091EE0691509093EE068093CA061F91CF
:100190000F910895CF93DF930E945842E4E0F1E07D
:1001A00080818F7D8083C5E0D1E0888180958072D9
:1001B000A3E0B1E08C9380818F7B808388818095E0
:1001C00080748C936A98729A54985C9A82E08093B7
:1001D000F80687DF1092EE06DF91CF91089581E057
:1001E0009091FB06911101C080E00895CF93DF93B9
:1001F0002091110721111EC0FC0101900020E9F798
:100200003197EF01C81BD90BC631D10534F03197B6
:100210002081207C2038D9F3F4CFBC01DD27AE014A
:100220008BEF96E00F94B456C550D94F188283E0F7
:1002300080932302DF91CF910895CF93DF93CDB7C1
:10024000DEB78E8190911107891780F08093110796
:100250009E01275F3F4F4F81588565E170E08BEF2E
:1002600096E00F94FD5683E080932302DF91CF91B7
:1002700008950F931F93CF93DF938C0167FF03C003
:100280001092110760E08091110790E0262F062E52
:10029000000C330B281739070CF160931107C801C4
:1002A0000F941656F801E80FF91FEF01C01BD10B90
:1002B000C631D10534F031978491807C8038D9F3F0
:1002C000F4CFDD27AE01B8018BEF96E00F943756DF
:1002D000C550D94F188283E080932302DF91CF91DC
:1002E0001F910F9108954F925F926F927F928F921C
:1002F0009F92AF92BF92CF92DF92EF92FF920F93B5
:100300001F93CF930E94D62C6B017C0186DEE9DE21
:100310008091F90682FF15C08091D506811113C026
:1003200091E09093D50620915E18211103C0809131
:10033000850689278093E40610925E1881E042DEEC
:1003400002C01092D50689B184FB992790F981E00B
:100350008927C091F8068C1749F18093F806882305
:1003600009F4B2C164EF71E080E090E00E947D9CEE
:100370000E94958DC23009F0A2C10E94668E83E072
:10038000809323020E9458420E94D62C6B017C016C
:10039000DC01CB018C599F4FAF4FBF4F8093D106EB
:1003A0009093D206A093D306B093D4068091D10641
:1003B0009091D206A091D306B091D406A7019601E0
:1003C000281B390B4A0B5B0B57FF05C08091F206C7
:1003D000882309F43BC2D701C6018C599F4FAF4F08
:1003E000BF4F8093D1069093D206A093D306B093CB
:1003F000D4066091EE06062E000C770B77FF03C043
:10040000719561957109062E000C770B880B990B7D
:100410000F94CE4E2B013C0120E030E040E050E450
:100420000F942F5087FF05C08091E40681117DC095
:100430008DC08091E906882309F456C08090E506B6
:100440009090E606A090E706B090E806811491042B
:10045000A104B104E1F120E030E040E05FE3C3013A
:10046000B2010F946A502B013C01C701B601681913
:1004700079098A099B090F94CC4E9B01AC01C301F9
:10048000B2010F94334E20E030E04AE754E40F9479
:100490006A504B015C0120E030E040EA52E40F94E6
:1004A0002F5087FF0FC020E030E040EF51E4C5013E
:1004B000B4010F942F5087FD0AC02AE030E040E0DD
:1004C00050E009C024E630E040E050E004C021E004
:1004D00030E040E050E0C092E506D092E606E092BF
:1004E000E706F092E80604C021E030E040E050E08A
:1004F000A091EE060091EF061091F0060A2E000C76
:10050000BB0B0F94D55122E030E040E050E00F9457
:100510009851DA01C901800F911FA11DB11D90935F
:10052000F0068093EF061092EE06D701C6018856BA
:10053000954CAF4FBF4F8093CD069093CE06A093BE
:10054000CF06B093D00681E0809323022091EA0683
:100550003091EB064EE72933340741F480912502B0
:10056000882309F4C4C08150809325022A59384455
:1005700051F580912502882321F081508093250236
:1005800022C084E0809325028091ED068F5F8093E6
:10059000ED069091EC06981728F41092ED068CE089
:1005A0008093250281E080932302D701C6018856FB
:1005B000954CAF4FBF4F8093CD069093CE06A0933E
:1005C000CF06B093D00680916F0081FB222720F9DF
:1005D00081FF05C080916F008D7F80936F008091B7
:1005E0000E0E90910F0EA091100EB091110E2223BD
:1005F00029F020916F00226020936F003AE0B695B9
:10060000A795979587953A95D1F7009721E0A2078E
:10061000B10520F08FEF9FEFA0E0B0E096958795B1
:1006200020912302211105C03091F20631110AC137
:1006300039C0009739F04091CB065091CC0648174D
:10064000590780F58091F206811103C0223008F02D
:100650005EC0C1E08091EA069091EB0689539E4707
:1006600009F0C0E08C2F0E944C3ECC2309F45BC003
:1006700000DB1092E4060E94D62CDC01CB018C1921
:100680009D09AE09BF090091CB061091CC0620E070
:1006900030E0081719072A073B0720F49093CC068F
:1006A0008093CB068091EA069091EB0689539E4792
:1006B00009F48BC08091F706811187C0B2C060E059
:1006C00086E293E3D6DD5BCEDBD5C23009F457CEAC
:1006D00060E089E193E3CDDD8091EA069091EB063D
:1006E00089539E4709F44BCE0E94007A48CE8CE095
:1006F000809325028091CB069091CC060197909330
:10070000CC068093CB0681E0809323022FCF243048
:1007100030F0243009F09DCF109223029ACF81E06F
:100720008093230296CF8091F206811114C08091AC
:10073000A404811107C081E08093A4048BE694E0B7
:100740000E94A1318BE694E00E94D83181E0809331
:10075000F1068093F20683E00E949D4161E08BE602
:1007600094E00E94FA31E091EA06F091EB061995C7
:100770001092F1068091F206882309F47ACF8BE675
:1007800094E00E94DC3191E0811101C090E09093EF
:10079000F206992309F46DCF0E94D62CDC01CB011F
:1007A0008C199D09AE09BF09C090CB06D090CC062C
:1007B000E12CF12CC816D906EA06FB0608F046C063
:1007C0009093CC068093CB0641C058E9C50E5AE3FE
:1007D000D51EE11CF11CC092CD06D092CE06E0924F
:1007E000CF06F092D0068091F20681112FC0809141
:1007F0002302813099F0833049F5CF911F910F91F9
:10080000FF90EF90DF90CF90BF90AF909F908F9030
:100810007F906F905F904F900C948A4210922302C9
:1008200015C08091CD069091CE06A091CF06B091D3
:10083000D006C81AD90AEA0AFB0AF7FCD4CF0E94EC
:10084000007AD1CF009709F404CFF5CECF911F9154
:100850000F91FF90EF90DF90CF90BF90AF909F905F
:100860008F907F906F905F904F90089561E001DDD1
:100870000C94007ACF93DF931F921F92CDB7DEB70F
:1008800089839A8387DC89819A81F0DF0F900F90AA
:10089000DF91CF910C945D428091A60982FD05C045
:1008A00080915318823061F410C0809157098111F2
:1008B00003C089E999E002C087E599E061E096CC40
:1008C000813031F08CEE92E305C08CE093E302C0FE
:1008D00080E093E36FEFCDCC8091A60982FF09C041
:1008E00083FF04C08091D607811106C020E02093C9
:1008F000FA068091FA060895809161079091620747
:10090000A0916307B09164070097A105B10571F349
:10091000BC01CD016D597F4F8F4F9F4F24E630E0D2
:1009200040E050E00F94765160915D0770915E0752
:1009300080915F07909160070F947651D8CF89E33B
:100940009EE79093EB068093EA06089561E0FC0130
:1009500080810E94062F8FEF0C94BAA9CF93DF936A
:10096000EC018A810E947BA960E08881DF91CF91B0
:100970000C94062F8F929F92AF92BF92EF92FF92AC
:100980000F931F93CF93DF93EC018B017A010E94A9
:10099000D62C4B015C012CE2820E21E0921EA11CA0
:1009A000B11C0E9494A98B838F3F61F40E94D62CC6
:1009B000DC01CB0188199909AA09BB09B7FDF1CF60
:1009C00081E10DC08E3F51F4B701C8010E949BA97F
:1009D0000E9494A90E9494A911E003C08FE089832A
:1009E00010E0CE01B3DF812FDF91CF911F910F91E6
:1009F000FF90EF90BF90AF909F908F900895CF920F
:100A0000DF92EF92FF926A017B010E94D62CC60E04
:100A1000D71EE81EF91E0E9494A98F3F61F00E9424
:100A2000D62CDC01CB018C199D09AE09BF09B7FD9D
:100A3000F2CF80E001C081E0FF90EF90DF90CF9097
:100A40000895EF92FF921F93CF93DF9300D01F92F0
:100A5000CDB7DEB77C01162F29833A834B835C83A5
:100A60007DDF48E552E060E070E0C701C8DF812F1C
:100A700080640E94BAA98C810E94BAA98B810E94CD
:100A8000BAA98A810E94BAA989810E94BAA91123B0
:100A900011F087E801C085E90E94BAA91C3011F461
:100AA0000E9494A910E00E9494A9F701838387FF14
:100AB00004C01F3F11F01F5FF6CF0F900F900F90F3
:100AC0000F90DF91CF911F91FF90EF9008958F923B
:100AD0009F92AF92BF92CF92DF92EF92FF920F93CD
:100AE0001F93CF93DF93EC01162F1C82198248834A
:100AF0000E94D62C6B017C0120EDC20E27E0D21E95
:100B0000E11CF11CA89561E088810E94062F61E03C
:100B100088810E94CA2E0E948CA985E08A830E9447
:100B20007BA90AE08FEF0E94BAA90150D9F7A895D6
:100B300020E030E0A90160E0CE0183DF8B838130CB
:100B400061F00E94D62CDC01CB018C199D09AE0905
:100B5000BF09B7FDEDCF81E055C0A8952AEA31E085
:100B600040E050E068E0CE016CDF853011F481E0B8
:100B700009C004E00E9494A98B830150D9F78A3AF6
:100B800051F482E08C83A8958C81823081F0812C95
:100B9000912C540111C00E94D62CDC01CB018C1980
:100BA0009D09AE09BF09B7FDD9CF82E02BC0812CCA
:100BB000912CA12C80E4B82E20E030E0A90167E35D
:100BC000CE013FDFA501940169E2CE013ADF8B83BC
:100BD000882361F00E94D62CDC01CB018C199D0981
:100BE000AE09BF09B7FDE8CF8AE00CC08C81823026
:100BF000D1F420E030E0A9016AE3CE0122DF8823AE
:100C000029F088E08983CE01A1DE16C00E9494A954
:100C1000807C803C11F483E08C830E9494A90E9424
:100C200094A90E9494A9CE0191DE173018F41A837A
:100C300081E003C088E1898380E0DF91CF911F913B
:100C40000F91FF90EF90DF90CF90BF90AF909F906B
:100C50008F9008950F931F93CF93DF93EC01890139
:100C60008C81833039F089E0440F551F661F771F50
:100C70008A95D1F79A01AB0161E1CE01E2DE8111E3
:100C800009C040E052E0B801CE01DF91CF911F9141
:100C90000F9170CE84E08983CE0158DE80E0DF9131
:100CA000CF911F910F910895CF93DF93EC01862F81
:100CB000BA010E94BFA98FEF0E94BAA98FEF0E94CC
:100CC000BAA90E9494A98B83982F9F71953031F017
:100CD00083E18983CE013ADE80E001C081E0DF91CB
:100CE000CF9108950F931F93CF93DF93EC01890168
:100CF0008C81833039F089E0440F551F661F771FC0
:100D00008A95D1F79A01AB0168E1CE019ADE811193
:100D10001EC0A8016EEFCE01C7DF8823E1F048E5D1
:100D200052E060E070E0CE016ADE882371F020E0DE
:100D300030E0A9016DE0CE0184DE81110AC00E947D
:100D400094A9811106C011E007C087E103C086E0C5
:100D500001C086E1898310E0CE01F8DD812FDF91AB
:100D6000CF911F910F910895CF93DF931F92CDB72D
:100D7000DEB72091601830916118CE0101962115DF
:100D8000310519F0821B930B02C0865698410F90D3
:100D9000DF91CF910895FC01238121110C94CB9711
:100DA000089582E197E0F7CF8DE297E0F4CF80914C
:100DB000A609847F8B7F8093A60910925D0710920D
:100DC0005E0710925F071092600710926107109201
:100DD000620710926307109264071092D207109274
:100DE00011088EE091E0E2E1F8E0DF019C011D9244
:100DF00021503040E1F78FEF809356090895FC01B0
:100E000020E03EE2DB014C91403241F0283011F409
:100E100030833196DB014C91408331962F5F6F5FB9
:100E20007F4F2B3079F7108208952F923F924F9287
:100E30005F926F927F928F929F92AF92BF92CF926A
:100E4000DF92EF92FF920F931F93CF93DF93CDB773
:100E5000DEB7C356D1090FB6F894DEBF0FBECDBFC3
:100E60008C015B014A014DB65EB6312C7E0187E5EF
:100E7000E80EF11C9BE1292E47E559E0BE016F5FAA
:100E80007F4FC5010E943B9618160CF005C18C855A
:100E9000282F2871203109F074C090915C0791507F
:100EA000923008F46EC06DB67EB6BE016F5F7F4FA4
:100EB000C701A5DF0115110521F0F801808181111D
:100EC00073C021E081E090E0F70101900020E9F794
:100ED0003197EE19FF09E80FF91F32968DB79EB7CB
:100EE0008E1B9F0B0FB6F8949EBF0FBE8DBFEDB744
:100EF000FEB731966F01211102C0B80102C06DEB3F
:100F000073E0C6010F949F56B701C6010F9489562E
:100F10006DEB73E0C6010F9489561CAE1FAE21E045
:100F2000A701B501CE01CC960E94C79981110DC0D1
:100F300080915C07811109C00E94B8A282E295E30A
:100F40000E94AAA2C7010E9451A8FE01FC96DE01E0
:100F50009196822D01900D928A95E1F740E050E044
:100F6000BE016F5D7F4FC60160DFCE01819613DF4A
:100F7000CE01CC9610DF0FB6F8947EBE0FBE6DBECC
:100F80007BCF9981992309F487C0953E09F474CFEA
:100F90009E3209F471CF909157099E3209F46CCFBB
:100FA0008A7009F069CF0AC0F80101900020E9F7C2
:100FB0003197CF01801B910B20E086CF81E020315B
:100FC00009F080E09091A60980FB94F99093A6091E
:100FD000811108C08985873409F04ECF8A858E3704
:100FE00009F44ACF80915C07813021F068F08230AB
:100FF000B9F142CF80915A0790915B070196909387
:101000005B0780935A0738CFBE016F5F7F4F89E936
:1010100099E0F5DE0115110511F0680105C089E9B7
:10102000C82E89E0D82E08C0F60181916F0188236F
:10103000B1F30E94FAA7F8CFF60181916F018823DE
:1010400019F00E94FAA7F8CF80E20E94FAA76D8DEE
:101050007E8D8F8D98A14AE050E00E9407A90CCFA9
:10106000BE016F5F7F4F89E999E0C9DE8114910469
:1010700041F069E979E0C4010F947656892B51F467
:101080000BC0832D90E020915807309159078217AB
:10109000930711F03394F0CE0FB6F8945EBE0FBEF6
:1010A0004DBECD59DF4F0FB6F894DEBF0FBECDBF9A
:1010B000DF91CF911F910F91FF90EF90DF90CF9034
:1010C000BF90AF909F908F907F906F905F904F9068
:1010D0003F902F900895CF93DF93CDB7DEB76B97F6
:1010E0000FB6F894DEBF0FBECDBF10925C0740E094
:1010F00050E0BA018BE399E00E94EA968BE1EBE3C2
:10110000F9E0DE01119601900D928A95E1F740E039
:1011100050E0BE016F5F7F4F80E090E086DECE0141
:10112000019639DE6B960FB6F894DEBF0FBECDBFC9
:10113000DF91CF9108950F931F93CF93DF93CDB796
:10114000DEB72D970FB6F894DEBF0FBECDBF8091EE
:10115000D607882391F0BE016F5F7F4F83ED97E044
:101160000E945D948E010F5F1F4FF80181918F01E6
:10117000882339F00E94FAA7F8CF88E195E30E940E
:10118000AAA28AE00E94FAA72D960FB6F894DEBFB5
:101190000FBECDBFDF91CF911F910F910895CF92D8
:1011A000DF92EF92FF920F931F93CF93DF93CDB710
:1011B000DEB7EDB6FEB6DC010D900020E9F79D012B
:1011C000281B390B2C5F3F4F4DB75EB7421B530BAB
:1011D0000FB6F8945EBF0FBE4DBF0DB71EB70F5FC1
:1011E0001F4F9F938F9382ED94E39F938F931F9351
:1011F0000F930F94CE56680154E0C50ED11C0F908A
:101200000F900F900F900F900F90F6018081882320
:1012100049F0082E000C990B0F94FA55F6018193B2
:101220006F01F3CFC8010F94663D8EEC94E30F94E9
:10123000613D0FB6F894FEBE0FBEEDBEDF91CF91BB
:101240001F910F91FF90EF90DF90CF9008958091C4
:10125000A60983FF03C084608093A60908951092B5
:101260007B0C8091A6098F7D8B7F8093A6090E94BD
:10127000B362882321F083ED97E00C94CB97089517
:10128000EEDF8091A609877F8093A60908950F93CA
:101290001F93CF93DF938B01EA01DB016D917C916A
:1012A0000E945D94D801ED91FC919081888191110B
:1012B0000EC08936B0F48FE28083F801808191817D
:1012C00001969183808388818F5F88830AC08936E5
:1012D00080F73196D801ED93FC9388818F5F8883E6
:1012E000E1CFDF91CF911F910F9108950F931F933D
:1012F000CF93DF9300D0CDB7DEB79C012F5F3F4F78
:101300003B832A832FE2FC01208381E0898310E064
:101310000BE180911108181770F4019FC00111248E
:10132000AE014F5F5F4FBE016E5F7F4F8E5E974F86
:10133000AEDF1F5FEECF89818B3570F4AE014F5F5A
:101340005F4FBE016E5F7F4F83ED97E0A0DF8A8124
:101350009B8101979B838A83EA81FB8110820F9096
:101360000F900F90DF91CF911F910F910895809171
:10137000A60982FF1FC086E993E30E94AAA260919A
:101380005D0770915E0780915F07909160074AE06A
:1013900050E00E94FCA88FE20E94FAA760916107CA
:1013A0007091620780916307909164074AE050E072
:1013B0000C9407A985E893E30C94AAA2EF92FF92FC
:1013C0000F931F93CF93DF938C01FC0101900020BA
:1013D000E9F73197EF01C81BD90B1092D3076EE4E0
:1013E00070E00F9494567C01009729F4FE01319728
:1013F000E00FF11F0EC060E270E00F9494568C0174
:101400000F5F1F4F6AE270E0C7010F949456FC0112
:1014100031978DE081838AE082831382B80183ED66
:1014200097E00E945A9C8091D307882361F00E9424
:10143000BBA28EE693E3DF91CF911F910F91FF90B6
:10144000EF900C94AAA2DF91CF911F910F91FF9082
:10145000EF90089583ED97E00E94809783ED97E0E9
:101460000E94CB978091A6098D7F8E7F8093A609DD
:1014700010925D0710925E0710925F07109260074E
:1014800081E080936C0C08950F931F93CF93DF93AB
:10149000CDB7DEB76B970FB6F894DEBF0FBECDBFEA
:1014A0008B0122E020935C079093590780935807A3
:1014B00040E050E0BA0180E299E00E94EA968BE1B8
:1014C000E0E2F9E0DE01119601900D928A95E1F7D4
:1014D000A801BE016F5F7F4F80E090E0A6DCCE01E7
:1014E000019659DC6B960FB6F894DEBF0FBECDBFE8
:1014F000DF91CF911F910F910895CF93DF93CDB7D7
:10150000DEB76B970FB6F894DEBF0FBECDBF81E09C
:1015100080935C0710925B0710925A0740E050E0FE
:10152000BA0180E299E00E94EA968BE1E0E2F9E0FC
:10153000DE01119601900D928A95E1F740E050E0AE
:10154000BE016F5F7F4F80E090E06FDCCE010196BF
:1015500022DC80915A0790915B076B960FB6F89446
:10156000DEBF0FBECDBFDF91CF9108952F923F9286
:101570004F925F926F927F928F929F92AF92BF92A3
:10158000CF92DF92EF92FF920F931F93CF93DF934F
:1015900000D01F92CDB7DEB77C018B01342E2DB762
:1015A0003EB73C832B838091500781110BC0109272
:1015B0002D071092300781E08093500784ED96E864
:1015C0000E94EF388091480781110BC010921207DA
:1015D0001092150781E08093480781ED96E80E94FC
:1015E000EF38F80180818F3251F48BE399E0F701F5
:1015F00091838083109211080F5F1F4F05C080E216
:1016000099E0F70191838083F7010190F081E02D4B
:10161000FA83E9832DE2A22E27E0B22E3BE1232EAE
:101620000115110509F47FC04DB65EB66FE270E09A
:10163000C8010F9494563C010817190708F073C0AD
:101640006C01C01AD10ADD24C60101962DB73EB740
:10165000281B390B0FB6F8943EBF0FBE2DBF8DB7B8
:101660009EB701964C01A601B8010F94B456F4013F
:10167000EC0DFD1D1082332019F0C4010E9451A809
:10168000F7016081718121E0A401C5010E94C79921
:10169000811111C0B40181E593E30E94BEA28EE4E2
:1016A00093E30E94AAA20FB6F8945EBE0FBE4DBE91
:1016B00080E090E039C0F7018081918129813A81F1
:1016C0008217930711F00E94CB97F701B182A08295
:1016D000A0911108AA3078F481E08A0F8093110854
:1016E0002A9ED0011124AE5EB74FF501822D0190E4
:1016F0000D928A95E1F7F701808191818D52974093
:1017000029F492E1A92E97E0B92E04C08DE2A82E0B
:1017100087E0B82E83010F5F1F4F0FB6F8945EBEAF
:101720000FBE4DBE7DCFC8012B813C810FB6F89412
:101730003EBF0FBE2DBF0F900F900F900F90DF9107
:10174000CF911F910F91FF90EF90DF90CF90BF90BE
:10175000AF909F908F907F906F905F904F903F9051
:101760002F9008950F931F93CF93DF931F921F9293
:10177000CDB7DEB72091A60923FF28C0BC0140E009
:10178000CE010196F3DE8C01009701F1BC01898145
:101790009A810E94A19AB801882381F083EC93E397
:1017A0000E94BEA28AE00E94FAA710925D071092E2
:1017B0005E0710925F071092600708C08BEA93E300
:1017C0000E94BEA288EA93E30E94AAA20F900F9003
:1017D000DF91CF911F910F910895EF92FF920F9398
:1017E0001F93CF93DF9300D0CDB7DEB72091A6092A
:1017F00023FF09C1F42EE62E8C010E94B3628823D8
:1018000009F451C0FF2009F45BC08091D2078823FE
:1018100059F00E94BBA289E894E30E94AAA280E04A
:1018200090E00F94A34BEFC085E697E05FDDE09179
:10183000D20784E0E89FF0011124E253F84F809131
:101840005D0790915E07A0915F07B091600780836C
:101850009183A283B3830E94B8A2B80180E794E386
:101860000E94BEA28091D20799E6899FB0011124FF
:101870006B59784F85E694E30E94BEA240915D07C4
:1018800050915E0760915F07709160078FE594E368
:101890000E941FA38AE00E94FAA78091D2078F5F5F
:1018A0008093D20725C0FF2039F00E94B8A28FE4B0
:1018B00094E30E94AAA21CC01092D20722E001C0A9
:1018C00021E02B830E94B8A28AE494E30E94AAA29A
:1018D0002B81213009F494C08EE394E30E94AAA2E4
:1018E000B80186E394E30E94BEA28AE00E94FAA7B0
:1018F000B6DC40E0B801CE01019638DE8C010097DD
:1019000009F481C069817A81EE2009F44FC021E099
:10191000AC0183ED97E00E94C799882309F43EC08B
:101920008091E4079091E507A091E607B091E70761
:101930008093610790936207A0936307B093640755
:1019400010925D0710925E0710925F071092600779
:10195000B80188E294E30E94BEA2409161075091D1
:101960006207609163077091640780E294E30E94CC
:101970001FA38AE00E94FAA781E194E30E94AAA231
:10198000B80180E090E080DD80915709811102C0AC
:10199000C80102C087E599E060E02FC0B8018DEF73
:1019A00093E30E94BEA28AEF93E30FC026E5AC0149
:1019B00083ED97E00E94C79981110AC0B80186EEB5
:1019C00093E30E94BEA283EE93E30E94AAA21BC0EF
:1019D0008091A60981608093A609B80180E090E01B
:1019E00053DD10926C0CB80181ED93E30E94BEA20E
:1019F0008AE00E94FAA760E0C8010E94F68003C056
:101A000084E494E36BCF0F900F900F90DF91CF9110
:101A10001F910F91FF90EF9008952091A6092260E9
:101A20002093A60940E060E0D8CE0F931F93CF9398
:101A3000DF93CDB7DEB76B970FB6F894DEBF0FBE5E
:101A4000CDBF8C0119821C8280912309811103C0B2
:101A50006BE379E002C060E279E021E0A801CE0109
:101A600001960E94C7998823F1F08BE1FE0131961F
:101A7000A0E2B9E001900D928A95E1F7A0911108DA
:101A8000AA30D8F481E08A0F809311088BE18A9FF5
:101A9000D0011124AE5EB74FE0E2F9E001900D9263
:101AA0008A95E1F70AC00E94B8A2B80188E393E3DF
:101AB0000E94BEA28AE00E94FAA7CE0101966BD9CD
:101AC0006B960FB6F894DEBF0FBECDBFDF91CF91FE
:101AD0001F910F910895809111088823C9F08150BA
:101AE00080931108882359F090E001972BE1289FFB
:101AF000F001299FF00D1124EE5EF74F02C0EBE3D9
:101B0000F9E08BE1A0E2B9E001900D928A95E1F74E
:101B10008091110808958BE1EBE3F9E0A0E2B9E0D0
:101B200001900D928A95E1F708958091A609877F2B
:101B30008093A60980913E09882321F08BE399E0E8
:101B40000E94CB9745E360E08CE098E00E946785B7
:101B5000811105C00E94B8A28AE095E32AC041E045
:101B60006CE078E08EEE97E07FD481110DC040E00C
:101B70006CE078E08EEE97E077D4811105C00E948A
:101B8000BBA286EF94E315C06EEE77E08BE399E09D
:101B9000F0D6811105C00E94BBA285EE94E309C076
:101BA0008091A60988608093A6090E94B8A289ED59
:101BB00094E30E94AAA2AFDF83E0809323020895FA
:101BC000AF92BF92CF92DF92EF92FF921F93CF938B
:101BD000DF93CDB7DEB7A8970FB6F894DEBF0FBE80
:101BE000CDBF8091560987FD61C08091A60982FD15
:101BF0005DC083FF9ADF8091A60983FF54C0809166
:101C00005609082E000C990BC0969F938F9385E67A
